:100000000000032099DA00007DDA000035DA0000F4
:1000100035DA000035DA000035DA000035DA0000A4
:1000200035DA000035DA000035DA00007DDA00004C
:100030007DDA000035DA000055CF0000CDD1000098
:100040007DDA00007DDA00007DDA00007DDA000054
:100050007DDA00007DDA00007DDA00007DDA000044
:100060007DDA00007DDA00007DDA00007DDA000034
:100070007DDA00007DDA00007DDA00007DDA000024
:100080007DDA00007DDA00007DDA00007DDA000014
:100090007DDA00007DDA00007DDA00007DDA000004
:1000A00009A1000065A200007DDA00007DDA0000F1
:1000B0007DDA00007DDA00007DDA0000B5EB00009B
:1000C0007DDA0000790101007DDA0000D50201002F
:1000D0007DDA0000050401007DDA00007DDA000011
:1000E0007DDA00007DDA00007DDA00007DDA0000B4
:1000F0007DDA00007DDA00007DDA00007DDA0000A4
:100100007DDA00007DDA00007DDA00007DDA000093
:100110007DDA0000E9EE00007DDA00007DDA000003
:100120007DDA00007DDA00007DDA00007DDA000073
:100130007DDA00007DDA00007DDA00007DDA000063
:10014000A1CC00007DDA0000350501007DDA000059
:100150007DDA00007DDA00007DDA00007DDA000043
:100160007DDA00007DDA0000C1A300007DDA000026
:100170007DDA00007DDA00007DDA00007DDA000023
:100180007DDA00007DDA00007DDA00007DDA000013
:100190007DDA00007DDA0000650601007DDA0000EE
:1001A0007DDA00007DDA00007DDA00007DDA0000F3
:1001B0007DDA00007DDA00007DDA00007DDA0000E3
:1001C0007DDA00007DDA00007DDA00007DDA0000D3
:1001D000FFFFFFFFFFFFFFFFFFFFFFFFFFFFFFFF2F
:10040000FFFFFFFFFFFFFFFFFFFFFFFFDEF9FFFF23
:1004100010B5054C237833B9044B13B10448AFF33E
:1004200000800123237010BD00B0FF1F00000000FA
:100430008C260E00084B10B51BB108490848AFF3D5
:1004400000800848036803B910BD074B002BFBD0A0
:10045000BDE81040184700BF0000000004B0FF1FB7
:100460008C260E0044A1FF1F00000000704700BF53
:10047000704700BF704700BF10B504460CF0C6FBC4
:10048000204610BD43F24040F8B51B21C0F20100E8
:100490000FF076FC4BF69023C1F6FF73FF21986CAA
:1004A00003681B68984743F25C400F21C0F20100CB
:1004B0000FF066FC4BF26C03C1F6FF73FF219B6CDF
:1004C0001A691F46501C1861117057F8106FBE4210
:1004D00024BF1B611E464FF0010E4FF0000C5A69FD
:1004E000B24202F1010113D0596110785A6B8F4268
:1004F0004FEA201598BF5B619C18511CBAB95A6924
:1005000083F83050B242C3F834E002F10101EBD17C
:1005100043F26C40C0F201000F210FF031FC49F6AC
:100520001400C1F6FF70BDE8F8400CF043BF03298A
:1005300084F830005963D2D1C3F830C0C3F834C056
:10054000CDE700BF43F27C40F8B51D21C0F20100A9
:100550000FF016FC4BF69023C1F6FF73FE21986C4A
:1005600003681B68984743F25C400F21C0F201000A
:100570000FF006FC4BF26C03C1F6FF73FE219B6C7F
:100580001A691F46501C1861117057F8106FBE424F
:1005900024BF1B611E464FF0010E4FF0000C5A693C
:1005A000B24202F1010113D0596110785A6B8F42A7
:1005B0004FEA201598BF5B619C18511CBAB95A6963
:1005C00083F83050B242C3F834E002F10101EBD1BC
:1005D00043F26C40C0F201000F210FF0D1FB49F64D
:1005E0001400C1F6FF70BDE8F8400CF0E3BE03292B
:1005F00084F830005963D2D1C3F830C0C3F834C096
:10060000CDE700BF43F29C40F8B51421C0F20100D1
:100610000FF0B6FB4BF69023C1F6FF73FC21986CEC
:1006200003681B68984743F25C400F21C0F2010049
:100630000FF0A6FB4BF26C03C1F6FF73FC219B6C21
:100640001A691F46501C1861117057F8106FBE428E
:1006500024BF1B611E464FF0010E4FF0000C5A697B
:10066000B24202F1010113D0596110785A6B8F42E6
:100670004FEA201598BF5B619C18511CBAB95A69A2
:1006800083F83050B242C3F834E002F10101EBD1FB
:1006900043F26C40C0F201000F210FF071FB49F6EC
:1006A0001400C1F6FF70BDE8F8400CF083BE0329CA
:1006B00084F830005963D2D1C3F830C0C3F834C0D5
:1006C000CDE700BF43F2B440F8B51821C0F20100F5
:1006D0000FF056FB4BF69023C1F6FF73FB21986C8D
:1006E00003681B68984743F25C400F21C0F2010089
:1006F0000FF046FB4BF26C03C1F6FF73FB219B6CC2
:100700001A691F46501C1861117057F8106FBE42CD
:1007100024BF1B611E464FF0010E4FF0000C5A69BA
:10072000B24202F1010113D0596110785A6B8F4225
:100730004FEA201598BF5B619C18511CBAB95A69E1
:1007400083F83050B242C3F834E002F10101EBD13A
:1007500043F26C40C0F201000F210FF011FB49F68B
:100760001400C1F6FF70BDE8F8400CF023BE032969
:1007700084F830005963D2D1C3F830C0C3F834C014
:10078000CDE700BF43F2D040F8B51521C0F201001B
:100790000FF0F6FA4BF69023C1F6FF73F821986C30
:1007A00003681B68984743F25C400F21C0F20100C8
:1007B0000FF0E6FA4BF26C03C1F6FF73F8219B6C65
:1007C0001A691F46501C1861117057F8106FBE420D
:1007D00024BF1B611E464FF0010E4FF0000C5A69FA
:1007E000B24202F1010113D0596110785A6B8F4265
:1007F0004FEA201598BF5B619C18511CBAB95A6921
:1008000083F83050B242C3F834E002F10101EBD179
:1008100043F26C40C0F201000F210FF0B1FA49F62B
:100820001400C1F6FF70BDE8F8400CF0C3BD032909
:1008300084F830005963D2D1C3F830C0C3F834C053
:10084000CDE700BF43F2E840F8B51521C0F2010042
:100850000FF096FA4BF69023C1F6FF73FA21986CCD
:1008600003681B68984743F25C400F21C0F2010007
:100870000FF086FA4BF26C03C1F6FF73FA219B6C02
:100880001A691F46501C1861117057F8106FBE424C
:1008900024BF1B611E464FF0010E4FF0000C5A6939
:1008A000B24202F1010113D0596110785A6B8F42A4
:1008B0004FEA201598BF5B619C18511CBAB95A6960
:1008C00083F83050B242C3F834E002F10101EBD1B9
:1008D00043F26C40C0F201000F210FF051FA49F6CB
:1008E0001400C1F6FF70BDE8F8400CF063BD0329A9
:1008F00084F830005963D2D1C3F830C0C3F834C093
:10090000CDE700BF2DE9F843044643F2005015211E
:10091000C0F201000FF034FA210401F4FE0141F4A9
:1009200073414BF2203041F00201C1F6FF704BF2EF
:100930006C080BF011FCC1F6FF7843F2185014213B
:10094000C0F201000FF01CFAD8F848301A699E4630
:10095000F321501C186111705EF8107F774524BF99
:100960001B611F464FF0010C4FF000095A69BA4253
:1009700002F1010114D0596110785A6B8E454FEA8B
:10098000201698BF5B619D18511C002A43D15A69FB
:1009900083F83060BA42C3F834C002F10101EAD1F1
:1009A000D8F848301A691F4604F07F04511C1961B9
:1009B000147057F8106FBE4224BF1B611E464FF0E3
:1009C000010E4FF0000C5A69B24202F1010113D03E
:1009D000596110785A6B8F424FEA201598BF5B61BE
:1009E0009C18511C0ABB5A6983F83050B242C3F8B4
:1009F00034E002F10101EBD143F26C40C0F201009E
:100A00000F210FF0BDF949F61400C1F6FF70BDE8E3
:100A1000F8430CF0CFBC032985F830005963A5D109
:100A2000C3F83090C3F83490A0E7032984F830006D
:100A30005963C8D1C3F830C0C3F834C0C3E700BF9E
:100A400043F2305008B51321C0F201000FF098F9BD
:100A50004BF69023C1F6FF73FB21986C03681B686B
:100A6000984743F25C400F21C0F201000FF088F973
:100A70004BF22030C1F6FF704FF60F310BF06CFBDC
:100A800043F21850C0F2010014210FF079F949F631
:100A90001400C1F6FF70BDE808400CF08BBC00BF2D
:100AA00043F2445008B51821C0F201000FF068F974
:100AB0004BF69023C1F6FF73FE21986C03681B6808
:100AC000984743F25C400F21C0F201000FF058F943
:100AD0004BF22030C1F6FF704FF60F610BF03CFB7C
:100AE00043F21850C0F2010014210FF049F949F601
:100AF0001400C1F6FF70BDE808400CF05BBC00BFFD
:100B000043F2605008B50F21C0F201000FF038F930
:100B10004BF69023C1F6FF73FC21986C03681B68A9
:100B2000984743F25C400F21C0F201000FF028F912
:100B30004BF22030C1F6FF704FF60F410BF00CFB6B
:100B400043F21850C0F2010014210FF019F949F6D0
:100B50001400C1F6FF70BDE808400CF02BBC00BFCC
:100B600043F2705008B51021C0F201000FF008F9EF
:100B70004BF69023C1F6FF73FA21986C03681B684B
:100B8000984743F25C400F21C0F201000FF0F8F8E3
:100B90004BF22030C1F6FF704FF60F210BF0DCFA5C
:100BA00043F21850C0F2010014210FF0E9F849F6A1
:100BB0001400C1F6FF70BDE808400CF0FBBB00BF9D
:100BC00043F28450F8B51621C0F201000FF0D8F8B6
:100BD0004BF22030C1F6FF704FF60F710BF0BCFAEC
:100BE00043F218501421C0F201000FF0C9F84BF283
:100BF0006C03C1F6FF73FF219B6C1A691F46501CE2
:100C00001861117057F8106FBE4224BF1B611E4659
:100C10004FF0010E4FF0000C5A69964202F10101AB
:100C200013D0596110785A6B8F424FEA201598BF44
:100C30005B619C18511CBAB95A6983F830509642CE
:100C4000C3F834E002F10101EBD143F26C40C0F291
:100C500001000F210FF094F849F61400C1F6FF705F
:100C6000BDE8F8400CF0A6BB032984F830005963B6
:100C7000D2D1C3F830C0C3F834C0CDE743F29C50A2
:100C800008B51021C0F201000FF07AF84BF690235E
:100C9000C1F6FF73F821986C03681B68984743F20C
:100CA0005C400F21C0F201000FF06AF84BF22030D7
:100CB000C1F6FF704FF60F010BF04EFA43F21850D9
:100CC000C0F2010014210FF05BF849F61400C1F6E0
:100CD000FF70BDE808400CF06DBB00BF43F2B050A0
:100CE00008B51621C0F201000FF04AF84BF6902328
:100CF000C1F6FF73FF21986C03681B68984743F2A5
:100D00005C400F21C0F201000FF03AF84BF22030A6
:100D1000C1F6FF704FF60F710BF01EFA43F2185038
:100D2000C0F2010014210FF02BF849F61400C1F6AF
:100D3000FF70BDE808400CF03DBB00BF43F2C85057
:100D4000F8B51821C0F201000FF01AF84BF220306C
:100D5000C1F6FF704FF60F610BF0FEF943F2185029
:100D60001421C0F201000FF00BF84BF26C03C1F636
:100D7000FF73FE219B6C1A691F46501C186111708D
:100D800057F8106FBE4224BF1B611E464FF0010E84
:100D90004FF0000C5A69964202F1010113D05961DB
:100DA00010785A6B8F424FEA201598BF5B619C18F0
:100DB000511CBAB95A6983F830509642C3F834E0EE
:100DC00002F10101EBD143F26C40C0F201000F21AE
:100DD0000EF0D6FF49F61400C1F6FF70BDE8F840EA
:100DE0000CF0E8BA032984F830005963D2D1C3F873
:100DF00030C0C3F834C0CDE743F2E450F8B50F215A
:100E0000C0F201000EF0BCFF4BF22030C1F6FF70C3
:100E10004FF60F410BF0A0F943F218501421C0F225
:100E200001000EF0ADFF4BF26C03C1F6FF73FC2125
:100E30009B6C1A691F46501C1861117057F8106F8F
:100E4000BE4224BF1B611E464FF0010E4FF0000C46
:100E50005A69964202F1010113D0596110785A6B18
:100E60008F424FEA201598BF5B619C18511CBAB99C
:100E70005A6983F830509642C3F834E002F1010118
:100E8000EBD143F26C40C0F201000F210EF078FF6D
:100E900049F61400C1F6FF70BDE8F8400CF08ABABC
:100EA000032984F830005963D2D1C3F830C0C3F8A5
:100EB00034C0CDE743F2F450F8B51021C0F2010080
:100EC0000EF05EFF4BF22030C1F6FF704FF60F219F
:100ED0000BF042F943F218501421C0F201000EF059
:100EE0004FFF4BF26C03C1F6FF73FA219B6C1A693A
:100EF0001F46501C1861117057F8106FBE4224BF76
:100F00001B611E464FF0010E4FF0000C5A699642CD
:100F100002F1010113D0596110785A6B8F424FEAE8
:100F2000201598BF5B619C18511CBAB95A6983F8A7
:100F300030509642C3F834E002F10101EBD143F2A4
:100F40006C40C0F201000F210EF01AFF49F61400A8
:100F5000C1F6FF70BDE8F8400CF02CBA032984F804
:100F600030005963D2D1C3F830C0C3F834C0CDE7E4
:100F700043F20860F8B51321C0F201000EF000FF43
:100F80004BF22030C1F6FF704FF60F310BF0E4F852
:100F900043F218501421C0F201000EF0F1FE4BF2A2
:100FA0006C03C1F6FF73FB219B6C1A691F46501C32
:100FB0001861117057F8106FBE4224BF1B611E46A6
:100FC0004FF0010E4FF0000C5A69964202F10101F8
:100FD00013D0596110785A6B8F424FEA201598BF91
:100FE0005B619C18511CBAB95A6983F8305096421B
:100FF000C3F834E002F10101EBD143F26C40C0F2DE
:1010000001000F210EF0BCFE49F61400C1F6FF707E
:10101000BDE8F8400CF0CEB9032984F830005963DC
:10102000D2D1C3F830C0C3F834C0CDE743F21C605E
:10103000F8B51021C0F201000EF0A2FE4BF22030F4
:10104000C1F6FF704FF60F010BF086F843F218500F
:101050001421C0F201000EF093FE4BF26C03C1F6B6
:10106000FF73F8219B6C1A691F46501C18611170A0
:1010700057F8106FBE4224BF1B611E464FF0010E91
:101080004FF0000C5A69964202F1010113D05961E8
:1010900010785A6B8F424FEA201598BF5B619C18FD
:1010A000511CBAB95A6983F830509642C3F834E0FB
:1010B00002F10101EBD143F26C40C0F201000F21BB
:1010C0000EF05EFE49F61400C1F6FF70BDE8F84070
:1010D0000CF070B9032984F830005963D2D1C3F8F9
:1010E00030C0C3F834C0CDE72DE9F0414BF6902570
:1010F0008046C1F6FF7543F230600F46C0F2010032
:1011000010210EF03DFEA86C0368F021DB6C9847BF
:1011100057B1444608EB0706A86C14F8011B036896
:101120001B689847A642F7D1A86C0368F721DB6CCF
:10113000984743F25C400F21C0F201000EF020FE00
:101140004BF220303A464146C1F6FF7000230BF0C7
:1011500041F843F21850C0F2010014210EF010FEC5
:1011600049F61400C1F6FF70BDE8F0410CF022B959
:101170002DE9F843044643F244601F21C0F2010008
:101180000EF0FEFD04F00F034FF202111B04C0F23B
:1011900010014BF220301943C1F6FF704BF26C087E
:1011A0000AF0DAFFC1F6FF7843F218501421C0F2BA
:1011B00001000EF0E5FDD8F848301A699E46F1218D
:1011C000501C186111705EF8107F774524BF1B61B9
:1011D0001F464FF0010C4FF000095A69BA4202F164
:1011E000010114D0596110785A6B8E454FEA2016D0
:1011F00098BF5B619D18511C002A41D15A6983F840
:101200003060BA42C3F834C002F10101EAD1D8F823
:1012100048301A691F46511C1961147057F8106F35
:10122000BE4224BF1B611E464FF0010E4FF0000C62
:101230005A69B24202F1010113D0596110785A6B18
:101240008F424FEA201598BF5B619C18511C0ABB66
:101250005A6983F83050B242C3F834E002F1010118
:10126000EBD143F26C40C0F201000F210EF088FD7B
:1012700049F61400C1F6FF70BDE8F8430CF09AB8C7
:10128000032985F830005963A7D1C3F83090C3F81B
:101290003490A2E7032984F830005963C8D1C3F819
:1012A00030C0C3F834C0C3E743F2646008B5162108
:1012B000C0F201000EF064FD4BF69023C1F6FF73FF
:1012C000F621986C0368DB6C984743F25C400F2171
:1012D000C0F201000EF054FD4BF22030C1F6FF7059
:1012E0004FF20F610AF038FF43F21850C0F20100CC
:1012F00014210EF045FD49F61400C1F6FF70BDE85B
:1013000008400CF057B800BF70B5054643F27C604A
:101310000C46013D0D21C0F201000EF031FDE9B295
:101320000F290FD84BF69026C1F6FF7641F0C00189
:10133000B06C03681B689847B06C036804F07F01C9
:101340001B68984743F25C400F21C0F201000EF089
:1013500017FD230403F4FE03290243F4404343F042
:101360000C0301F470614BF220301943C1F6FF7099
:101370000AF0F2FE43F21850C0F2010014210EF000
:10138000FFFC49F61400C1F6FF70BDE870400CF098
:1013900011B800BF70B5054643F28C600C46013DA4
:1013A0000D21C0F201000EF0EBFCE9B20F290FD8BD
:1013B0004BF69026C1F6FF7641F0D001B06C036881
:1013C0001B689847B06C036804F07F011B6898475E
:1013D00043F25C400F21C0F201000EF0D1FC230467
:1013E00003F4FE03290243F4504343F00D0301F4D8
:1013F00070614BF220301943C1F6FF700AF0ACFE69
:1014000043F21850C0F2010014210EF0B9FC49F665
:101410001400C1F6FF70BDE870400BF0CBBF00BFF9
:10142000F8B5064643F29C600C46C0F2010012215A
:1014300015460EF0A5FC711EC9B20F2915D84BF642
:101440009027C1F6FF7741F0A001B86C03681B68D4
:101450009847B86C036804F07F011B689847B86C24
:10146000036805F07F011B68984743F2B0600A21CA
:10147000C0F201000EF084FC6B1E1B02240404F475
:10148000FE0403F470632343310143F4504343F0FB
:101490000D03C9B24BF220301943C1F6FF700AF0B8
:1014A0005BFE43F21850C0F2010014210EF068FCFC
:1014B00049F61400C1F6FF70BDE8F8400BF07ABFA2
:1014C00043F2BC60F8B51621C0F201000EF058FCE2
:1014D0004BF22030C1F6FF704FF20F610AF03CFE74
:1014E00043F218501421C0F201000EF049FC4BF2F7
:1014F0006C03C1F6FF73F6219B6C1A691F46501CE2
:101500001861117057F8106FBE4224BF1B611E4650
:101510004FF0010E4FF0000C5A69B24202F1010186
:1015200013D0596110785A6B8F424FEA201598BF3B
:101530005B619C18511CBAB95A6983F83050B242A9
:10154000C3F834E002F10101EBD143F26C40C0F288
:1015500001000F210EF014FC49F61400C1F6FF70D3
:10156000BDE8F8400BF026BF032984F8300059632A
:10157000D2D1C3F830C0C3F834C0CDE7F8B50546C2
:1015800043F2D4600C46013D0D21C0F201000EF083
:10159000F7FBE9B20F2917D84BF69026C1F6FF7674
:1015A00041F0E001B06C03681B689847B06C0368B9
:1015B00004F500571B6807F07F019847B06C03687B
:1015C000C7F3C6111B68984743F25C400F21C0F275
:1015D00001000EF0D5FB04F30D0303F500532902BF
:1015E0001A0402F4FE0201F47061114341F46041F7
:1015F0005B0403F0FE4341F00E014BF2203019432F
:10160000C1F6FF700AF0A8FD43F21850C0F20100C5
:1016100014210EF0B5FB49F61400C1F6FF70BDE8C9
:10162000F8400BF0C7BE00BF43F2E460F8B51B21E1
:10163000C0F201000EF0A4FB4BF69023C1F6FF733D
:10164000F621986C0368DB6C984743F25C400F21ED
:10165000C0F201000EF094FB4BF26C03C1F6FF7375
:10166000F6219B6C1A691F46501C1861117057F8BF
:10167000106FBE4224BF1B611E464FF0010E4FF09B
:10168000000C5A69B24202F1010113D0596110787D
:101690005A6B8F424FEA201598BF5B619C18511C12
:1016A000BAB95A6983F83050B242C3F834E002F153
:1016B0000101EBD143F26C40C0F201000F210EF0AA
:1016C0005FFB49F61400C1F6FF70BDE8F8400BF06F
:1016D00071BE032984F830005963D2D1C3F830C0F9
:1016E000C3F834C0CDE700BF2DE9F8434BF6902591
:1016F0000446C1F6FF7543F200702421C0F20100D8
:101700000EF03EFBA86C0368F1211B689847A86C9B
:10171000036821461B684BF26C089847C1F6FF78B6
:1017200043F25C400F21C0F201000EF029FBD8F813
:1017300048301A699E46F121501C186111705EF8FC
:10174000107F774524BF1B611F464FF0010C4FF0FF
:1017500000095A69BA4202F1010114D059611078A6
:101760005A6B8E454FEA201698BF5B619D18511C3D
:10177000002A41D15A6983F83060BA42C3F834C0B4
:1017800002F10101EAD1D8F848301A691F46511C0C
:101790001961147057F8106FBE4224BF1B611E46BA
:1017A0004FF0010E4FF0000C5A69B24202F10101F4
:1017B00013D0596110785A6B8F424FEA201598BFA9
:1017C0005B619C18511C0ABB5A6983F83050B242C5
:1017D000C3F834E002F10101EBD143F26C40C0F2F6
:1017E00001000F210EF0CCFA49F61400C1F6FF708B
:1017F000BDE8F8430BF0DEBD032985F830005963DE
:10180000A7D1C3F83090C3F83490A2E7032984F835
:1018100030005963C8D1C3F830C0C3F834C0C3E73F
:101820002DE9F0474BF690270646C1F6FF7743F2C5
:1018300028700D46C0F2010015210EF0A1FAB86C17
:101840000368F021DB6C984755B1344606EB050878
:10185000B86C14F8011B03681B6898474445F7D11E
:10186000B86C0368F721DB6C4BF26C089847C1F643
:10187000FF7843F25C400F21C0F201000EF080FAC5
:10188000D8F848301A691F46501CF02118611170B1
:1018900057F8102FBA42C0F0A0801B619E464FF04F
:1018A000010C4FF000095A69724502F1010114D090
:1018B000596110785A6B8F424FEA201A98BF5B61CA
:1018C0009C18511C002A7DD15A6983F830A07245BA
:1018D000C3F834C002F10101EAD17DB3B64606EB8C
:1018E000050901274FF0000CD8F848301EF8011BFD
:1018F0001A691E46501C1861117056F8105FB542E7
:1019000024BF1B611D465A69AA4202F1010113D08E
:10191000596110785A6B8E424FEA201A98BF5B616A
:101920009C18511C002A5AD15A6983F830A0AA4247
:101930005F6302F10101EBD1F145D5D1D8F8483010
:101940001A691E46F721501C1861117056F8107F55
:10195000B74201D31B611F464FF0010E4FF0000C40
:101960005A69BA4202F1010113D0596110785A6BD9
:101970008E424FEA201598BF5B619C18511CBAB982
:101980005A6983F83050BA42C3F834E002F10101D9
:10199000EBD143F26C40C0F201000F210EF0F0F9E0
:1019A00049F61400C1F6FF70BDE8F0470BF002BD28
:1019B000032984F830005963D2D1C3F830C0C3F88A
:1019C00034C0CDE7032984F8300059637FF46BAF4E
:1019D000C3F83090C3F8349065E796465FE7032973
:1019E00084F8300059638ED1C3F830C0C3F834C0D6
:1019F00089E700BF2DE9F047054643F240700C46E9
:101A0000C0F2010010210EF0BBF94BF2203022464B
:101A100000232946C1F6FF704BF26C080AF0DAFB8E
:101A2000C1F6FF7843F218501421C0F201000EF005
:101A3000A7F9D8F848301A691F46501CF0211861E0
:101A4000117057F8102FBA4226BF1B619E4696466A
:101A50004FF0010C4FF000095A69724502F1010183
:101A600014D0596110785A6B8F424FEA201A98BFF0
:101A70005B619E18511C002A7DD15A6983F830A001
:101A80007245C3F834C002F10101EAD17CB3AE461D
:101A900005EB040901274FF0000CD8F848301EF878
:101AA000011B1A691E46501C1861117056F8105F10
:101AB000B54224BF1B611D465A69AA4202F10101C9
:101AC00013D0596110785A6B8E424FEA201A98BF92
:101AD0005B619C18511C002A58D15A6983F830A0C8
:101AE000AA425F6302F10101EBD1CE45D5D1D8F80E
:101AF00048301A691E46F721501C1861117056F8BB
:101B0000107FB74201D31B611F464FF0010E4FF00B
:101B1000000C5A69BA4202F1010113D059611078E0
:101B20005A6B8E424FEA201598BF5B619C18511C7E
:101B3000BAB95A6983F83050BA42C3F834E002F1B6
:101B40000101EBD143F26C40C0F201000F210EF015
:101B500017F949F61400C1F6FF70BDE8F0470BF025
:101B600029BC032984F830005963D2D1C3F830C0AE
:101B7000C3F834C0CDE7032986F8300059637FF4F9
:101B80006BAFC3F83090C3F8349065E7032984F84D
:101B90003000596390D1C3F830C0C3F834C08BE72C
:101BA0002DE9F8434BF690240746C1F6FF7443F243
:101BB00054701A21C0F201000EF0E2F8A06C036824
:101BC000F3211B689847A06C036807F07F07DB6C64
:101BD00039464BF26C089847C1F6FF7843F25C40F7
:101BE0000F21C0F201000EF0CBF8D8F848301A6986
:101BF0009E46501CF321186111705EF8100F70455D
:101C000024BF1B6118464FF0010C4FF000095A69C0
:101C1000824202F1010114D0596114785A6B8E4549
:101C20004FEA241698BF5B619D18511C002A3FD1D2
:101C30005A6983F830608242C3F834C002F101016E
:101C4000EAD1D8F848301A699E46511C19611770BC
:101C50005EF8106F764524BF1B611E4601274FF0CA
:101C6000000C5A69B24202F1010112D05961107898
:101C70005A6B8E454FEA201598BF5B619C18511C2A
:101C800002BB5A6983F83050B2425F6302F101012E
:101C9000ECD143F26C40C0F201000F210EF070F85D
:101CA00049F61400C1F6FF70BDE8F8430BF082BBA3
:101CB000032985F830405963A9D1C3F83090C3F89F
:101CC0003490A4E7032984F830005963C9D1C3F8DC
:101CD00030C0C3F834C0C4E738B54BF6902504468D
:101CE000C1F6FF7543F270701521C0F201000EF0CD
:101CF00047F8A86C0368F3211B689847A86C036831
:101D000004F07F01DB6C984743F25C400F21C0F286
:101D100001000EF035F8210401F4FE0141F4734195
:101D20004BF2203041F00201C1F6FF700AF014FAC4
:101D300043F21850C0F2010014210EF021F849F6C8
:101D40001400C1F6FF70BDE838400BF033BB00BF94
:101D500038B54BF690250446C1F6FF7543F28870FE
:101D60001F21C0F201000EF00BF8A86C0368F121EE
:101D70001B689847A86C036821461B68984743F284
:101D80005C400F21C0F2010004F00F040DF0F8FFD9
:101D900044F010044FF202114BF2203041EA0441AA
:101DA000C1F6FF700AF0D8F943F21850C0F20100F2
:101DB00014210DF0E5FF49F61400C1F6FF70BDE8EF
:101DC00038400BF0F7BA00BF2DE9F843044643F260
:101DD000A8700F46C0F2010012210DF0D1FF601E65
:101DE000C0B20F2800F293804BF69025C1F6FF7524
:101DF00040F0D004A86C036821461B689847A86C83
:101E0000036807F07F071B683946984743F25C4038
:101E10000F21C0F201000DF0B3FF4BF26C0CC1F6C4
:101E2000FF7C4FF00108DCF848301A699E46511CCF
:101E3000196114705EF8101F714524BF1B611946AB
:101E40004FF000095A69914202F1010014D0586123
:101E500014785A6B86454FEA241698BF5B619D182B
:101E6000501C002A3FD15A6983F830609142C3F870
:101E7000348002F10100EAD1DCF848301A699E464C
:101E8000511C196117705EF8106F764524BF1B61F5
:101E90001E4601274FF0000C5A69964202F10101DB
:101EA00012D0596110785A6B8E454FEA201598BFB1
:101EB0005B619C18511C02BB5A6983F830509642F2
:101EC0005F6302F10101ECD143F26C40C0F201000A
:101ED0000F210DF055FF49F61400C1F6FF70BDE863
:101EE000F8430BF067BA032885F830405863A9D14E
:101EF000C3F83090C3F83490A4E7032984F8300085
:101F00005963C9D1C3F830C0C3F834C0C4E743F241
:101F10005C400F21C0F201000DF032FFD4E700BF9A
:101F20002DE9F843044643F2BC700F46C0F20100AD
:101F300012210DF025FF601EC0B20F2800F2938021
:101F40004BF69025C1F6FF7540F0C004A86C0368FD
:101F500021461B689847A86C036807F07F071B6839
:101F60003946984743F25C400F21C0F201000DF062
:101F700007FF4BF26C0CC1F6FF7C4FF00108DCF858
:101F800048301A699E46511C196114705EF8101F82
:101F9000714524BF1B6119464FF000095A699142EF
:101FA00002F1010014D0586114785A6B86454FEA4B
:101FB000241698BF5B619D18501C002A3FD15A69B6
:101FC00083F830609142C3F8348002F10100EAD115
:101FD000DCF848301A699E46511C196117705EF88A
:101FE000106F764524BF1B611E4601274FF0000C81
:101FF0005A69964202F1010112D0596110785A6B68
:102000008E454FEA201598BF5B619C18511C02BB9E
:102010005A6983F8305096425F6302F10101ECD1B6
:1020200043F26C40C0F201000F210DF0A9FE49F609
:102030001400C1F6FF70BDE8F8430BF0BBB90328EC
:1020400085F830405863A9D1C3F83090C3F8349074
:10205000A4E7032984F830005963C9D1C3F830C01C
:10206000C3F834C0C4E743F25C400F21C0F2010062
:102070000DF086FED4E700BF2DE9F843044643F295
:10208000D0700D46C0F201000D210DF079FE2B0439
:10209000013C03F4FE03210243F4504343F00D03DB
:1020A00001F470614BF220301943C1F6FF700AF061
:1020B00053F843F21850C0F201001421E4B20DF0BD
:1020C0005FFE0F2C5BD84BF26C0EC1F6FF7E64F006
:1020D0002F04DEF848301A699C46511C19611470AF
:1020E0005CF8107F674505F07F0824BF1B611F4621
:1020F00001254FF000095A69974202F1010013D0FF
:10210000586114785A6B84454FEA241698BF5B6176
:102110009918501C002A41D15A6983F830609742BF
:102120005D6302F10100EBD1DEF848301A691F4609
:10213000511C196182F8008057F8106FBE4224BF0D
:102140001B611E464FF0010E4FF0000C5A6996427B
:1021500002F1010113D0596110785A6B8F424FEA96
:10216000201598BF5B619C18511C0ABB5A6983F803
:1021700030509642C3F834E002F10101EBD143F252
:102180006C40C0F201000F210DF0FAFD49F6140079
:10219000C1F6FF70BDE8F8430BF00CB9032881F8D5
:1021A00030405863A7D1C3F83090C3F83490A2E709
:1021B000032984F830005963C8D1C3F830C0C3F88C
:1021C00034C0C3E72DE9F843044643F2E0700D46FE
:1021D000C0F201000D210DF0D3FD2B04013C03F4EE
:1021E000FE03210243F4404343F00C0301F4706109
:1021F0004BF220301943C1F6FF7009F0ADFF43F2F6
:102200001850C0F201001421E4B20DF0B9FD0F2CFA
:102210005BD84BF26C0EC1F6FF7E64F03F04DEF833
:1022200048301A699C46511C196114705CF8107F83
:10223000674505F07F0824BF1B611F4601254FF04D
:1022400000095A69974202F1010013D058611478CD
:102250005A6B84454FEA241698BF5B619918501C4D
:10226000002A41D15A6983F8306097425D6302F1D8
:102270000100EBD1DEF848301A691F46511C196184
:1022800082F8008057F8106FBE4224BF1B611E46C3
:102290004FF0010E4FF0000C5A69964202F1010115
:1022A00013D0596110785A6B8F424FEA201598BFAE
:1022B0005B619C18511C0ABB5A6983F830509642E6
:1022C000C3F834E002F10101EBD143F26C40C0F2FB
:1022D00001000F210DF054FD49F61400C1F6FF7006
:1022E000BDE8F8430BF066B8032881F83040586326
:1022F000A7D1C3F83090C3F83490A2E7032984F83B
:1023000030005963C8D1C3F830C0C3F834C0C3E744
:10231000F8B54BF21C27C1F6FF7704463B780D4613
:1023200016467BB398422DD043F2F0701E21C0F2C6
:1023300001000DF025FD49F6140000230A22214674
:10234000C1F6FF700BF048F843F610000E21C0F202
:1023500001000DF015FD49F61400397800230A221A
:10236000C1F6FF700BF038F843F61C400121C0F2B3
:1023700001000DF005FD49F61400C1F6FF700BF0E9
:1023800019F808E048F2F803C2F200033246186870
:10239000294604F0DDFE43F620001121013CC0F285
:1023A00001000DF0EDFCE1B20F2915D84BF6902796
:1023B000C1F6FF7741F09001B86C03681B6898473D
:1023C000B86C036805F07F011B689847B86C036818
:1023D00006F07F011B68984743F25C400F21C0F272
:1023E00001000DF0CDFC230203F4706343F41043AD
:1023F0002D0405F4FE05310643F009032B4301F0DB
:10240000FE414BF220301943C1F6FF7009F0A4FEE3
:1024100043F21850C0F2010014210DF0B1FC49F64E
:102420001400C1F6FF70BDE8F8400AF0C3BF00BF5A
:10243000F8B54BF21C27C1F6FF7705463B780E46F0
:1024400014467BB398422DD043F2F0701E21C0F2A7
:1024500001000DF095FC49F6140000230A222946DC
:10246000C1F6FF700AF0B8FF43F610000E21C0F26B
:1024700001000DF085FC49F61400397800230A228A
:10248000C1F6FF700AF0A8FF43F61C400121C0F21C
:1024900001000DF075FC49F61400C1F6FF700AF05A
:1024A00089FF08E048F2F803C2F20003002218682E
:1024B000314604F04DFE43F634001221013DC0F2D6
:1024C00001000DF05DFCE9B20F2915D84BF69027FD
:1024D000C1F6FF7741F08001B86C03681B6898472C
:1024E000B86C036806F07F011B689847B86C0368F6
:1024F00004F07F011B68984743F25C400F21C0F253
:1025000001000DF03DFC230603F0FE4343F40043BD
:102510002D0205F47065310443F008032B4301F4E8
:10252000FE014BF220301943C1F6FF7009F014FE92
:1025300043F21850C0F2010014210DF021FC49F6BD
:102540001400C1F6FF70BDE8F8400AF033BF00BFC9
:10255000F8B54BF21C27C1F6FF7704463B780E46D0
:1025600015467BB398422DD043F2F0701E21C0F285
:1025700001000DF005FC49F6140000230A22214653
:10258000C1F6FF700AF028FF43F610000E21C0F2DA
:1025900001000DF0F5FB49F61400397800230A22FA
:1025A000C1F6FF700AF018FF43F61C400121C0F28B
:1025B00001000DF0E5FB49F61400C1F6FF700AF0CA
:1025C000F9FE09E048F2F803C2F200032A4618684F
:1025D000036831465B68984743F648000D21013C8B
:1025E000C0F201000DF0CCFBE1B20F2915D84BF67B
:1025F0009027C1F6FF7741F0B001B86C03681B6803
:102600009847B86C036806F07F011B689847B86C60
:10261000036805F07F011B68984743F25C400F2177
:10262000C0F201000DF0ACFB2B0603F0FE433104B9
:1026300043F4304343F00B0301F4FE012402194339
:1026400004F470644BF220302143C1F6FF7009F0AE
:1026500083FD43F21850C0F2010014210DF090FBED
:1026600049F61400C1F6FF70BDE8F8400AF0A2BEBA
:102670002DE9F047044643F658000F46C0F201002A
:10268000172115460DF07CFB601EC0B20F2800F22A
:10269000D1804BF69026C1F6FF7640F0A004B06CD6
:1026A000036821461B689847B06C036807F07F07F2
:1026B0001B6839469847B06C036805F07F051B68B6
:1026C00029464BF26C069847C1F6FF7643F2B0609C
:1026D0000A21C0F201000DF053FBB36C1A699C464D
:1026E000511C196114705CF8102F624526BF1B61E4
:1026F0009E4696464FF001084FF0000958698645FE
:1027000000F1010414D05C610278586BA4454FEAD3
:10271000221A98BF5B611918441C00286BD15869B4
:1027200083F830A08645C3F8348000F10104EAD173
:10273000B36C1A699C46511C196117705CF8102F14
:10274000624526BF1B619E4696464FF001084FF03A
:1027500000095969714501F1010014D058610A78E6
:10276000596B84454FEA221798BF5B615C18481C7F
:10277000002955D1596983F830707145C3F8348008
:1027800001F10100EAD1B36C1A691F46511C1961AD
:10279000157057F8106FBE4224BF1B611E464FF0E4
:1027A000010E4FF0000C5A69B24202F1010113D040
:1027B000596110785A6B8F424FEA201598BF5B61C0
:1027C0009C18511C12BB5A6983F83050B242C3F8AE
:1027D00034E002F10101EBD143F26C40C0F20100A0
:1027E0000F210DF0CDFA49F61400C1F6FF70BDE8D7
:1027F000F0470AF0DFBD032C81F830205C637FF4E2
:102800007DAFC3F83090C3F8349077E7032984F89C
:1028100030005963C7D1C3F830C0C3F834C0C2E731
:10282000032884F83020586393D1C3F83090C3F85C
:1028300034908EE743F2B0600A21C0F201000DF03F
:102840009FFAC9E72DE9F84F064643F67000154692
:102850000C46C0F2010012210DF092FA6B1E220408
:102860001B0203F4706102F4FE030B4343F4504374
:10287000310143F00D03C9B24BF220301943C1F6C8
:10288000FF7009F069FC43F21850C0F201001421F6
:10289000013E0DF075FAF3B20F2B00F287804BF278
:1028A0006C06C1F6FF7663F05F02B36C19699E4651
:1028B000481C18610A705EF8107F774504F07F0CA1
:1028C00005F07F0B24BF1B611F464FF0010800225B
:1028D0005869874200F1010414D05C610578586B97
:1028E000A6454FEA251A98BF5B611918441C0028B9
:1028F0006BD1586983F830A08742C3F8348000F167
:102900000104EAD1B36C19699846481C186181F832
:1029100000C058F8101F414526BF1B619E468E46D9
:1029200001224FF000095969714501F1010013D0EE
:1029300058610C78596B80454FEA241798BF5B614A
:102940005D18481C002949D1596983F830707145D8
:102950005A6301F10100EBD1B36C19691F46481CA1
:10296000186181F800B057F8106FBE4224BF1B6198
:102970001E464FF0010E4FF0000C5A69B24202F1B0
:10298000010113D0596110785A6B8F424FEA20151C
:1029900098BF5B619C18511C52BB5A6983F8305038
:1029A000B242C3F834E002F10101EBD143F26C40D2
:1029B000C0F201000F210DF0E3F949F61400C1F651
:1029C000FF70BDE8F84F0AF0F5BC032C81F83050D9
:1029D0005C637FF47DAF1A635A6379E7032885F857
:1029E000304058639FD1C3F83090C3F834909AE7D1
:1029F000032984F830005963BFD1C3F830C0C3F84D
:102A000034C0BAE72DE9F84F0E46054606F30D042B
:102A100043F684000D21013D04F50054C0F201008D
:102A20000DF0AEF92304290203F4FE0201F47063F1
:102A30001343610443F4604343F00E0301F0FE418D
:102A40004BF220301943C1F6FF7009F085FB43F2C9
:102A50001850C0F2010014210DF092F9EBB20F2BC7
:102A600000F289804BF26C05C1F6FF7563F01F021E
:102A7000AB6C19699E46481C18610A705EF8107F9D
:102A800006F50054774504F07F08C4F3C61B24BF45
:102A90001B611F464FF0010C00245A69974202F156
:102AA000010114D0596110785A6B8E454FEA201AF3
:102AB00098BF5B619E18511C002A6BD15A6983F83C
:102AC00030A09742C3F834C002F10101EAD1AB6CE7
:102AD0001A699C46511C196182F800805CF8102F1D
:102AE000624526BF1B619E46964601244FF00009B1
:102AF0005A69724502F1010113D0596110785A6B7D
:102B00008C454FEA201798BF5B619E18511C002A24
:102B100049D15A6983F8307072455C6302F1010152
:102B2000EBD1AB6C1A691F46511C196182F800B0D9
:102B300057F8106FBE4224BF1B611E464FF0010EB6
:102B40004FF0000C5A69B24202F1010113D05961F1
:102B500010785A6B8F424FEA201598BF5B619C1822
:102B6000511C52BB5A6983F83050B242C3F834E06A
:102B700002F10101EBD143F26C40C0F201000F21E0
:102B80000DF0FEF849F61400C1F6FF70BDE8F84FED
:102B90000AF010BC032986F8300059637FF47DAF3A
:102BA0001C635C6379E7032986F8300059639FD181
:102BB000C3F83090C3F834909AE7032984F83000C2
:102BC0005963BFD1C3F830C0C3F834C0BAE700BFFF
:102BD0002DE9F047054643F694000C46C0F201008B
:102BE00012210DF0CDF8681EC0B20F2800F2D3807C
:102BF0004BF69026C1F6FF7640F0E007B06C036814
:102C000039461B689847B06C04F50054036804F01B
:102C10007F051B6829469847B06C0368C4F3C61447
:102C20001B6821464BF26C069847C1F6FF7643F2CB
:102C30005C400F21C0F201000DF0A2F8B36C1A69DC
:102C40009C46511C196117705CF8102F624526BF15
:102C50001B619E4696464FF001084FF000095A69E5
:102C6000724502F1010114D0596110785A6B8C45FC
:102C70004FEA201A98BF5B619F18511C002A6BD144
:102C80005A6983F830A07245C3F8348002F101011B
:102C9000EAD1B36C1A699C46511C196115705CF835
:102CA000102F624526BF1B619E4696464FF00108D5
:102CB0004FF000095A69724502F1010114D05961BF
:102CC00010785A6B8C454FEA201798BF5B619D18AE
:102CD000511C002A55D15A6983F830707245C3F8E7
:102CE000348002F10101EAD1B36C1A691F46511C0C
:102CF0001961147057F8106FBE4224BF1B611E4645
:102D00004FF0010E4FF0000C5A69B24202F101017E
:102D100013D0596110785A6B8F424FEA201598BF33
:102D20005B619C18511C12BB5A6983F83050B24247
:102D3000C3F834E002F10101EBD143F26C40C0F280
:102D400001000F210DF01CF849F61400C1F6FF70C8
:102D5000BDE8F0470AF02EBB032987F8300059631D
:102D60007FF47DAFC3F83090C3F8349077E7032940
:102D700084F830005963C7D1C3F830C0C3F834C0F9
:102D8000C2E7032985F83000596393D1C3F8309026
:102D9000C3F834908EE743F25C400F21C0F201008B
:102DA0000CF0EEFFC9E700BF10B443F2FC3400237F
:102DB000C0F201044172026104600372C36041B158
:102DC000194600E0026942F82310427A01339A4220
:102DD000F8DC49F28853C2F200031A680AB90CE021
:102DE0001A465369002BFBD1506100234361838055
:102DF000C38083725DF8044B70471860F5E700BF2D
:102E00002DE9F8434BF69024C1F6FF7447F61221E2
:102E1000A06C0368DB69984743F6F175032044F220
:102E2000012744F2114142F2790242F6052384F867
:102E30006400C0F20005C0F20007C0F20001C0F259
:102E40000002C0F2000342F2C51065602760E16035
:102E50006261A361C0F2000041F6F51541F27117FD
:102E600042F6450140F6051241F2C1432061C0F22D
:102E70000005C0F20007C0F20001C0F20002C0F27B
:102E8000000341F22D00E5612762A160A262E362C6
:102E9000C0F2000040F6B56540F6717740F6F95192
:102EA00040F63D5240F6C133C0F20002C0F20003CA
:102EB0002063C0F20005C0F20007C0F2000149F62D
:102EC000140643F6A80022646364C1F6FF766563C6
:102ED000A76300254FF6FF77E163C0F201001721D9
:102EE00084F84C5084F84E5084F84D50A5656565C3
:102EF00084F8E95084F8665084F8655084F8675087
:102F000084F86850E76527660CF03AFF30460AF00F
:102F100051FA07F005FB4BF22033C1F6FF7344F280
:102F2000F50244F20530C0F20002C0F2000044F2A3
:102F30001951C3F85423C3F85003C0F2000141F6FD
:102F4000C95442F6D13241F62170C3F85C13C0F285
:102F50000004C0F20002C0F2000041F62101C3F8F3
:102F60006443C3F86823C3F86003C0F2000141F270
:102F7000E96442F2716241F6A130C3F87013C0F205
:102F80000004C0F20002C0F2000041F22961C3F85F
:102F90007443C3F85823C3F87C03C0F2000140F225
:102FA000857440F6450240F2C560C3F88013C0F254
:102FB0000004C0F20002C0F2000040F20561C3F854
:102FC0008443C3F88823C3F88C03C0F2000140F2A5
:102FD000455440F2854243F6C000C0F20002C3F8F7
:102FE0009013C0F200041D21C0F20100C3F8944305
:102FF000C3F898230CF0C4FE30460AF0DBF94BF21C
:103000006C03C1F6FF7342F211309A6C02F11801A1
:10301000156095615560D5619560D5601562556202
:1030200012615261D1629162C0F2000041F29534A6
:1030300041F27D524FF001095860C0F20004C0F225
:10304000000241F2093083F84E5083F84D509D65DF
:103050005D65DF651F6683F8E95083F8665083F885
:10306000655083F8675083F868505C619A6109FA8B
:1030700009F8C0F2000042F2314C42F2515E41F2D6
:10308000E90141F6515741F2214541F6D94441F257
:10309000A9221861C0F2000E48EA0908C0F2000C2B
:1030A000C0F20001C0F20007C0F20005C0F2000447
:1030B000C0F2000240F67D4083F84C9083F86480B3
:1030C000C3F800C0C3F80CE0C0F20000D9611F6271
:1030D0009D609C62DA6240F6613140F6412740F61D
:1030E000013540F6A12440F6DD421863C0F200012C
:1030F000C0F20007C0F20005C0F20004C0F20002F6
:1031000043F6E00059639F63DD631C645A64C0F2B8
:10311000010018210CF034FE3046BDE8F8430AF0F7
:1031200049B900BF70B5DFEDF17A2DED048B60EE8B
:10313000277A49F24863FCEEE77A49F2446549F29E
:103140004C6492B0C1F6FF73C1F6FF75C1F6FF740F
:103150000220CDED017AF0EE408AB0EE608AB0EE4A
:10316000419A83ED000AC5ED000A84ED001A0AF0C9
:1031700075FB9DF80460864200F013823146022000
:103180000AF086FBD5ED007A9FEDD87A67EE877A54
:103190000320FCEEE77ACDED017A0AF05FFB9DF8A3
:1031A0000450854203D0294603200AF071FBD4ED78
:1031B000007A9FEDCE7A67EE877A0420FCEEE77AFC
:1031C000CDED017A0AF04AFB9DF80440844203D019
:1031D000214604200AF05CFB43F20044C0F20104E3
:1031E0000FCC02AD0FC50FCC0FC50FCC0FC594E8A7
:1031F0000F0085E80F0000200AF030FBC24312A93F
:1032000002F00F0201EB8202034652F8404C84F0B8
:103210007044E44384EA231303F00F0301EB8303B8
:10322000012053F8403C83EA14140AF017FBE443EE
:1032300080EA040212A902F00F0201EB82020346A7
:1032400052F8402C82EA141484EA231303F00F038B
:1032500001EB8303022053F8403C83EA14140AF084
:10326000FDFAE44380EA040212A902F00F0201EB26
:103270008202034652F8402C82EA141484EA231393
:1032800003F00F0301EB8303032053F8403C83EA70
:1032900014140AF0E3FAE44380EA040212A902F0EB
:1032A0000F0201EB8202034652F8402C82EA14140A
:1032B00084EA231303F00F0301EB8303042053F884
:1032C000403C83EA14140AF0C9FAE44380EA040299
:1032D00012A902F00F0201EB8202034652F8402CC1
:1032E00082EA141484EA231303F00F0301EB83032F
:1032F00040F6FC7053F8403C83EA14140AF0AEFA2E
:10330000E443250E854204D0294640F6FC700AF0BD
:10331000BFFA40F6FD700AF0A1FAC4F307458542F2
:1033200004D0294640F6FD700AF0B2FA40F6FE706D
:103330000AF094FAC4F30725854204D0294640F6E2
:10334000FE700AF0A5FA40F6FF700AF087FAE4B2C0
:10335000844204D0214640F6FF700AF099FA43F601
:10336000FC001421C0F201000CF00AFD18EE900AD6
:103370000EF032FF41EC100B49F614000A21C1F6A1
:10338000FF700AF069F843F614100121C0F2010041
:103390000CF0F6FC02200AF061FA019049F61400E4
:1033A00000230A220199DFED518AC1F6FF700AF06D
:1033B00013F843F618100121C0F201000CF0E0FCF4
:1033C000DDED017AF8EE677A87EEA87A17EE100A3B
:1033D0000EF002FF41EC100B49F614000A21C1F671
:1033E000FF700AF039F843F61C100821C0F2010002
:1033F0000CF0C6FC19EE100A0EF0EEFE41EC100BBC
:1034000049F614000A21C1F6FF700AF025F843F6C8
:1034100014100121C0F201000CF0B2FC04200AF0EB
:103420001DFA019049F6140000230A220199C1F601
:10343000FF7009F0D1FF43F618100121C0F201001E
:103440000CF09EFCDDED017AF8EE677A87EEA87A43
:1034500017EE100A0EF0C0FE41EC100B49F61400F6
:103460000A21C1F6FF7009F0F7FF43F62810082182
:10347000C0F201000CF084FC18EE100A0EF0ACFE55
:1034800041EC100B49F614000A21C1F6FF7009F057
:10349000E3FF43F614100121C0F201000CF070FCB0
:1034A00003200AF0DBF9019049F6140000230A22F8
:1034B0000199C1F6FF7009F08FFF43F61810012142
:1034C000C0F201000CF05CFCDDED017AF8EE677AE9
:1034D00087EEA87A17EE100A0EF07EFE41EC100B74
:1034E00049F614000A21C1F6FF7005E000007F4391
:1034F00000FEFF4600FEFFC609F0AEFF43F63410A3
:103500000121C0F201000CF03BFC49F61400C1F6A9
:10351000FF7009F04FFF5FED0A7AB4EEE78AF1EE33
:1035200010FA0ADC5FED0D7AB4EEE78AF1EE10FADC
:1035300025D50022C8F2010202E00022C7F6FF7280
:103540005FED157A48F24813C2F20003B4EEE79A31
:10355000F1EE10FA9A6120DC5FED1A7AB4EEE79A88
:10356000F1EE10FA12D50022C8F2010248F2081357
:10357000C2F200039A6112B0BDEC048B70BDF0EE94
:10358000487AFEEEC87A17EE902AD9E7F0EE497A2B
:10359000FEEEC87A17EE902AE8E70022C7F6FF721F
:1035A000E4E7F0EE487AEFE5F0B52DED028B40F65A
:1035B000FC7093B00AF052F9064640F6FD700AF02E
:1035C0004DF9030440F6FE7043EA06660AF046F938
:1035D000074640F6FF700AF041F943F20044C0F29A
:1035E000010406430FCC02AD0FC50FCC0FC50FCCA5
:1035F0000FC594E80F0085E80F0000200AF02EF9AF
:10360000C24312A902F00F0201EB8202034652F8F4
:10361000405C85F07045ED4385EA231303F00F030A
:1036200001EB8303012053F8403C83EA15150AF0AF
:1036300015F9ED4380EA050212A902F00F0201EB31
:103640008202034652F8402C82EA151585EA2313BC
:1036500003F00F0301EB8303022053F8403C83EA9D
:1036600015150AF0FBF8ED4380EA050212A902F0F5
:103670000F0201EB8202034652F8402C82EA151534
:1036800085EA231303F00F0301EB8303032053F8B0
:10369000403C83EA15150AF0E1F8ED4380EA0502A3
:1036A00012A902F00F0201EB8202034652F8402CED
:1036B00082EA151585EA231303F00F0301EB830358
:1036C000042053F8403C83EA15150AF0C7F8ED438F
:1036D00080EA050212A902F00F0201EB8202034602
:1036E00052F8402C82EA151585EA231303F00F03E4
:1036F00001EB830343F6381053F8403C1321C0F22A
:10370000010083EA151546EA07240CF039FB49F657
:103710001400002310222146C1F6FF7009F05CFE60
:1037200043F64C100521C0F201000CF029FBED43DB
:1037300049F614002946C1F6FF700023102209F053
:103740004BFEA54239D102200AF088F807EE900A14
:103750009FEDA58AB8EE677A49F24863C7EE087A0A
:10376000C1F6FF730320C3ED007A0AF077F807EE85
:10377000900AB8EE677A49F24463C7EE087AC1F658
:10378000FF730420C3ED007A0AF068F807EE900A90
:10379000B8EE677A49F24C63C7EE087AC1F6FF7358
:1037A000C3ED007A49F61400C1F6FF7013B0BDEC0A
:1037B000028BBDE8F04009F0FDBD43F65410232113
:1037C000C0F201000CF0DCFA49F24863C1F6FF7365
:1037D000D3ED007A9FED847A67EE877A0220FCEEC3
:1037E000E77ACDED017A0AF039F89DF80440844279
:1037F00003D0214602200AF04BF849F24463C1F697
:10380000FF73D3ED007A9FED787A67EE877A032015
:10381000FCEEE77ACDED017A0AF020F89DF804403D
:10382000844203D0214603200AF032F849F24C6367
:10383000C1F6FF73D3ED007A9FED6B7A67EE877A5E
:103840000420FCEEE77ACDED017A0AF007F89DF846
:103850000440844203D0214604200AF019F843F2C0
:103860000045C0F201050FCD02AC0FC40FCD0FC44F
:103870000FCD0FC495E80F0084E80F00002009F079
:10388000EDFFC24312A902F00F0201EB82020346D0
:1038900052F8404C84F07044E44384EA231303F06C
:1038A0000F0301EB8303012053F8403C83EA141417
:1038B00009F0D4FFE44380EA040212A902F00F02E7
:1038C00001EB8202034652F8402C82EA141484EA87
:1038D000231303F00F0301EB8303022053F8403C52
:1038E00083EA141409F0BAFFE44380EA040212A93F
:1038F00002F00F0201EB8202034652F8402C82EAEA
:10390000141484EA231303F00F0301EB8303032051
:1039100053F8403C83EA141409F0A0FFE44380EA22
:10392000040212A902F00F0201EB8202034652F8D0
:10393000402C82EA141484EA231303F00F0301EBF2
:103940008303042053F8403C83EA141409F086FFF3
:10395000E44380EA040212A902F00F0201EB8202A2
:10396000034652F8402C82EA141484EA231303F02D
:103970000F0301EB830340F6FC7053F8403C83EAED
:10398000141409F06BFFE443250E854204D0294648
:1039900040F6FC7009F07CFF40F6FD7009F05EFF18
:1039A000C4F30745854204D0294640F6FD7009F06E
:1039B0006FFF40F6FE7009F051FFC4F30725854202
:1039C00004D0294640F6FE7009F062FF40F6FF7011
:1039D00009F044FFE4B284423FF4E4AE214640F6ED
:1039E000FF7009F055FFDDE600007F432DE9F84345
:1039F00049F20E69C2F2000943F678102DED028BF0
:103A00000521C0F201000CF0BBF9B9F80030DFED80
:103A1000548A9FED548A07EE103AB8EEC77A49F6F9
:103A2000140437EE287AC1F6FF74C7EE087A49F21B
:103A30000867C2F2000749F20C68C2F2000849F2B6
:103A40008C56C2F2000648F20415C2F2000517EEC9
:103A5000900A0EF0C1FB41EC100B0A21204609F040
:103A6000FBFC43F680100C21C0F201000CF088F939
:103A70003B8807EE903AF8EEE77A77EEA87A87EE81
:103A8000887A17EE100A0EF0A7FB41EC100B0A2102
:103A9000204609F0E1FC43F690100721C0F2010036
:103AA0000CF06EF9B8F80010204609F025FC43F63A
:103AB00098100C21C0F201000CF062F93188204608
:103AC00009F01AFC43F6A8101421C0F201000CF012
:103AD00057F92988204609F00FFC43F6C010092148
:103AE000C0F201000CF04CF948F20013C2F20003DE
:103AF0000A2219682046002309F06EFC43F6CC1018
:103B00000D21C0F201000CF03BF94BF22023C1F66D
:103B1000FF730A2219682046002309F05DFC43F672
:103B2000DC100921C0F201000CF02AF948F2FC0374
:103B3000C2F200030A2219682046002309F04CFC57
:103B4000204609F037FCBDEC028BB9F80030B8F81C
:103B500000203B80002332802B80BDE8F88300BF2B
:103B6000333323433333A343F0B52DED028BDC20F5
:103B700083B00AF0C7FB49F6140443F6E810C1F617
:103B8000FF744021C0F201000CF0FAF8204609F061
:103B900011FC43F62C202921C0F201000CF0F0F8B2
:103BA000204609F007FC43F658202D21C0F2010001
:103BB0000CF0E6F8204609F0FDFB43F688201121C1
:103BC000C0F201000CF0DCF84EF224410A2200237E
:103BD0002046C0F20C0109F0FFFB43F69C200621B1
:103BE000C0F201000CF0CCF8204609F0E3FB2046BF
:103BF00009F0E0FB43F6A4200D21C0F201000CF017
:103C0000BFF8204609F0D6FB41F224000AF00AF979
:103C100048F2F805C2F20005064602F007FF2E60E2
:103C2000FFF7C2FCFFF7ECF84EF28813CEF2000368
:103C3000012640F200201E60C1F6FF70802108F0CE
:103C400053FE43F6B4200F21C0F201000CF098F8A7
:103C5000204609F0AFFBB7EE001AB0EE410AF0EED5
:103C6000410AFFF75FFA49F20E6749F20C61C2F2AE
:103C70000007C2F2000149F2086249F28C53C2F215
:103C80000002C2F2000343F6C420B7F800E00F8838
:103C9000A2F800E01421C0F201001F800CF070F8BF
:103CA0002046802109F028FB43F6DC201121C0F2D8
:103CB00001000CF065F8204640F65A3109F01CFB73
:103CC00043F6F0200321C0F201000CF059F8204621
:103CD00009F070FB28689FED448A0368B6EE000A7D
:103CE000DB6800219847286803683146DB68B6EE38
:103CF000000A984728680368B0EE480ADB6802218A
:103D0000984728689FED390A03680321DB689847C4
:103D100028689FED370A03680A21DB6898472868FE
:103D20000368B7EE000ADB68062198472868036835
:103D3000B0EE480ADB680721984728689FED2D0AF6
:103D400003680B21DB68984741F644624BF69033D9
:103D500045F26061C2F20002C1F6FF7346F2C40090
:103D60005052585272B645F25C6545F25E6141F6BA
:103D7000991746F267605753505262B672B65F5356
:103D8000585262B64BF2340248F268134EF20811F0
:103D9000C1F6FF72C2F20003CEF200014BF23337DC
:103DA00044F6CC4543F6F4209761D5619F61DD610F
:103DB000C0F201000E600B210BF0E2FF204609F07B
:103DC000F9FAFFF713FE49F23462C2F200024BF235
:103DD000242312680192C1F6FF73019A1A6003B09E
:103DE000BDEC028BF0BD00BF3333333F9A99593F8E
:103DF000CDCCCC3D9A99993E2DE9F04F9DF82450B9
:103E0000013DEDB20F2D02D84EB2002E01DBBDE810
:103E1000F08FE02900F28B80846C27693543A4463B
:103E20007E1C26613D705CF8105F654502F07F08DE
:103E300026BF2461A646AE4601224FF000096569FF
:103E4000754505F1010615D066612F78656BB4459F
:103E50004FEA271B98BF646104EB050A6E1C002D16
:103E600040F09C80656984F830B07545626305F167
:103E70000106E9D1846C2569A4466E1C266185F88B
:103E800000805CF8102F624526BF2461A646964646
:103E90004FF001084FF000096269724502F1010517
:103EA00014D065611678626BAC454FEA261A98BF4C
:103EB0006461A718551C002A7BD1626984F830A080
:103EC0007245C4F8348002F10105EAD101F0EF0136
:103ED000C0299CD0826C1169174603F07F03481CEF
:103EE00010610B7057F8106FBE4224BF1261164666
:103EF0004FF0010E4FF0000C5369B34203F1010182
:103F000085D051611878536B8F424FEA201598BFC6
:103F10005261D418591C002B56D1536982F8305085
:103F2000B342C2F834E003F10101EAD16FE7F729A7
:103F30007FF66DAF01F10803DAB20123934013F06D
:103F4000DD0F3FF464AF836C1A691F46501C186183
:103F5000117057F8106FBE4224BF1B611E464FF010
:103F6000010E4FF0000C5A69B24202F101013FF418
:103F70004EAF596110785A6B8F424FEA201598BFA7
:103F80005B619C18511C4ABB5A6983F83050B2429D
:103F9000C3F834E002F10101EBD138E7032E8AF8CF
:103FA000307066637FF44BAFC4F83090C4F834903F
:103FB00045E7032D87F8306065637FF46DAFC4F883
:103FC0003090C4F8349067E7032984F830005163D7
:103FD00092D1C2F830C0C2F834C08DE7032984F80A
:103FE00030005963BFD1C3F830C0C3F834C0BAE75A
:103FF000F0B54BF21C27C1F6FF7783B03B7804463F
:104000000D4616467BB398422DD043F2F0701E2128
:10401000C0F201000BF0B4FE49F6140000230A229E
:104020002146C1F6FF7009F0D7F943F610000E21C2
:10403000C0F201000BF0A4FE49F614003978002309
:104040000A22C1F6FF7009F0C7F943F61C400121AE
:10405000C0F201000BF094FE49F61400C1F6FF70A7
:1040600009F0A8F908E048F2F803C2F2000332466A
:104070001868294603F06CF843F600301121C0F2AD
:1040800001000BF07DFE631E1B0203F47063290424
:1040900043F41043320601F4FE0143F009030B43DD
:1040A0004BF2203002F0FE411943C1F6FF7008F0D8
:1040B00053F843F218501421C0F201000BF060FED7
:1040C0004BF26C0033462A460094C1F6FF709021F3
:1040D000FFF792FE43F26C400F21C0F201000BF09B
:1040E0004FFE49F61400C1F6FF7003B0BDE8F04082
:1040F00009F060B9F0B54BF21C24C1F6FF7483B02F
:10410000237805460E4617467BB398422DD043F2DE
:10411000F0701E21C0F201000BF032FE49F61400CF
:1041200000230A222946C1F6FF7009F055F943F62B
:1041300010000E21C0F201000BF022FE49F614001F
:10414000217800230A22C1F6FF7009F045F943F6F1
:104150001C400121C0F201000BF012FE49F61400D0
:10416000C1F6FF7009F026F908E048F2F803C2F240
:1041700000033A461868314602F0EAFF43F614306D
:104180001621C0F201000BF0FBFD691EC9B20F2918
:1041900015D84BF69024C1F6FF7441F09001A06C45
:1041A00003681B689847A06C036806F07F011B68D2
:1041B0009847A06C036807F07F011B68984743F29B
:1041C0005C400F21C0F201000BF0DAFD4BF26C00F5
:1041D0003B4632460095C1F6FF709021FFF70CFE7A
:1041E00043F26C400F21C0F201000BF0C9FD49F60B
:1041F0001400C1F6FF7003B0BDE8F04009F0DAB872
:10420000F0B54BF21C27C1F6FF7783B03B7804462C
:104210000D4616467BB398422DD043F2F0701E2116
:10422000C0F201000BF0ACFD49F6140000230A2295
:104230002146C1F6FF7009F0CFF843F610000E21B9
:10424000C0F201000BF09CFD49F614003978002300
:104250000A22C1F6FF7009F0BFF843F61C400121A5
:10426000C0F201000BF08CFD49F61400C1F6FF709E
:1042700009F0A0F808E048F2F803C2F200030022B7
:104280001868294602F064FF43F62C301221C0F270
:1042900001000BF075FD3306611E03F0FE4343F48D
:1042A000004309022A0401F4706143F008030B4340
:1042B0004BF2203002F4FE011943C1F6FF7007F003
:1042C0004BFF43F218501421C0F201000BF058FDCF
:1042D0004BF26C0033462A460094C1F6FF708021F1
:1042E000FFF78AFD43F26C400F21C0F201000BF092
:1042F00047FD49F61400C1F6FF7003B0BDE8F04079
:1043000009F058B8F0B54BF21C24C1F6FF7483B025
:10431000237805460E4617467BB398422DD043F2CC
:10432000F0701E21C0F201000BF02AFD49F61400C6
:1043300000230A222946C1F6FF7009F04DF843F622
:1043400010000E21C0F201000BF01AFD49F6140016
:10435000217800230A22C1F6FF7009F03DF843F6E8
:104360001C400121C0F201000BF00AFD49F61400C7
:10437000C1F6FF7009F01EF808E048F2F803C2F237
:10438000000300221868314602F0E2FE43F6403096
:104390001721C0F201000BF0F3FC691EC9B20F290E
:1043A00015D84BF69024C1F6FF7441F08001A06C43
:1043B00003681B689847A06C036806F07F011B68C0
:1043C0009847A06C036807F07F011B68984743F289
:1043D0005C400F21C0F201000BF0D2FC4BF26C00EC
:1043E0003B4632460095C1F6FF708021FFF704FD81
:1043F00043F26C400F21C0F201000BF0C1FC49F602
:104400001400C1F6FF7003B0BDE8F04008F0D2BF61
:10441000F0B54BF21C27C1F6FF7783B03B7804461A
:104420000D4616467BB398422DD043F2F0701E2104
:10443000C0F201000BF0A4FC49F6140000230A228C
:104440002146C1F6FF7008F0C7FF43F610000E21A9
:10445000C0F201000BF094FC49F6140039780023F7
:104460000A22C1F6FF7008F0B7FF43F61C40012195
:10447000C0F201000BF084FC49F61400C1F6FF7095
:1044800008F098FF09E048F2F803C2F20003324650
:104490001868036829465B68984743F658300D2131
:1044A000C0F201000BF06CFC330603F0FE4329045C
:1044B000621E43F4304343F00B0301F4FE01120289
:1044C000194302F470624BF220301143C1F6FF70C1
:1044D00007F042FE43F218501421C0F201000BF025
:1044E0004FFC4BF26C0033462A460094C1F6FF7035
:1044F000B021FFF781FC43F26C400F21C0F20100B4
:104500000BF03EFC49F61400C1F6FF7003B0BDE8A5
:10451000F04008F04FBF00BFF0B54BF21C24C1F6CD
:10452000FF7483B0237805460E4617467BB3984246
:104530002DD043F2F0701E21C0F201000BF020FCE0
:1045400049F6140000230A222946C1F6FF7008F03C
:1045500043FF43F610000E21C0F201000BF010FCE7
:1045600049F61400217800230A22C1F6FF7008F0F2
:1045700033FF43F61C400121C0F201000BF000FCA8
:1045800049F61400C1F6FF7008F014FF09E048F284
:10459000F803C2F200033A461868036831465B68C4
:1045A000984743F668301221C0F201000BF0E8FB97
:1045B000691EC9B20F2915D84BF69024C1F6FF74B5
:1045C00041F0B001A06C03681B689847A06C0368B9
:1045D00006F07F011B689847A06C036807F07F0115
:1045E0001B68984743F25C400F21C0F201000BF0BA
:1045F000C7FB4BF26C003B4632460095C1F6FF709C
:10460000B021FFF7F9FB43F26C400F21C0F201002B
:104610000BF0B6FB49F61400C1F6FF7003B0BDE81D
:10462000F04008F0C7BE00BF2DE9F0479DF82040DC
:10463000013CE4B20F2C03D84EB2002E0D4601DB34
:10464000BDE8F087E0290FD9F729F9D90835EDB28F
:10465000012303FA05F515F0DD0FF1D0806C036836
:10466000BDE8F0471B6818478146806C1F46036809
:1046700046EA0401C9B21B6890469847D9F8480039
:10468000036808F07F011B6805F0EF059847C02D0F
:10469000D6D0D9F84800036807F07F011B68BDE851
:1046A000F0471847F8B50446806C03681B699847C3
:1046B00008B90020F8BDA06C03685B699847C3B2D5
:1046C00003F0FB01F929F4D0A26D82B994F84D20D2
:1046D00084F84F30150600F19C8040B20028C0F2EB
:1046E0005081002084F84D00A0656065F8BD01068A
:1046F00067D494F84F10F02904EB020140D081F800
:104700004F30616D4B1E9A4240D394F84F20F02AEF
:10471000E7D013063DD4002384F86630B02B4CD08C
:10472000A02B4AD0D02B48D0E02B46D0C02B44D071
:10473000002094F8505084F86750032908BF94F87B
:10474000515084F8650018BF002500210120B02BCE
:1047500084F86850A165616584F8E90000F0B580CF
:1047600000F2AC80902B00F0B080A02B00F0AD8068
:10477000802B00F0AA80002384F84D300120F8BD82
:1047800081F86930636D013B9A42AAD20132A26579
:104790008FE702F10C03DBB2012BBCD902F0FB0363
:1047A000F92BB8D0EF2A00F2DB8002F0F003802B67
:1047B00084F8663001D0902BB0D102F00F000130A8
:1047C000B7E7A3F1F701082993D8012505FA01F00D
:1047D00010F4DD7F40F0968000298AD194F869308A
:1047E000F02B7FF47EAF561C2244F720370A82F864
:1047F000690084F8676084F8687084F8651084F84C
:104800004D10284684F8663084F8E950A16561654A
:10481000F8BD02F10C05EEB2012E7FF65EAF02F09C
:10482000FB0EBEF1F90F3FF458AFEF2A2DD802F07E
:10483000F007802F2AD140B20028FFF64FAF0121A8
:1048400084F84F2084F85030A165EDB2012D7FF639
:1048500048AFBEF1F90F3FF444AFEF2A5FD802F042
:10486000F003B02B26D01ED9D02B04D0E02B21D0C2
:10487000C02B7FF436AF022363650121A36D9942FB
:1048800027D90133A3650020F8BD174607F0DF06DE
:10489000902ED0D007F0BF06A02ECCD007F0EF07A7
:1048A000C02FC8D019E7902B04D0A02B02D0802BAA
:1048B0007FF417AF032363650221DFE7D02B04D019
:1048C000E02B02D0C02B7FF456AF84F84D2001209E
:1048D000F8BDEF2A94BF02F0F005154602F00F0272
:1048E0000023013294F8501084F86520012084F8E8
:1048F000671084F8683084F86650A365636584F8AF
:10490000E900F8BD002284F8672084F8682084F864
:10491000652084F8663084F8E9502846F8BDF62A08
:104920000FD007D8F12AA6D01CD9F22AC2D0F32A78
:10493000A1D0D6E6FC2A21D8FA2A02D2F82A7FF49E
:10494000D0AE0023012084F8653084F8673084F805
:10495000683084F86620A365636584F8E900F8BDD3
:104960001346D9E6F02A7FF4BCAE802100236165AE
:1049700084F8692084F84D307F217FE7FE2AE0D259
:10498000AFE61A468E4603F10C055EE790F86630F6
:10499000F12B7CD00ED9FA2B2BD01FD8F32B38D08B
:1049A000C0F08180F62B7AD0F82B40F08B80036B1F
:1049B000F3B11847B02B6ED031D9D02B21D03ED9CE
:1049C000E02B42D0F02B7ED1C3698BB1B0F86710D9
:1049D000802900F1690028BF80211847FC2B0CD0EA
:1049E00051D3FE2B4BD0FF2B6BD1436C002BE0D16E
:1049F0007047436B002BDCD1FAE7C36B002BD8D197
:104A0000F6E74369002BF3D090F8671090F8650043
:104A10001847836A002BEBD090F867001847902B5B
:104A200029D0A02B23D0802BE2D10368002BDFD02C
:104A300090F8682090F8671090F865001847C02B30
:104A400042D10369002BDFD1D2E78269002ACFD09F
:104A500090F8681090F8673090F86500C90101F48B
:104A60007E5103F07F031943A1F50051104783687D
:104A7000002BDDD1BCE74368002BD9D1B8E7036C2C
:104A8000002B96D1B4E7836B002B92D1B0E7036A79
:104A9000002BC1D1ACE7C368002BC9D1A8E7C36A1A
:104AA000002B86D1A4E7426A002AA1D090F8683092
:104AB00090F86700DB0103F47E5300F07F00184399
:104AC0001047704770477047704700BF90F86430D8
:104AD000DA0725D513F0FE0F22D070B590F8665096
:104AE00085F08002602A82B004461AD9F62D6ED075
:104AF00067D8F12D7ED04FD9F22D2DD0F32D1AD1BC
:104B0000806C94F86760036829461B689847A06C1E
:104B10000368DB6C06F07F0102B0BDE87040184707
:104B2000704790F865608E4207D031B15B08012B69
:104B300008D0032B27D002B070BD5B08012B01D039
:104B4000022BF8D194F8683094F867200096294633
:104B50002046FFF769FDEEE7806C94F86730026845
:104B600094F868601268294643EAC6159047A06C1D
:104B7000036805F07F019B6C9847A06C0368C5F340
:104B8000C6119B6CC8E794F8683094F867200096CB
:104B90002946FFF749FDCEE7F02DCCD1B0F867608C
:104BA000802E28BF802600F16905002EC3D02E4438
:104BB000A06C15F8011B03681B689847AE42F7D13B
:104BC000B9E7FC2D26D8FA2D01D2F82DB3D105F185
:104BD0000803DBB2072BAED8012202FA03F313F06D
:104BE000DD0FA8D0A06C03681B68294602B0BDE8A1
:104BF00070401847806C94F8672094F86830066815
:104C00001201294603F00F0302F0700532681D43BC
:104C10009047E7E7FE2D8ED3D9E700BFF8B50546EC
:104C2000846C0BF009F8C0F30723C0F30742010EB0
:104C300010F0FF005BD004F1280604F1180712E021
:104C4000A02829D024DDC0283ED0D0283CD0B028D0
:104C500022D00AF0F1FFC0F30723C0F30742010E90
:104C600010F0FF0043D00001E02815D0E8DDFC285B
:104C700039DCFA2803DAF62801D0F828E9D1A26A4B
:104C8000511CA1621370A36AB342E2D3A762E0E7AA
:104C9000802801D09028DCD1A06A00F1010EC4F870
:104CA00028E00370A36AB34228BF3B46581CA062A9
:104CB0001A70A36A9E4298BF3B465A1CA2621970A2
:104CC000A36A9E42C5D8E1E7A16A481CA0620B70A6
:104CD000A36AB34228BF3B46591CA1621A70A36A5B
:104CE0009E42B6D8D2E7FE380128B2D8C7E7E16ABB
:104CF000A36A994246D047D318341B1B03F1100214
:104D00000B1BD31A002B3DD0AB6CDA6A511CD96255
:104D100003F128008142127824BF03F11801D962FF
:104D200002F0FB03F92B2DD0AB6D7BB3140600F121
:104D3000AB8095F84F10F02905EB03011AD081F8EC
:104D40004F20696D4A1E93421AD395F84F20F02ADE
:104D500026D010062AD4002385F86630B02B39D02F
:104D6000A02B37D0D02B35D0E02B33D0C02B31D077
:104D7000002032E081F869206A6D013A93420FD237
:104D80000133AB650020F8BD5B1ABBE795F84D30E9
:104D900085F84F201E0641D453B2002BC0F221816A
:104DA000002085F84D00A8656865F8BD02F10C0388
:104DB000DBB2012BCFD902F0FB03F92BCBD0EF2ACA
:104DC00000F2018102F0F003802B85F8663001D0FB
:104DD000902BC3D102F00F00013095F8504085F8B8
:104DE0006740032908BF95F8514085F8650018BF52
:104DF000002400210120B02B85F86840A965696571
:104E000085F8E90006D069D9D02B03D0E02B01D07A
:104E1000C02B69D185F84D200120F8BD03F10C04A9
:104E2000E1B20129B8D903F0FB01F929B4D0EF2B85
:104E30005FD803F0F00080285CD1110672D4012104
:104E400085F84F3085F85020A965E4B2012CA7D928
:104E500003F0FB02F92AA3D0EF2B00F2918003F0BC
:104E6000F002B02A5AD052D9D02A03D0E02A55D025
:104E7000C02A95D102226A650121AA6D914259D9B1
:104E80000132AA650020F8BD02F10901C9B2082962
:104E90003FF64FAF012404FA01F010F4DD7F62D138
:104EA00000297FF446AF95F86920F02A7FF478AFA7
:104EB0005E1C2B44F720370A83F8690085F8676089
:104EC00085F8687085F8651085F84D10204685F8DE
:104ED000662085F8E940A9656965F8BD902B99D0F1
:104EE000A02B97D0802B95D0002385F84D30012042
:104EF000F8BD184600F0DF0190299ED000F0BF01F8
:104F0000A0299AD000F0EF00C02896D044E7902A5C
:104F100004D0A02A02D0802A7FF442AF03226A651F
:104F20000221AAE702F10C03DBB2012B7FF638AFB6
:104F3000134691E7EF2B94BF03F0F001194603F0FD
:104F40000F03013395F8502085F8653000230120C8
:104F500085F8672085F8683085F86610AB656B6565
:104F600085F8E900F8BD002385F8673085F86830DA
:104F700085F8653085F8662085F8E9402046F8BD5B
:104F8000F62B11D009D8F12B3FF474AF1DD9F22BB9
:104F9000C4D0F32B3FF46EAF02E7FC2B25D8FA2BDD
:104FA00002D2F82B7FF4FCAE0022012085F86520A8
:104FB00085F8672085F8682085F86630AA656A65F7
:104FC00085F8E900F8BD1346C6E6F02B7FF4E8AE9D
:104FD00080210022696585F8693085F84D207F21A0
:104FE0004BE7134602F10C042FE7FE2BDCD2D7E689
:104FF00090F86630F12B7CD00ED9FA2B2BD01FD82D
:10500000F32B38D0C0F08180F62B7AD0F82B40F00B
:105010008B80036BF3B11847B02B6ED031D9D02BF6
:1050200021D03ED9E02B42D0F02B7ED1C3698BB189
:10503000B0F86710802900F1690028BF8021184767
:10504000FC2B0CD051D3FE2B4BD0FF2B6BD1436CE0
:10505000002BE0D17047436B002BDCD1FAE7C36B28
:10506000002BD8D1F6E74369002BF3D090F86710F6
:1050700090F865001847836A002BEBD090F8670022
:105080001847902B29D0A02B23D0802BE2D1036886
:10509000002BDFD090F8682090F8671090F865003A
:1050A0001847C02B42D10369002BDFD1D2E78269B8
:1050B000002ACFD090F8681090F8673090F865001B
:1050C000C90101F47E5103F07F031943A1F500519A
:1050D00010478368002BDDD1BCE74368002BD9D192
:1050E000B8E7036C002B96D1B4E7836B002B92D109
:1050F000B0E7036A002BC1D1ACE7C368002BC9D16C
:10510000A8E7C36A002B86D1A4E7426A002AA1D08F
:1051100090F8683090F86700DB0103F47E5300F0EC
:105120007F0018431047704770477047704700BFB3
:1051300090F86430DA0777D513F0FE0F74D02DE9BC
:10514000F04790F8664084F08002602A82B086467C
:105150006BD9F62C00F0998100F28F81F12C00F0D0
:10516000D78140F24481F22C00F08180F32C58D199
:10517000836C90F867801A699C46511C1961147001
:105180005CF8106F664524BF1B611E4601274FF077
:1051900000095A69B24202F1010114D05961107834
:1051A0005A6B8C454FEA201598BF5B619C18511CC7
:1051B000002A40F0FC805A6983F83050B2425F63A5
:1051C00002F10101EAD1DEF848301A6908F07F07E0
:1051D0001E46511C1961177056F8107FB74224BF44
:1051E0001B611F464FF0010E4FF0000C5A69BA4286
:1051F00002F1010115D0596110785A6B8E424FEAC5
:10520000201598BF5B619C18511C002A40F0E48077
:105210005A6983F83050BA42C3F834E002F1010110
:10522000E9D102B0BDE8F087704790F865508D4233
:105230000ED069B15B08012B0FD0032BF1D19EF882
:1052400068309EF8672000952146FEF7D5FDE8E717
:105250005B08012B01D0022BE3D19EF868309EF849
:105260006720009521467046FEF7C6FDD9E7836C9E
:105270009EF867101A6990F868009C46551C1D61DD
:1052800014705CF8107F674541EAC01424BF1B61AD
:105290001F464FF001084FF000095A69BA4202F167
:1052A000010114D0596110785A6B8C454FEA2016D1
:1052B00098BF5B619D18511C002A6DD15A6983F813
:1052C0003060BA42C3F8348002F10101EAD1DEF85D
:1052D000483019699C4604F07F02481C18610A7026
:1052E0005CF8107F674524BF1B611F464FF0010823
:1052F0004FF000095A69BA4202F1010114D0596114
:1053000010785A6B8C454FEA201698BF5B619D1848
:10531000511C002A36D15A6983F83060BA42C3F86A
:10532000348002F10101EAD1DEF848301A691E46E4
:10533000C4F3C614511C1961147056F8107FB7429B
:1053400024BF1B611F464FF0010E4FF0000C5A693D
:10535000BA4202F101013FF464AF596110785A6B0F
:105360008E424FEA201598BF5B619C18511C4ABBC6
:105370005A6983F83050BA42C3F834E002F10101AF
:10538000EBD14EE7032985F830005963B2D1C3F859
:105390003090C3F83490ADE7032985F830005963A5
:1053A0007FF47BAFC3F83090C3F8349075E70329DE
:1053B00084F8300059637FF4ECAEC3F83090C3F842
:1053C0003490E6E6032984F830005963BFD1C3F86E
:1053D00030C0C3F834C0BAE7032984F830005963F9
:1053E0007FF404AFC3F830C0C3F834C0FEE6F02C3D
:1053F0007FF417AFB0F86730802B28BF802300F10F
:10540000690C002B3FF40DAF0CEB030901204FF0AA
:105410000008DEF848301CF8011B1A691F46541CAE
:105420001C61117057F8106FBE4224BF1B611E46ED
:105430005A69B24202F1010112D0596114785A6BD3
:105440008F424FEA241A98BF5B619D18511C52B9D4
:105450005A6983F830A0B242586302F10101ECD1DD
:10546000CC45D6D1DDE6032985F830405963DFD13C
:10547000C3F83080C3F83480DAE7FC2C00F2BE8039
:10548000FA2C02D2F82C7FF4CCAE04F10803DBB284
:10549000072B3FF6C6AE012202FA03F313F0DD0F2D
:1054A0003FF4BFAEDEF848301A691F46511C19613F
:1054B000147057F8106FBE4224BF1B611E464FF098
:1054C000010E4FF0000C5A69B24202F101013FF4A3
:1054D000A8AE596110785A6B8F424FEA201598BFD9
:1054E0005B619C18511C4AB95A6983F83050B2422A
:1054F000C3F834E002F10101EBD192E6032984F80C
:1055000030005963DFD1C3F830C0C3F834C0DAE7E4
:10551000836C90F86720196990F868C01F46481C92
:1055200018610C7057F8106F1201BE4202F0700241
:105530000CF00F0C42EA0C0C24BF1B611E464FF00E
:1055400001084FF000095A69B24202F1010114D07A
:10555000596110785A6B8F424FEA201598BF5B61F2
:105560009C18511C002A35D15A6983F83050B24238
:10557000C3F8348002F10101EAD1DEF848301A693B
:105580001F46511C196182F800C057F8106FBE42C7
:1055900024BF1B611E464FF0010E4FF0000C5A69EC
:1055A000964202F101013FF43CAE596110785A6B0A
:1055B0008F424FEA201598BF5B619C18511C9AB925
:1055C0005A6983F830509642C3F834E002F1010181
:1055D000EBD126E6032984F830005963B3D1C3F830
:1055E0003090C3F83490AEE7032984F83000596353
:1055F000D5D1C3F830C0C3F834C0D0E7FE2CFFF4D7
:1056000010AE42E738B54BF69024C1F6FF7494F81B
:105610004C50102D11D94BF26C0405F0B5FFC1F6BA
:10562000FF744BF22030C1F6FF70002106F08EFEB1
:1056300094F84C50102D1BD938BD2046FFF732F896
:105640000028E8D094F86630902B36D083F08003A1
:10565000602B35D94BF69020C1F6FF70FFF796F915
:105660004BF690202946C1F6FF70FFF72FFAD2E7DC
:105670002046FFF7D3FA0028DED094F86630902B4E
:1056800011D083F08003602B10D94BF26C00C1F66F
:10569000FF70FFF7ADFC4BF26C002946C1F6FF70BE
:1056A000FFF746FD38BD94F86830A3B194F8653033
:1056B0009D42EAD0002DE8D0EDE794F8683033B190
:1056C00094F865309D42C5D0002DC3D0C8E7802333
:1056D00084F86630F4E7802384F86630E6E700BF9C
:1056E00070B54BF2282082B0C1F6FF7003F0C8F805
:1056F00018B9FFF787FF02B070BD4BF27C10C1F6FE
:10570000FF7003F0BDF80028F3D04BF21C06C1F681
:10571000FF7608F0CFFD3368C01AB0F5356FE8D9D1
:1057200049F23464C2F200044BF2242508F0C2FDB1
:10573000C1F6FF75236800932A68009B30609B1AAE
:1057400041F28832934200F2DF804BF22820C1F60A
:10575000FF7003F0A5F80546002800F0DC804BF24E
:105760007C10C1F6FF7003F09BF80446002800F09F
:10577000E08008F09FFD48F2F803C2F200030646FD
:10578000186803682A461B682146984708F092FD6E
:1057900040F65A33801B984206D948F20013C2F2F1
:1057A00000031A6801321A6048F20413C2F20003BF
:1057B0001A88824238BF188072B64BF2DC23C1F6D9
:1057C000FF731A7F02F0FF010AB100221A7762B656
:1057D00059B372B647F6FF764FF40040B3F91E1086
:1057E000B3F92020DE83188462B6002982EAE273CE
:1057F000A3EBE273B8BF49428B42B8BF0B4607EE3A
:10580000903ADFED536AF8EEE77A87EEA67AF7EE84
:10581000007AB4EEE77AF1EE10FA06DD48F2FC0306
:10582000C2F200031A6801321A6072B64BF25813C2
:10583000C1F6FF731A7F02F0FF010AB100221A7746
:1058400062B659B372B647F6FF764FF40040B3F92B
:105850001E10B3F92020DE83188462B6002982EA84
:10586000E273A3EBE273B8BF49428B42B8BF0B4669
:1058700007EE903ADFED366AF8EEE77A87EEA67A21
:10588000F7EE007AB4EEE77AF1EE10FA06DD48F2B0
:10589000FC03C2F200031A6801321A6049F248633D
:1058A000C1F6FF7393ED007AA11E05F1FE00AC1E58
:1058B00034F9023F07EE903AF8EEE77A844267EE59
:1058C000877AFDEEE77A17EE903A238031F9023FAE
:1058D00007EE903AF8EEE77A67EE877AFDEEE77A20
:1058E00017EE903A0B80E3D14BF22820C1F6FF70FF
:1058F00002F0E8FF4BF27C10C1F6FF7002F0E2FF0D
:10590000FFF780FE02B070BDFEF770F823680193C8
:10591000019B2B6019E743F67C302621C0F2010081
:105920000AF02EFA49F61400C1F6FF7007F042FDA6
:1059300015E743F6A4302621C0F201000AF020FA50
:1059400049F61400C1F6FF7007F034FD11E700BFFF
:1059500000FEFF462DE9F04F4BF69026C1F6FF768C
:1059600087B007F029FF96F864300024012249F23D
:10597000F87743F0010362F347034FF6FF782146BF
:1059800086F8654086F8664086F8674086F8684085
:1059900086F8E940C1F6FF7706F16900802286F8B3
:1059A0006430B76486F84C4086F84D4086F84E4027
:1059B0007465B465C6F85C80C6F860800DF09CFA2A
:1059C00049F2406240F26D41C0F200013046C1F63A
:1059D000FF7234607460B460F46034617461B46107
:1059E000F46134627462B462F46234637463B46305
:1059F000F463346474640AF035FF4BF22033C1F66B
:105A0000FF734BF6582742F2C822C1F6FF77C0F267
:105A10000E025C6018469C604BF26C06C1F6FF7685
:105A20001A6006F053FB07F1180349F2406240F296
:105A30007141BC613C607C60BC60FC60BB62FB622D
:105A4000FC613C627C623846C1F6FF72C0F2000124
:105A50003F617F610AF006FF96F8643086F8654082
:105A6000012243F0010362F34703214686F86640B2
:105A700086F8674086F8684086F8E94006F16900D4
:105A8000802286F86430B76486F84C4086F84D4032
:105A900086F84E407465B465C6F85C80C6F86080D0
:105AA0000DF02AFA4BF2282849F2406240F2754183
:105AB000C1F6FF783046C1F6FF72C0F200014BF22A
:105AC0007C17C1F6FF7734607460B460F4603461B1
:105AD0007461B461F46134627462B462F462346318
:105AE0007463B463F4633464746442F28C150AF032
:105AF000B9FE4BF2DC2B224621464046FDF754F915
:105B0000C1F6FF7BC0F20E0522462146384688F8D2
:105B10009C40C8F8984088F89D40C8F80050FDF7B0
:105B200043F941F644630BF118025846012187F806
:105B30009C401E463D60C7F8984087F89D400297FC
:105B40004BF2581AFDF730F94BF690374FF40043FB
:105B5000C1F6FF7AABF82030019342F24C093B4684
:105B60000AF118020121C0F20E0947F6FF75C1F6CD
:105B7000FF735046C2F200061F46CBF80090ABF808
:105B80001E500096FDF710F94BF23406019B009869
:105B9000AAF82030C1F6FF76CAF80090AAF81E5085
:105BA00002F020F848F268153846C2F20005019765
:105BB0004BF6442902F016F842F2741706F1280257
:105BC00004213046FDF7F0F8C1F6FF794FF4803339
:105BD00005F128020421C0F20E0728463760B361A0
:105BE000F361336273620393FDF7DEF8039BAB61ED
:105BF0004846EB612B626B6289E8000989F808402E
:105C000089F80940C9F80C4089F810402F604BF220
:105C1000C82B06F0C7FF49F2406240F27941C1F655
:105C2000FF7BC1F6FF72C0F2000148460AF01AFE7F
:105C3000029FCBF804A05846CBF800708BF80840C0
:105C40008BF80940CBF80C408BF810404BF2003930
:105C500006F0A8FF49F2406240F27941C1F6FF79AF
:105C6000C1F6FF72C0F2000158460AF0FBFD009B2E
:105C7000C9F804304846C9F8008089F8084089F816
:105C80000940C9F80C4089F8104048F2E40A06F0CF
:105C900089FF49F2406240F27941C2F2000AC0F243
:105CA00000014846C1F6FF720AF0DCFD019ACAF80D
:105CB00000705046CAF804208AF808408AF8094063
:105CC000CAF80C408AF810404BF67C3906F06AFF9F
:105CD00049F2406240F27941C1F6FF79C1F6FF72A4
:105CE000C0F2000150460AF0BDFD4846C9F80080E8
:105CF00089F8084089F80940C9F80C4089F8104033
:105D0000C9F804604BF6E01806F04CFF49F2406217
:105D100040F27941C1F6FF78C1F6FF72C0F200018E
:105D200048460AF09FFD3B46404688E8280088F830
:105D3000084088F80940C8F80C4088F8104006F080
:105D400031FF49F2406240F27941C1F6FF724046AC
:105D5000C0F200014BF6F4170AF084FDC1F6FF779C
:105D6000009B3C7238464FF0010187E84800797289
:105D7000FC603C7406F016FF49F2406240F2794143
:105D8000C0F200013846C1F6FF724BF608280AF04F
:105D900069FDC1F6FF78019A88F808404FF00103C9
:105DA000404688F8093088E82400C8F80C4088F894
:105DB000104006F0F7FE49F2406240F27941C1F628
:105DC000FF72C0F2000148F2281740460AF04AFD6F
:105DD000C2F2000743F2FC30C0F20100022107F1D9
:105DE000180223463C72FC603860797220463A61A2
:105DF0003C4600E0226942F82300797A013348F2F8
:105E000028129942C2F20002F4DC49F28853C2F22D
:105E10000003196809B9B9E019464B69002BFBD199
:105E20004F61002448F2281048F2481B42F28013C8
:105E3000C2F2000BC0F20E03C2F200007C61BC8013
:105E4000FC80BC723B6048F2081A02F0E7FB0BF1E1
:105E50001C0258460121FCF7A7FFC2F2000A4BF6CC
:105E60001C2942F26813C1F6FF79C0F20E030AF151
:105E70001C024FF4803801215046CBF800300093CB
:105E8000CBF81880FCF790FF009BCAF8003048461A
:105E9000CAF8188089E8400889F8084089F809405C
:105EA000C9F80C4089F810404BF6302806F07AFE0D
:105EB00049F2406240F27941C1F6FF78C1F6FF72C3
:105EC000C0F2000148460AF0CDFC404688E82004B4
:105ED00088F8084088F80940C8F80C4088F8104055
:105EE0004BF2200606F05EFE49F2406240F2794134
:105EF000C1F6FF76C1F6FF72C0F2000140460AF01B
:105F0000B1FC012330467372C6F800B0776034727A
:105F1000F460347441F6306506F044FE49F24062A4
:105F200040F27941C2F20005C1F6FF72C0F20001F1
:105F300030460AF097FC2846C5F800A06F602C7226
:105F40006C72EC602C7406F02DFE49F2406240F257
:105F50007941C1F6FF72C0F2000128460AF082FCC6
:105F600008F0A8F949F23463C2F200034BF21C02B4
:105F70001B6805934BF22423C1F6FF72C1F6FF7331
:105F800005991060196007B0BDE8F08F1A6048E706
:105F900000F5815382681B7803EBC30302EBC30354
:105FA00003EB810191ED000A704700BF2DE9F04F2E
:105FB0002DED048B844600F5805385B000F6E47423
:105FC00000F6E87500F6EC7900F57F6800F57D6B6A
:105FD000D3ED014AD4ED000A95ED000A99ED003A9F
:105FE000D8ED003ADBED002ADCF8BCEF9FED9C5ABF
:105FF000DFED9C9A0CF6D47300F6D8701C4690ED39
:10600000001A02930CF6DC700CF57E6393ED008AA7
:1060100094ED004AD0ED008A02F1FE030239A2F1AC
:10602000020A0193F6EE001AB7EE002ABFEE009ABC
:10603000BEF1000F9FED8C6A40F30481DCF8C06F65
:10604000F0EE465A0CF53C70002550F8307C50F8C4
:10605000343C50F82C2C50F8284C3B4402EB2342A3
:1060600001359BB2A2422DB240F82C2C40F8303CB6
:1060700004DD50F8244C121B40F82C2C06EB420493
:1060800036F91220B4F9027010ED087A50ED076A63
:10609000BF1A03FB07F302EB234307EE903AF8EE37
:1060A000E77A67EE266A67EE877A40ED086A67EE60
:1060B000857AF5EEC07AF1EE10FA0EDD24EEA77ABD
:1060C000E7EEC77AB0EE677AF1EE667AB4EEE77A79
:1060D000F1EE10FA58BFF0EE477A50ED036A10ED7A
:1060E000027A7545E7EEA65A00F13400A7EE876AFA
:1060F000ABDB36EE637A75EEC37AE7EE003A029BCD
:10610000A7EE803AE1EE042A36EE637AA2EEC14AA7
:10611000A7EE206A75EEC37A26EE087AE7EEA05A5B
:10612000A4EE076A65EEA87A26EE216AE4EE275A05
:10613000B4EEC26AF1EE10FA89ED003A65EEA15AAA
:10614000C8ED003ACBED002A83ED004A6CDD47F63E
:10615000FF73F4EEC25AF1EE10FA57DD47F6FF7204
:106160002AF8022F21F8023F019B9A457FF460AF85
:10617000DFED3E7AB0EEC33AB4EEE73ADFED3B7ABC
:10618000F1EE10FAF0EEE33A48BF0023F4EEE73AFE
:1061900048BFC9F80030F1EE10FA44BF0023C8F838
:1061A0000030BEF1000F2CDD00239FED317A1E463A
:1061B000342706E0DCF8BCEF013636B276453346CC
:1061C0001FDA07FB03C3D3EDB47A0EF1FF3EF4EE02
:1061D000C77A07FB0EC4F1EE10FA04F52F7403F52D
:1061E0002F75E7D50FCCCCF8BCEF0FC50FCC0FC582
:1061F0000FCC0FC5013636B223682B607645334687
:10620000DFDB05B0BDEC048BBDE8F08FF4EEC95ABE
:10621000F1EE10FA19D465EEA95AFDEEE57ACDED4E
:10622000037ABDF90C209BE7B4EEC96AF1EE10FACF
:1062300010D426EE296AFDEEC67ACDED037ABDF9BB
:106240000C3086E7F0EE465A53E748F20102CFF6EB
:10625000FF7285E748F20103CFF6FF7379E700BFCD
:106260000000003800FEFF4600000000FFE6DB2EC5
:1062700017B7D13810B54FF48843C4F22C7343F2EA
:10628000C672C360C3F2BE7200F5815302611B780F
:1062900082689FED127ADFED127A03EBC30302EB03
:1062A000C303D3ED056AE6EE877A044604F6D87494
:1062B00017EE900A0BF090FF41EC100B0AF0D8FAA1
:1062C00051EC100B0CF0D4FADFED067A07EE100A51
:1062D00067EE277AC4ED007A10BD00BF3D0AC740C3
:1062E0003D0A27C0716415392DE9F8432DED028B65
:1062F00000F5815386681B78072903EBC30306EB7F
:10630000C30657D00FD9402901D0422936D102F017
:106310004002D2B2C0F8CC2F002A5ED0BDEC028B76
:106320000120BDE8F883012928D107EE902ADFED8E
:106330004B6A9FED4B7AF8EE677A00F5805367EE73
:10634000A67AF4EEC77AF1EE10FAC3ED077AE5DD2E
:1063500000F6DC7300F57E60C3ED007AC0ED007AD4
:10636000D6ED046AB6EE007AF4EEC76AF1EE10FAE2
:10637000D4D5F1EE677AC0ED007ACFE77A29CDD98E
:1063800047F2A401C3F67D71034600F55062C3F8DD
:10639000D41234339342FAD1BDEC028B00F5805312
:1063A0000022C4F220320021C0F8CC1F01209A60E4
:1063B000BDE8F88312FB02F207EE902ABDEC028BD7
:1063C000F8EEE77A9FED277A67EE877A00F580503E
:1063D000C0ED067A0120BDE8F8830746044600F5C3
:1063E0005065B1EE048A02E03434A54296D0D4F868
:1063F000EC32802BF8D1D7F8CC3F002BF4D13869A0
:1064000080F000400BF0E8FED6ED017A67EE887A66
:10641000804617EE900A89460BF0DEFE0B4641F6E9
:10642000B8610246C4F21D014FF0A0400BF074FDAC
:1064300041EC100B0AF01CFA404653EC102B494675
:106440000BF01EFF41EC100B0AF012FA51EC100B8E
:106450000CF00EFAC4F8D402C6E700BF2497FF3B45
:10646000CDCC4C3DACC5A73770B500F581532DEDB3
:10647000028B19708568D0ED045A9FED6D7A9FEDFF
:106480006D5AC9B201EBC10105EBC10595ED024A98
:1064900095ED036AF2EE084AF9EE087AE4EE247A02
:1064A00000F6E47300F6E876F1EE006A66EE266A1E
:1064B000BFEE008AF0EE484AE6EE264A0446FDEEBC
:1064C000E77AF6EE008A17EE902AC0F8C82FC3EDDF
:1064D000004AD5ED037AF4EEE87AF1EE10FAD4BF73
:1064E000F0EE457AF0EE477AC6ED007A65EEE77A8F
:1064F00017EE900A0BF070FE41EC100B0AF0B8F9A1
:1065000051EC100B0CF0B4F907EE100AF7EE007A1C
:1065100077EEC77AB0EE007AC6ED007AD5ED047A50
:10652000A7EE878A04F6DC7204F57E6382ED008AAA
:1065300083ED008A95ED047AB4EEE87AF1EE10FA74
:1065400003D5F1EE487AC3ED007ADFED3B6A95EDB5
:10655000056A9FED3A7AD4ED047A9FED398AA6EE6A
:10656000267A04F6D87627EE888A17EE100A0BF002
:1065700033FE41EC100B0AF07BF951EC100B0CF0E0
:1065800077F907EE900A27EE888AF7EE007A86ED13
:10659000008A95ED067A77EE277A04F5805377EE38
:1065A000877AF5EE006AC3ED057A95ED067AB4EECA
:1065B000E67AF1EE10FA03F1140309D5B0EE086A99
:1065C000F6EE086AE7EE466A77EEE67AC3ED007A01
:1065D00095ED077A9FED1B6ADFED1B7ADFED1B6AF5
:1065E00027EE067A04F6C47383ED007A95ED097AF6
:1065F000B6EE006A37EE467A04F6F87383ED007A59
:1066000095ED0A7A67EE277A04F5805367EE877A6C
:10661000002204F6FC71C1ED007ABDEC028B1A6019
:10662000D5ED0B7A67EEA67AC3ED017A70BD00BF97
:1066300000C05A4600409C453D0AC7403D0A27C05D
:10664000560EC9408FC2F53C2DB29D3D6666E63FB1
:1066500070B52DED028B00F5815285681378D0ED71
:10666000045A9FED717A9FED715A03EBC30305EB5A
:10667000C30303EB810181ED000A137803EBC3032D
:1066800005EBC30595ED024A95ED036AF2EE084A63
:10669000F9EE087AE4EE247A00F6E47300F6E87680
:1066A000F1EE006A66EE266ABFEE008AF0EE484A16
:1066B000E6EE264A0446FDEEE77AF6EE008A17EE8D
:1066C000902AC0F8C82FC3ED004AD5ED037AF4EE46
:1066D000E87AF1EE10FAD4BFF0EE457AF0EE477AA0
:1066E000C6ED007A65EEE77A17EE900A0BF074FDBE
:1066F00041EC100B0AF0BCF851EC100B0CF0B8F8A0
:1067000007EE100AF7EE007A77EEC77AB0EE007A5D
:10671000C6ED007AD5ED047AA7EE878A04F6DC721E
:1067200004F57E6382ED008A83ED008A95ED047A9C
:10673000B4EEE87AF1EE10FA03D5F1EE487AC3ED43
:10674000007ADFED3B6A95ED056A9FED3A7AD4ED6C
:10675000047A9FED398AA6EE267A04F6D87627EEDB
:10676000888A17EE100A0BF037FD41EC100B0AF087
:106770007FF851EC100B0CF07BF807EE900A27EE37
:10678000888AF7EE007A86ED008A95ED067A77EE34
:10679000277A04F5805377EE877AF5EE006AC3ED29
:1067A000057A95ED067AB4EEE67AF1EE10FA03F189
:1067B000140309D5B0EE086AF6EE086AE7EE466AF9
:1067C00077EEE67AC3ED007A95ED077A9FED1B6AC6
:1067D000DFED1B7ADFED1B6A27EE067A04F6C47341
:1067E00083ED007A95ED097AB6EE006A37EE467AC7
:1067F00004F6F87383ED007A95ED0A7A67EE277A4E
:1068000004F5805367EE877A002204F6FC71C1ED2F
:10681000007ABDEC028B1A60D5ED0B7A67EEA67A92
:10682000C3ED017A70BD00BF00C05A4600409C45D0
:106830003D0AC7403D0A27C0560EC9408FC2F53CED
:106840002DB29D3D6666E63F70B52DED028B00F5DD
:10685000815385681B78D0ED045A9FED6C7A9FEDCB
:106860006C5A03EBC30305EBC30595ED024A95EDA6
:10687000036AF2EE084AF9EE087AE4EE247A00F6AA
:10688000E47300F6E876F1EE006A66EE266ABFEE83
:10689000008AF0EE484AE6EE264A0446FDEEE77A24
:1068A000F6EE008A17EE902AC0F8C82FC3ED004A12
:1068B000D5ED037AF4EEE87AF1EE10FAD4BFF0EEFB
:1068C000457AF0EE477AC6ED007A65EEE77A17EE84
:1068D000900A0BF081FC41EC100B09F0C9FF51EC60
:1068E000100B0BF0C5FF07EE100AF7EE007A77EEFB
:1068F000C77AB0EE007AC6ED007AD5ED047AA7EE3D
:10690000878A04F6DC7204F57E6382ED008A83EDEB
:10691000008A95ED047AB4EEE87AF1EE10FA03D528
:10692000F1EE487AC3ED007ADFED3A6A95ED056A3B
:106930009FED397AD4ED047A9FED388AA6EE267A57
:1069400004F6D87627EE888A17EE100A0BF044FC7E
:1069500041EC100B09F08CFF51EC100B0BF088FF91
:1069600007EE900A27EE888AF7EE007A86ED008A15
:1069700095ED067A77EE277A04F5805377EE877ADD
:10698000F5EE006AC3ED057A95ED067AB4EEE67A87
:10699000F1EE10FA03F1140309D5B0EE086AF6EE31
:1069A000086AE7EE466A77EEE67AC3ED007A95ED7F
:1069B000077A9FED1B6ADFED1B7ADFED1B6A27EE7E
:1069C000067A04F6C47383ED007A95ED097AB6EE83
:1069D000006A37EE467A04F6F87383ED007A95ED97
:1069E0000A7A67EE277A04F5805367EE877A0022E9
:1069F00004F6FC71C1ED007ABDEC028B1A60D5ED96
:106A00000B7A67EEA67AC3ED017A70BD00C05A46D4
:106A100000409C453D0AC7403D0A27C0560EC9406C
:106A20008FC2F53C2DB29D3D6666E63F2DE9F84FDD
:106A30004FF4884243F2C67343F6D431C4F22C7249
:106A4000C3F2BE73C0F2010104460160C26003617B
:106A50004FF4107007F0E8F943F6EC32C0F201028F
:106A6000034603CA43F6F432C0F2010243F6FC388F
:106A70009688DFEDEB7A92F806B01863C0F2010851
:106A800046F2666C48F2061A00254FF07A5EC3F6AD
:106A9000267C4FF07E57C3F6156A1068A3F87C6019
:106AA0004FF07C5243F6044659639867C3F814C00C
:106AB000C3F818E01F62C3F828A0DD6283F87EB037
:106AC0001F65C3F85CC0C3F860E09F66A3601A60EE
:106AD0005A609A60DA601A61DA615A629A64DA641A
:106AE0009A655A66C3ED157AC0F20106DA66D8F8DF
:106AF0000000C3F8C00003CE4EF26D7943F60C4699
:106B0000B8F804B098F80680C3F870A0C3F67B69A3
:106B1000C0F20106A3F8C4B083F8C680C3F8985049
:106B2000C3F89C50C3F8A4C0C3F8A8E0C3F8B07081
:106B3000C3F8BC50C3F8E8E0C3F8ECC0C3F8F0E019
:106B4000C3F80801C3F80C11C3F8B8905A67C3F82A
:106B50009020C3F89420C3F8A020C3F8AC20C3F859
:106B6000B420C3F8D820C3F8DC20C3F8E020C3F871
:106B7000E420C3F8F420C3F8F87003CE43F61446BB
:106B8000C0F20106C3F85001C3F8541103CEB04659
:106B9000C3F80091C3F848914FF07D59C3F8309184
:106BA00038F80899C3F80451C3F834C1C3F838E180
:106BB000C3F84071C3F84C51C3F89801C3F89C1155
:106BC000A3F8A091C3F87CC1C3F880E1C3F8FC200E
:106BD000C3F82021C3F82421C3F82821C3F82C21AD
:106BE000C3F83C21C3F84421C3F86821C3F86C21E1
:106BF000C3F87021C3F87421C3F87821C3F8842145
:106C0000B8E80300083EC3F8E001C3F8E41103CE7E
:106C100004F581580026C3F88871C3F890A1C3F821
:106C20009451A3F8E891C3F8C4C1C3F8C8E1C3F80C
:106C3000D071C3F8D8A1C3F8DC51C3F82802A3F877
:106C40003092C3F82C12C3F80CC2C3F88C21C3F8DD
:106C5000B021C3F8B421C3F8B821C3F8BC21C3F8EC
:106C6000C021C3F8CC21C3F8D4212046C3F8F821B1
:106C7000C3F8FC21C3F80022C3F80422C3F8082299
:106C8000C3F810E288F80060C3F81872C3F820A2B5
:106C9000C3F82452C3F81422C3F81C22FFF7D4FD12
:106CA000E6615126C4F8BC615426C4F8F461572645
:106CB000C4F8F8615B26C4F830625D26C4F834621B
:106CC0006026C4F86C6243F6204340F2E736C0F217
:106CD0000103C4F8706242F21C16C4F8C03F266279
:106CE000392341F23016C4F8CC3066623C2342F2BC
:106CF0001D16C4F8043126633F2343F67876C4F8A2
:106D000008316663432341F22736C4F84031A66355
:106D1000452343F67976C4F844316664482348F243
:106D200005762420C4F87C31A6644B2341F6FE0688
:106D30004FF027084FF02B0C4FF02D0E30274FF05F
:106D4000330B6061C4F8803137204F23E66448F28A
:106D50000676C4F81880C4F850C0C4F854E0C4F8EB
:106D60008C70C4F890B0C4F8C800C4F8B831A665F7
:106D70004AF2A816E66540F6627626664AF2A91639
:106D8000E6664BF2C026266743F2223140F2616686
:106D9000C0F2010166674FF2AE234BF2C126C0F28A
:106DA0000103C4F88060C4F8AC104FF6BB6640F62F
:106DB0009B0148F6230CC0F2010CC4F88460C4F8AF
:106DC000B01041F27D46C4F8F83041F6C14A40F6B1
:106DD0001B4341F6C24943F2233845F22051C0F229
:106DE000010AC0F20109C0F20108C4F88860C0F2CB
:106DF00002014FF6BC66C4F8C0C0C4F800314FF4BD
:106E0000C75C41F2BC0348F6240E4CF249674FF2CE
:106E1000AD20C0F2010EC0F20107C0F2010001E096
:106E2000CDCC4C3FC4F89460C4F898A0C4F8A890A6
:106E3000C4F8BC80C4F8C4C0C4F81431C4F820112C
:106E40002A4640F64C714CF24A6543F2F12643F271
:106E5000F22A45F21F594AF233484AF2344C49F2B9
:106E60004A13C0F20105C0F20206C0F2020AC0F2E3
:106E70000209C0F20208C0F2020CC4F8D0E0C4F863
:106E8000D470C4F8E80042F6D40741F26140C0F281
:106E90000303C4F828114FF2DE0E40F67931C0F238
:106EA000020EC4F8D870C4F8E450C4F8EC00C4F87A
:106EB000FC60C4F80CA1C4F81091C4F82481C4F893
:106EC0009C1045F27476C4F834C14CF6CC08C4F872
:106ED0003C11C4F8843141F27C2141F20203C0F23A
:106EE0000306C0F20308C4F838E1C4F85011C4F82E
:106EF0008C3141F27D2141F203034FF2DF0741F66D
:106F0000367541F6377045F2737B49F2491A4CF6F3
:106F1000CB0940F6474C40F6484EC0F20207C0F29B
:106F20000305C0F20300C0F2030BC0F2030AC0F273
:106F30000309C0F2040CC0F2040EC4F86411C4F8D2
:106F4000706140F6ED01C4F89881C4F8A0314CF2AC
:106F5000F64640F6196345F2D928C4F84871C4F8DA
:106F60004C51C4F85C01C4F860B1C0F20406C4F826
:106F700074A1C4F87811C4F88891C0F20508C4F867
:106F80009CC1C4F8ACE1C4F8B43144F68F6740F654
:106F90008E1344F6906547F6903047F6913B4CF2DD
:106FA000F74140F6D81A40F6D91945F2DA2C49F2E1
:106FB0006B4EC0F20407C0F20405C0F20400C0F238
:106FC000040BC0F20401C0F2050AC0F20509C0F2C8
:106FD000050CC0F2050EC4F8C831C4F8D86141F6FA
:106FE000860340F6EB06C4F8008240F68128C4F818
:106FF000B071C4F8C051C4F8C401C4F8D4B1C4F825
:10700000DC31C4F8E811C4F8ECA1C4F8F061C4F8AC
:10701000FC91C4F8048249F26C47C4F810C24DF6E2
:10702000AD259D20C4F814E241F2121EC0F20507FE
:10703000C0F20505C0F2060043F21D2B45F21733DE
:1070400047F208214DF6AE264FF09C0943F21E2868
:1070500045F2163CC4F818E241F2694EC0F206034C
:10706000C0F20506C0F20609C0F20608C0F2060C1E
:10707000C0F2060BC0F20601C4F82472C4F828520C
:1070800041F2AA1740F6790AC4F82CE2C4F860026B
:1070900040F6FB2E40F6021047F2A405C4F89C32DD
:1070A000C4F87C02C4F89002C4F864B2C3F67D75DB
:1070B000C4F86872C4F8A012C4F8A4A2C4F8386274
:1070C000C4F84C62C4F83C92C4F85092C4F874827C
:1070D000C4F88882C4F878C2C4F88CC2C4F840E20C
:1070E000C4F854E2234604F55060C3F8D022C3F834
:1070F000D452343383424FF00001F6D104F580506E
:1071000002464CF6CD47002604F6D875C3F64C6708
:10711000C4F2203687610023966004F57F6004F690
:10712000D47204F57D6704F6EC76C4F8BC3FC4F86D
:10713000CC3F29604FF07E553960016031602046B8
:1071400015606360FFF780FB2046BDE8F88F00BF45
:107150002DE9F04F2DED028B064600F58150B36806
:1071600090F800A0B2F100080AEBCA0A83B00D46FD
:1071700003EBCA0A40F3C881D6F8BC4F3F2C40F35A
:10718000A0810024DFEDEA7A2346324692EDB47AFC
:10719000B4EEE77AF1EE10FA48BF1C4603F10103A2
:1071A00048BFF0EE477A402B02F13402EED1A5F150
:1071B0003C094EF64F4309FB09F2C4F6C46383FB56
:1071C0000231D317C3EBA10303EB430103EB8103AC
:1071D000D31A07EE903AF8EEE77AB1EE0A7A06F69D
:1071E000FC7106F6F87377EEC77AD3ED006A91ED7D
:1071F000007A3C2DE7EE276A09DD07EE102A06F536
:107200008053D3ED007AB8EEC77AE7EE876AD6F8F6
:10721000C83FB2691A44AA4280F20082726D1A44D1
:10722000954240F30D82D6F890201A44954240F3DF
:107230000582D6F8CC201A44954240F3FD81D6F859
:1072400008211A44954240F3F581D6F844211A44A6
:10725000954240F3ED81D6F880211A44954240F3DF
:10726000E581D6F8BC211A44954240F3DD81D6F879
:10727000F8211A44954240F3D581D6F834221A44B5
:10728000954240F3CD81D6F870721F44BD42CCBF09
:1072900021271E274FEA870B0BEB070306EB83031F
:1072A000D6ED047A5B699FEDA38A9FEDA36AEB1A82
:1072B00007EE103AB8EEC77A27EE888A77EE267A7C
:1072C00067EE867A17EE900A0AF086FF41EC100B03
:1072D00009F0CEFA342303FB046351EC100B009346
:1072E0000BF0C6FA07EE900A27EE888A009BBEEEE6
:1072F000C88A0022B8F1300FC3F8C02283EDAF8AEC
:1073000006DDB8F1500FD4BF013702374FEA870BC3
:107310005F4406EB870706F58052F869796A3B6A95
:10732000D2ED058A342707FB0467013BC7F8C83252
:10733000C7F8C402C7F8CC1218EE900A0AF04CFF46
:1073400007EE908A9FED7D7AF8EEE77ACDE90001AD
:1073500067EE877AB0EE088A17EE900A0AF03CFFD3
:107360009DED001B41EC100B09F006FBF0EE007ADE
:1073700051EC100BA8EEA78A0BF07AFA07EE900AF0
:1073800028EE278A3C2D87EDB48A00F32881DAEDB8
:10739000046A9FED6B7ADFED6B5ADFED6B7A9FED40
:1073A0006B6A96ED048A06F5805393ED025A66EEF9
:1073B000A66AA8F14008A6EE857A06F5805306F580
:1073C000805105EE105AF0EE476A07EE108AD3EDB1
:1073D000034AB8EEC77AB8EEC55AE4EE876A34239A
:1073E00003FB0463E5EE257AC3F8EC5206F6C4729B
:1073F000F4EEE76AF1EE10FA58BFF0EE667AF4EEBA
:10740000C67AF1EE10FAD4BF67EEA77ADFED507AB4
:1074100068EE277A0B2DC3EDB87A5EDD6C2D40F354
:107420001181D1ED067A92ED007A9FED4A6A27EE3E
:10743000877AF0EE675AE7EE065A4EF685394FF036
:10744000A858F0EE006AB0EE657AC4F20109B0EE19
:10745000476A97EEA66A83EDBA7A83EDB96ADAEDE8
:10746000007A77EEA77A17EE900A0AF0B5FE024688
:107470000B46404649460AF04FFD41EC100B09F01F
:10748000F7F9F1EE487A53EC102B17EE900ACDE99C
:1074900000230AF0A1FEDDE900230AF0F1FE41EC31
:1074A000100B09F0E5F9342351EC100B03FB0466D3
:1074B0000BF0DEF9C6F8D40203B0BDEC028BBDE8D8
:1074C000F08F342303FB04630022611CC6F8BC1F49
:1074D000C3F8DC22C3F8D82269E6D1ED067A92ED32
:1074E000007A9FED1D6A27EE877AF0EE675AE7EE85
:1074F000065A47F6E1294FF02058F0EE006AB0EE48
:10750000657AC3F6D479A2E7344606F550674FF0A2
:10751000800B02E03434A742CED0D4F8EC329D4246
:10752000F8D1D6F8CC3FDBB1C4F8ECB2F2E700BF3B
:107530000000C6420000FA4620986C3D2497FF3BAD
:1075400000004842CDCCCC3E00005C4200005243DB
:1075500000442C4700004042000040C20AD7233CB0
:10756000306980F000400AF037FECDE9000128467E
:107570000AF020FE47F6E1234FF08042C3F6847301
:107580000AF07EFE00230022C4F218030AF0C6FCB3
:107590009AED017AF1EE047A67EE277A804617EECB
:1075A000900A89460AF018FE02460B4640464946B4
:1075B0000AF0B2FC41EC100B09F05AF9DDE90001C8
:1075C00053EC102B0AF05CFE41EC100B09F050F963
:1075D00051EC100B0BF04CF9C4F8D4029AE7C5F14A
:1075E0003C0307EE903A1FED237AF8EEE77A67EE58
:1075F000877A17EE900A0AF0EFFD41EC100B09F0C4
:1076000037F951EC100B0BF033F9D7EDB47A07EEE4
:10761000100A67EE877AC7EDB47AB8E6002739E634
:107620001B2737E6182735E6152733E6122731E6FC
:107630000F272FE60C272DE609272BE6062729E63C
:10764000032727E691ED067AD2ED006A07EE909ABD
:1076500067EE266AF8EEE77AF0EE475AE6EEA75AAA
:107660002B2DB0EE006AF0EE656AD7EE066AC3ED28
:10767000BA5AC3EDB96A06DC47F6E1294FF0205843
:10768000C3F6D479EBE628460AF094FD4BF6510395
:107690004FF06042C3F69E730AF0F2FD0023002211
:1076A000C3F6F0730AF038FC80468946D7E600BF7F
:1076B00070B50021064605F0F1F9C0B1B6F91E40DB
:1076C000B6F92010031D00F5827533F9022B9442A0
:1076D000A8BF14469142B8BF11469D42F5D8012378
:1076E000F48331843377BDE8704005F08FB970BD05
:1076F0002DE9F04F9BB0044605F030F916900028B4
:1077000000F05F820021204605F0C8F9179000289C
:1077100000F0608242F25003C0F20E03199345F26A
:107720004C6945F24E6734F90930049345F25266CC
:10773000E35F099345F25460A35F089345F25661F5
:10774000235E189345F25862635E059345F25A6AC8
:10775000A35E079334F90A30069304F5AC431A4646
:1077600004F5C5491E46CDF8449002F13C093E326D
:107770000B9206F140020C9206F142020D9206F1C4
:1077800044020E9206F146020F9206F14802119B46
:10779000109232464A3203921A46183211921A4611
:1077A0001A3245F25065129245F25E681A4645F269
:1077B0005C6C45F2606E1C321E3334F905B01392D6
:1077C00034F9088034F90CC034F90EE0CDF8089093
:1077D0001493179B18989A1C0192169A03F58173BB
:1077E00002321593019B0A924FF0000A5D4633F96D
:1077F000022F019302EB021202EB0222520022F34B
:107800004F42029B04991E8804EB460701FB0CF9CA
:10781000B7F91C3003FB089929F3CF390FFA89F126
:10782000049112B201FB0EF929F3CF39914409F307
:107830000F090136A7F81C900299B6B240F25B47D7
:10784000BE4294BF0E80A1F800A00B99099F0E883C
:1078500004EB460907FB0CFBB9F9D4783B4407FB62
:1078600008BB2BF3CF3B0FFA8BF7099707FB0EF7FB
:1078700027F3CF37174407F30F070136A9F8D47859
:107880000B99B6B240F2A347BE4294BF0E80A1F856
:1078900000A00C990E8804EB460707F590571C379B
:1078A000B7F9009005FB0CF54B4409FB085525F38F
:1078B000CF352DB205FB0EF929F3CF39914409F3E9
:1078C0000F090136A7F80090B6B240F2FC47BE425D
:1078D00094BF0E80A1F800A00D990E88089904EBC2
:1078E000460707F5E0571637B7F9009001FB0CFB88
:1078F0004B4409FB08BB2BF3CF3B0FFA8BF9CDF8B8
:10790000209009FB0EF929F3CF39914409F30F09AF
:107910000136A7F800900D99B6B240F24B57BE421F
:1079200094BF0E80A1F800A00E990E8804EB4607C4
:1079300007F51A572E37B7F9009000FB0CF04B44AF
:1079400009FB080020F3CF3000B200FB0EF929F349
:10795000CF39914409F30F090136A7F80090B6B268
:1079600040F28D57BE4294BF0E80A1F800A00F993F
:107970000E88059904EB460707F547570A37B7F90C
:10798000009001FB0CFB4B4409FB08BB2BF3CF3BE6
:107990000FFA8BF9CDF8149009FB0EF929F3CF39C2
:1079A000914409F30F090136A7F800900F99B6B278
:1079B00040F2D257BE4294BF0E80A1F800A01099A9
:1079C0000E88079904EB460707F575573037B7F966
:1079D000009001FB0CFB4B4409FB08BB2BF3CF3B96
:1079E0000FFA8BF9CDF81C9009FB0EF929F3CF396A
:1079F000914409F30F090136A7F800901099B6B227
:107A000040F21467BE4294BF0E80A1F800A0039913
:107A10000E88069904EB460707F593471A37B7F91E
:107A2000009001FB0CF14B4409FB081121F3CF310D
:107A300009B2069101FB0EF929F3CF394A4402F34A
:107A40000F020136B6B2B6F5CA6F3A808ABF039A02
:107A50000399A2F800A047F6E12298BF0E8002FB2E
:107A600003F323F34F4311990E8804EB460707F500
:107A7000AC470FFA83F9B7F9622003EB6203A7F86A
:107A80006230C9EB020222F34F020136B6B2B6F5FC
:107A90000B7F34BF0E80A1F800A012990E8804EB72
:107AA000460707F5B5470FFA82F9B7F93A3002EB06
:107AB00063027A87C9EB030323F34F030136B6B29F
:107AC000B6F5DC7F94BF0E80A1F800A013990E8854
:107AD00004EB460707F5BC470FFA83F9B7F92C20EA
:107AE00003EB6203BB85C9EB020222F34F020136AE
:107AF000B6B2B6F5AA7F94BF0E80A1F800A0149983
:107B00000E8804EB460707F5C1470FFA82F9B7F96B
:107B1000563002EB6302A7F85620C9EB030323F3A8
:107B20004F030136B6B21BB2E02EC3EB031394BF72
:107B30000E80A1F800A05B0003F30F030A9A22F85D
:107B4000023F019B0A92159A93427FF450AE04992A
:107B5000002213461E4661F30F02079965F30F03D7
:107B6000354661F30F05099961F31F42089961F3E6
:107B70001F43059960F30F0661F31F46069945F20E
:107B8000546E45F2586C45F2506045F24C6761F313
:107B90001F45E251235044F80E60204644F80C5033
:107BA000169C0022214604F05FFF204604F02EFFC1
:107BB0001798199A90420AD01BB0BDE8F04F04F014
:107BC00025BF0146204604F069FF0028F4D11BB010
:107BD000BDE8F08F42F25003C0F20E0319931793E1
:107BE0009DE500BFF8B543F2FC330446C0F2010343
:107BF00003600021012004F118020B46607222612B
:107C00002172E16000E0226942F82310627A0133B8
:107C10009A42F8DC49F28853C2F200031A680AB9A2
:107C2000B9E01A465369002BFBD15461204642F259
:107C30005C130025C0F20E036561A580E580A57286
:107C4000294640F81C3B40F6B8020BF055F929468E
:107C500040F6481204F6D4000BF04EF904F59050AB
:107C6000294640F6FA121C300BF046F904F5E050B4
:107C7000294640F6982216300BF03EF904F51A50CA
:107C8000294640F61C322E300BF036F904F54750E9
:107C9000294640F6A6320A300BF02EF904F575504D
:107CA000294640F62A4230300BF026F904F593407D
:107CB000294640F6A2421A300BF01EF945F23C6309
:107CC00045F23E6045F2406745F2426145F244624A
:107CD000E55245F24666255245F2486345F24A6050
:107CE000E553655245F24C67A55245F24E6145F2A7
:107CF0005062A553E55245F25266255245F254634F
:107D000045F25660E553655245F25867A55245F273
:107D10005A6145F25C62A553E55245F25E66255212
:107D200045F2606341F69910E553655246F2676784
:107D3000A05246F6843204F5AC402946A75362307F
:107D4000E2524FF48B620BF0D7F804F5B5402946A8
:107D500040F272323A300BF0CFF804F5BC402946BD
:107D600040F2AA222C300BF0C7F804F5C140294696
:107D70004FF4E17256300BF0BFF846F2982046F20D
:107D80009A2146F29C2246F29E23255265522046B5
:107D9000A552E552F8BD1C6048E700BF10B5044687
:107DA00005F06EF8204610BD49F2406247F69D513D
:107DB00048F2A010C1F6FF72C0F20001C2F200004A
:107DC00008F050BD38B549F2406547F69D54C1F6FC
:107DD000FF75C0F2000448F2A8102A462146C2F2FC
:107DE000000008F03FFD48F2B0102A462146C2F2DA
:107DF0000000BDE8384008F035BD00BF49F24062E0
:107E000047F69D5148F2B810C1F6FF72C0F200016A
:107E1000C2F2000008F026BD49F2406247F69D51CB
:107E200048F2C010C1F6FF72C0F20001C2F20000B9
:107E300008F018BD49F2406247F69D5148F2C8105B
:107E4000C1F6FF72C0F20001C2F2000008F00ABDE4
:107E500049F2406247F69D5148F2D010C1F6FF72D8
:107E6000C0F20001C2F2000008F0FCBC2DE9F843AA
:107E70004FF00008064600F11805474641463046D7
:107E8000002F4FD004F00AFEF0B12C68B4F5803F0B
:107E900007F1040100F1040E07F5827C27D05EF89B
:107EA000042B34FB02F334FB12F903F30F0209F342
:107EB0000F03C2EA03430A6893FA12F341F8043B42
:107EC0008C45ECD804F0A2FD08F10108B8F1040FCC
:107ED00005F10405D2D1002F40D0304639460022AA
:107EE00004F0C2FD3846BDE8F84304F08FBD07F149
:107EF0000C0100F10C0451F8083C54F8082C93FADA
:107F000012F341F8083C54F8042C51F8043C93FA5D
:107F100012F38C4541F8043C04F1080401F1080116
:107F2000E9D8CFE704F0C6FD07460028CCD0286882
:107F3000B0F5803FC8D0391D07F582740B6830FB5F
:107F400003F230FB13F302F30F0203F30F03C2EA51
:107F5000034341F8043B8C42F0D8B5E7BDE8F88311
:107F600070B584692CB3B4F5803F06464FF000012C
:107F700025D004F09FFD054600B3011D00F5827079
:107F80000B6834FB03F234FB13F302F30F0203F329
:107F90000F03C2EA034341F8043B8842F0D830465D
:107FA0000022294604F060FD2846BDE8704004F038
:107FB0002DBD214604F072FD0028F6D170BD04F0FD
:107FC0006DFD04460028F9D030462146002204F019
:107FD0004BFD2046BDE8704004F018BD49F24062F8
:107FE00047F69D5148F2D810C1F6FF72C0F2000169
:107FF000C2F2000008F036BC49F2406247F69D51DB
:1080000048F2E010C1F6FF72C0F20001C2F20000B7
:1080100008F028BC49F2406247F69D5148F2E8104A
:10802000C1F6FF72C0F20001C2F2000008F01ABCF3
:1080300049F2406247F69D5148F2F010C1F6FF72D6
:10804000C0F20001C2F2000008F00CBC49F240622C
:1080500047F69D5148F2F810C1F6FF72C0F20001D8
:10806000C2F2000008F0FEBB48F24823C2F200034F
:108070002DE9F04F18681B79006848F21F0148F697
:108080000002C1F6FF72C4F20001904297B00B707B
:108090000FD248F22023C2F200031B78002B00F01D
:1080A00011814EF20823CEF200030121904619609F
:1080B00001E0A2F5806848F20023C2F2000348F212
:1080C000782248F2102148F27020C2F20002C2F277
:1080D0000001C2F2000014931B6815920C911090DD
:1080E0001268098800880F93089209910A90002B62
:1080F00000F0A281002A00F0078148F218263746D6
:1081000048F23C26304648F2442548F2582632468A
:10811000C2F200052E460E953D461746C2F20005F6
:10812000C2F2000748F21424C2F200042946119555
:1081300013970546384648F26427C2F200070D94AB
:10814000D4F800E0D0F800B0D7F800A00B970446B0
:108150004068009078680590B868326806921F46BB
:10816000099BA4680E684968019107EB430C089BC2
:10817000C2F200051F460A9B12952A4607EB4303ED
:108180000CF1020752680397023308F582672D68E5
:108190000493079708F11003069FDDF814800295F9
:1081A0009446D146224604460398049D30F9021FA6
:1081B000039035F9020F0591CEEB010E029906905E
:1081C000C71B781A01990495C6EB0E06711A009D1B
:1081D00002908B44CCEB00005D448144AC462A44C1
:1081E000C844DC4408EB040102EB0C04DC4404EB5F
:1081F0000C0A0BEB0C05C844121101EB080023F824
:10820000102CC84424110AEB050200EB080C23F8DB
:108210000C4CC844141123F8044C09110CEB08044D
:1082200023F80E1C211123F8021C4FEA2C1C00110C
:108230004FEA2A1A079923F806CC23F808AC23F84A
:108240000A0C103399420196DDF808C00095764675
:108250000297DDF814E0069FA6D1099BCDF81480A3
:1082600020461446624603F1400C0A9B069703F130
:1082700040080D9B0199C3F800E00E9B029D1F6012
:10828000119F3E60129E79600B997260139A35605F
:108290000B46009D5560059DC2F800B0C3F80090E4
:1082A0004D6094608860BCF17F0F1ED80C9BA3F8D2
:1082B00000C0B8F17F0F07D8109BA3F8008017B05B
:1082C000BDE8F08F9046F6E6109B089800241C80CD
:1082D00004F09CFB48F27423C2F2000315991A685B
:1082E0000A601C6017B0BDE8F08F0C9B0F9800244B
:1082F0001C8004F08BFB48F20C23C2F2000314999B
:108300001A680A601C60D4E7084648F21421C2F2D9
:108310000001174648F2242348F20422C2F2000367
:10832000C2F20002D1F800A00D9101920F99D3F88A
:108330000090029392E850001A4601EB400B5B68F4
:10834000926808F5826055460BF1020B08F11001A6
:108350000090CA46BBF902C021F80E7CC5EB0C08A0
:10836000C4EB0809C6EB0906B24453441A4453440B
:1083700002EB030E53440EEB0305534414114FEA72
:108380002E1EEA1821F80CEC28114FEA221E21F8C3
:10839000104C21F8080C21F804EC21F80A7C21F893
:1083A000067C21F8027C6546BBF904C04446C5EB57
:1083B0000C084E46C4EB0809C6EB0906B244534408
:1083C00008461A44534402EB030E1411534420F898
:1083D000104B0EEB03055344EA184FEA2E1E2911E9
:1083E00020F80CEC4FEA221E20F8081C20F80E7C26
:1083F00000F1100120F80A7C20F8067C20F8027CAD
:1084000020F804EC009888424E46444665460BF13D
:10841000040B9FD10999019801F1400C0A9980E859
:10842000500001F1400802980D99D1460D60C0F846
:1084300000904360826036E71046002A00F08D808D
:1084400048F24421C2F2000148F25022C2F2000276
:1084500048F230230E91D1F800A002921146C2F2E8
:108460000003126800924E68039301461A460A9868
:10847000D3F8009092685B680F9F01EB400B08F502
:1084800082600BF1020B08F110010190BBF902E0D0
:10849000009821F8107CCAEB0E0CC0EB0C08C6EB60
:1084A0000806B1444B441A444B44D5184B44EC18CD
:1084B00012114B4421F80E2C2D11E21821F80A5C00
:1084C0002411151121F8064C21F8025C21F80C7CCE
:1084D00021F8087C21F8047CF246BBF904E06046F0
:1084E000CAEB0E0C4646C0EB0C08C6EB0806B144BE
:1084F0004B441A444B44D51801F110004B44EC187E
:1085000012114B4420F8107C2D114A80E218CD80C6
:10851000241115118F800F818F814C8120F8025C0E
:108520000198CDF800C0203188424646F2460BF152
:10853000040BABD109990298644601F1400C0A99E9
:1085400080E8500001F1400803980E99C1F800E05E
:10855000C0F8009043608260A5E6114640464FF4A3
:10856000806217B0BDE8F04F0AF0C6BCF8B5002134
:10857000054604F093FAC8B172B648F20023C2F27D
:1085800000031968002938D048F20C22C2F2000218
:10859000166866B348F21024C2F2000400271E6079
:1085A0001060278062B6084604F030FA28460121A0
:1085B00004F074FAD0B172B648F27823C2F2000324
:1085C0001C6814B348F27422C2F2000215688DB11F
:1085D00048F27021C2F2000100261D6010600E807A
:1085E00062B62046BDE8F84004F010BAF8BD10604D
:1085F00062B6DBE7106062B6F8BD48F21022C2F244
:1086000000021860118062B6D0E748F27022C2F210
:1086100000021860148062B6F8BD00BF48F248201E
:10862000F8B5C2F20000012104F084FB48F23C03DB
:10863000C4F2040348F20024196848F27820C2F218
:108640000004C2F2000048F240020025C4F2040215
:1086500041F40041256005601960116841F0020194
:1086600011601A684FF4704142F00202C4F2020134
:108670001A600B68AB424BDB4FF47142C4F202024A
:108680004FF0804313601368002BFCDB4FF20413A0
:10869000C4F202034FF26007C4F202074FF2FE0E6B
:1086A0004FF20406C3F800E0C4F202064FF0000ED9
:1086B000C7F800E04FF2080401273760C4F2020453
:1086C0004FF20C0240F61376C4F2020267F31F4623
:1086D0004FF210054FF0E0674FF214004BF2080123
:1086E0004BF20C032760C4F20205C4F20200C4F28C
:1086F0000401C4F204034FF470644FF48037176030
:10870000C0F60F744FF4C0622E6004600A601A60F5
:1087100048F24824C2F200044BF204002368C4F279
:10872000040048F2004202214FF4C065C1F6FF7216
:1087300005601A6099802279996002F180424FF2B7
:10874000200102F50432C4F2020140F201164FF496
:1087500078451961DE8000214FF48060CFF6FF7507
:1087600006278D26D882DD609982D88399619F8300
:108770001170167004F07AFA48F2202348F21B01B7
:108780002279C2F20003C4F200014FF47046C4F231
:10879000020618700A70531131689B0003F16043A0
:1087A00048F6004402F11007012041F0124103F5A0
:1087B000614302F01F02C1F6FF7448F269050143EC
:1087C00000FA02F2C0F20005316044F827501A6046
:1087D000F8BD00BF49F2406247F69D5148F248207B
:1087E000C1F6FF72C0F20001C2F2000008F03AB810
:1087F00049F2406247F69D5148F27C20C1F6FF7273
:10880000C0F20001C2F2000008F02CB849F2406248
:1088100047F69D5148F28420C1F6FF72C0F2000174
:10882000C2F2000008F01EB849F2406247F69D51BE
:1088300048F28C20C1F6FF72C0F20001C2F20000C3
:1088400008F010B890F89D3090F89C20DBB293426D
:1088500015D001331F2B84BF00210B4610B598BFE4
:10886000D9B20633002250F8234080F89D102146EB
:1088700004F0FAF82046BDE8104004F0C7B870478D
:10888000D0F898300BB10120704710B5044604F0C1
:1088900065F8C4F89800003018BF012010BD00BF73
:1088A00010B50446D0F8980018B1043010BD07F098
:1088B000DFFB04F053F8C4F898000028F7D0043028
:1088C00010BD00BFD0F89810B1B190F89C200132D3
:1088D0001F2A10B4CABF0024D4B2224690F89D309B
:1088E0009342FBD00632002340F8221080F89C40CF
:1088F0005DF8044BC0F89830704700BF10B4047F97
:108900004160022CC26003D05DF8044B04F0D6BA7B
:1089100083685DF8044B1847F0B449F27063C1F600
:10892000FF7348F21F02996BC4F2000208791070BD
:10893000586B48F21C02C4F20002047914700979E1
:1089400011701A6B002A4FD05968C9688A4247D8FB
:108950000168CC8B240402F1FF3073D4C0F30E0005
:10896000C883C88B80B2C882996B0968C88B000421
:1089700060D4C2F30E00C883C88B002480B212F109
:10898000FF32C88218BF01221C63596B086849F284
:1089900070610568C1F6FF7101F12C04A54241D058
:1089A0000968CC6814F0804F0468056815BF2488F6
:1089B00024780235013544F0004405604C63996B1E
:1089C00048F21B03C4F200030979197049F270617F
:1089D000C1F6FF7112B14A6B12791A70F0BC704780
:1089E000521A1A630122D0E71968D86B0A6300246F
:1089F000CFF60F74CC620468CD68266848F6FD0493
:108A0000C0F2000425F080450327A642CD6083F81C
:108A10002D701FD1037F4260022BC2601ED0F0BCBC
:108A200004F04CBA086891F82C10C46841F0004179
:108A30004163C4E7CC8BC2F3080004F47E442043B6
:108A4000C88399E7CC8BC0F3080004F47E4420432C
:108A5000C88386E733461146F0BC18478368F0BCEC
:108A6000184700BF00207047704700BF48F29423AA
:108A7000C2F20003022242F22C21C0F20E015A601F
:108A80000022D9629A7083F8242083F8302083F87A
:108A90003220704741F23003C4F20B0341F224024A
:108AA0001968C4F20B0241F0800119601146136885
:108AB000DB07FCD40B689B07F9D441F20C03C4F22A
:108AC0000B0310B441F230041860C4F20B044FF0F1
:108AD000807200E0D2B121680123C0F20E030B4086
:108AE00041F23001013AC4F20B01002BF2D06AB11D
:108AF000012B0BD10B6813F0800F0B6813D043F0E0
:108B0000011303200B605DF8044B704741F2300203
:108B1000C4F20B020120136843F470230343136073
:108B20005DF8044B704713F4803305D00B6843F0B5
:108B300001130B600520F3E70A6842F001021846B2
:108B40000A60EDE72DE9F04341F2240241F23004DE
:108B5000C4F20B04C4F20B0241F2080841F20C0CFF
:108B60004FF0000E27461546C4F20B08C4F20B0C5A
:108B7000C0F6DB4E64264FF00009C8F80090236869
:108B800043F0800323601368D807FCD42B6899074F
:108B9000F9D4CCF800E04FF0807100E0E1B101239E
:108BA0002068C0F20E0303400139002BF6D099B1C2
:108BB000012B11D13B6813F0800F3B681BD043F0B1
:108BC00001133B600320013E10D013685B0710D5F2
:108BD0000028D2D0BDE8F083236843F4702343F02B
:108BE0000103013E23604FF00100EED1002808BFD1
:108BF0000520BDE8F08313F4803305D03B6843F0D3
:108C000001133B600520DEE7396841F00101184699
:108C10003960D8E7F8B548F2E823C2F200031A78C1
:108C20000AB10320F8BD5B78064603B9490241F258
:108C3000300541F2080241F20403C4F20B05C4F20C
:108C40000B02C4F20B034FF6FF774FF48134102070
:108C50002F60C1F23A1011601C60FFF71BFF002863
:108C6000E0D141F21003C4F20B0341F224044FF4AB
:108C700081511B68C4F20B04C4F20B0106F14002DF
:108C800006F510702B6841F2300643F0200713F40C
:108C9000E00F2F60C4F20B0646D123681E05FCD5F9
:108CA0000B6842F8403C0B6842F83C3C0B6842F8C9
:108CB000383C0B6842F8343C0B6842F8303C0B6897
:108CC00042F82C3C0B6842F8283C0B6842F8243CE4
:108CD0000B6842F8203C0B6842F81C3C0B6842F8D9
:108CE000183C0B6842F8143C0B6842F8103C0B68C7
:108CF00042F80C3C0B6842F8083C0B6842F8043C14
:108D000040328242BED1002041F23001C4F20B0158
:108D10000A6841F230039207C4F20B03F8D522220D
:108D2000C0F200121A60F8BD43F4E00343F02003E0
:108D30003360FFF707FF0120E6E700BFF8B548F210
:108D4000E823C2F200031A780AB10320F8BD5B7869
:108D5000074603B9490241F2300541F2080241F2E7
:108D60000403C4F20B05C4F20B02C4F20B034FF66A
:108D7000FF764FF4813400202E60C1F63A00116076
:108D80001C60FFF787FE0028E0D141F21003C4F217
:108D90000B034FF481541B6807F140012E46C4F2C7
:108DA0000B0407F510772A6841F23003D006C4F2AD
:108DB0000B03F8D5326812F4E00F4BD151F8402C78
:108DC000226051F83C2C226051F8382C226051F876
:108DD000342C226051F8302C226051F82C2C226067
:108DE00051F8282C226051F8242C226051F8202CB4
:108DF000226051F81C2C226051F8182C226051F886
:108E0000142C226051F8102C226051F80C2C226096
:108E100051F8082C226051F8042C2260326842F08C
:108E200010023260326812F4E00001F1400111D109
:108E3000B942B8D141F23001C4F20B010A6841F2E3
:108E400030039207C4F20B03F8D51222C0F20012CD
:108E50001A60F8BD1A6842F4E00242F010021A608B
:108E6000FFF770FE0120E5E7F0B549F23466C2F283
:108E7000000683B0336801934FF44044C4F2020407
:108E8000019F0546A4464FF0004EFF20236843F49F
:108E900080632360C4F82CE06063E36A002BFCDA93
:108EA000DCF83830DBB2FF2B06D033680093009B30
:108EB000DB1BB3F5967FE9D34FF44043C4F20203C2
:108EC0004FF00046186841F0400440F4806018609C
:108ED000DE6218465C63C36A002BFCDA4FF4404440
:108EE000C4F2020418204FF00047266822FA00F36B
:108EF00046F48066DBB22660E7626363E36A002BB8
:108F0000FCDA083810F1080FEFD1002932D0082917
:108F10000CBF8721FF214FF44043C4F202034FF0FE
:108F200000401A6842F480621A60D8621A46596397
:108F3000D36A002BFCDA4FF44042C4F20202164618
:108F400000274FF00044FF21136843F4806313604F
:108F5000D4625163D36A002BFCDAB36BD8B21B0620
:108F6000687001D403B0F0BD0137B7F5807FEBD155
:108F700003B0F0BD9521CEE72DE9F04148F2FC2584
:108F80008378C2F20005032B2B780F4682B004468B
:108F9000164618BF4F02002B6AD00021207805F03A
:108FA00027F93A4611212046FFF75EFF60BB49F2E0
:108FB0003460C2F200004FF4404103680093C4F2F1
:108FC0000201DDF800808C464FF0004EFF270B6851
:108FD00043F480630B60C1F82CE04F63CA6A4FF41E
:108FE0004043002AC4F20203F8DADCF83820D2B297
:108FF000FF2A627040F0918003680193019BC8EBE7
:109000000303B3F5967FE2D92078012105F0F0F84B
:109010002B7848F2FC22C2F200022BB349F27063B3
:10902000C1F6FF730020D97A10700A46E1B1CC076F
:1090300006D54FF46142CEF20002D86910600A46AC
:10904000880706D54EF20412CEF20002196A1160AA
:10905000DA7A510700F1EE80120705D54EF20C12B4
:10906000CEF200029B6A1360002002B0BDE8F081DE
:1090700049F27063C1F6FF7348F2F822C2F20002AF
:10908000D97A126801202870002933D072B6D97AB3
:1090900011F0010F08460DD04EF2801CCEF2000CEC
:1090A000D868DCF800E00EEA000EC3F81CE00846C1
:1090B000CCF800E089070BD54EF2841ECEF2000EEC
:1090C0001869DEF8001001401962CEF80010D87A55
:1090D00041070BD54EF2881ECEF2000E5869DEF81D
:1090E000001001405962CEF80010D87A010700F153
:1090F000A98062B61B68D96891423FF44EAF44F232
:109100000100C0F23F0000211860C8F23F0142F0A8
:109110008040DA60186119603FE7FE2A7FF474AF7F
:109120004FF480604FF6FF71C9F20001C8F21F00D2
:1091300018608E4659631A4659631846596306F5F6
:10914000FE77B11CD36A13F0F00FFBD0C0F834E007
:10915000836B01F8013C1B1201F8023C02318F4283
:10916000F0D106F5FD7106F50076B14210D24FF44C
:109170004042C4F202021746D36A13F0F00FFBD04C
:10918000BB6B181201F8020BB14201F8013CF3D39A
:109190004FF44043C4F202034FF480614FF6FF7274
:1091A000C8F21F01C9F20002196019465A63CA6A5F
:1091B0004FF4404312F0F00FC4F20203F7D02078CE
:1091C0009B6B012105F014F82B7848F2FC22C2F2C7
:1091D00000025BB349F27063C1F6FF730020D97AD5
:1091E00010700A4611B3C80706D54FF46142CEF29B
:1091F0000002D86910600A468F0706D54EF20412A5
:10920000CEF20002196A1160DA7A560706D54EF2DC
:109210000812CEF20002596A1160DA7A150705D5F4
:109220004EF20C12CEF200029B6A1360012002B0D3
:10923000BDE8F0814EF20812CEF20002596A1160C8
:10924000DA7A09E74EF28C1ECEF2000E9869DEF84B
:10925000001001409962CEF800104AE7F0B44FF4D4
:109260004046C4F202064FF00047336843F480637F
:1092700033603D46F762344671633346511C02F257
:109280000127E26A002AFCDA1A6811F8016C42F43C
:1092900080621A60DD625E63E26A002AFCDA1A68A4
:1092A00011F8026B42F48062B9421A60DD625E63BB
:1092B000E7D14FF44041C4F20201CA6A4FF440437F
:1092C000002AC4F20203F8DA1A684FF0004542F4AB
:1092D0008062FF241A601946DD625C63CA6A4FF43B
:1092E0004043002AC4F20203F8DA1A684FF000453E
:1092F00042F48062FF241A601946DD625C63CA6A28
:109300004FF44043002AC4F20203F8DA1A684FF01F
:10931000004542F48062FF241A601946DD625C63F6
:10932000CA6A4FF44043002AC4F20203F8DA9B6B86
:10933000DBB203F01F024370A2F10500B0FA80F027
:109340004009F0BC704700BF2DE9F041064682B0ED
:10935000002900F0AC8048F2FC258378C2F20005B9
:10936000032B2B780C46174618BF4C02002B3FD01E
:109370000021307804F03CFF224618213046FFF7E8
:1093800073FD002800F098803078012104F030FF50
:109390002B7848F2FC22C2F200022BB349F2706330
:1093A000C1F6FF730020D97A10700A46E1B1CC07EC
:1093B00006D54FF46142CEF20002D86910600A4629
:1093C000880706D54EF20412CEF20002196A116027
:1093D000DA7A510700F1A480120705D54EF20C127B
:1093E000CEF200029B6A1360002002B0BDE8F0815B
:1093F00049F27063C1F6FF7348F2F822C2F200022C
:10940000D97A12680120287000293DD072B6D87A26
:1094100010F0010F01460DD04EF2801CCEF2000C70
:10942000D968DCF800E00EEA010EC3F81CE0014642
:10943000CCF800E080070BD54EF2841ECEF2000E71
:109440001869DEF8001001401962CEF80010D97AD0
:1094500048070BD54EF2881ECEF2000E5869DEF892
:10946000001001405962CEF80010D97A09070AD5D8
:109470004EF28C1ECEF2000E9869DEF8001001400C
:109480009962CEF8001062B61B68D96891423FF429
:109490006FAF44F20100C0F23F0000211860C8F233
:1094A0003F0142F08040DA601861196060E748F2DD
:1094B000FC25C2F2000567E73A46FE213046FFF779
:1094C000CDFE00283FF460AF49F23461C2F20001E2
:1094D0004FF440420B680193C4F20202DDF80480AD
:1094E00094464FF0004EFF20136843F480631360EE
:1094F000C2F82CE05063D36A4FF44044002BC4F20E
:109500000204F8DADCF83870FFB2FF2F10D00B68D5
:109510000093009BC8EB0303B3F5167FE4D333E756
:109520004EF20812CEF20002596A1160DA7A53E75D
:1095300000220D213046FFF797FC00287FF424AF6E
:1095400023684FF0004243F4806323602146E262C7
:109550006763CA6A4FF44043002AC4F20203F8DA90
:109560009B6B13F0FF047FF40FAF3078012104F000
:109570003FFE2B7848F2FC22C2F2000253B349F2BC
:109580007063C1F6FF731470D97A0A4611B3C80725
:1095900006D54FF46142CEF20002D86910600A4647
:1095A0008F0706D54EF20412CEF20002196A11603E
:1095B000DA7A560706D54EF20812CEF20002596A40
:1095C0001160DA7A150705D54EF20C12CEF20002C0
:1095D0009B6A1360012008E748F2F823C2F20003F7
:1095E00042F20302C3F600021A6070472DE9F04F01
:1095F000837987B0012B0546029205D001232B7198
:10960000002007B0BDE8F08F42799007F6D55307E8
:109610000E4626D5EB68AF69BB4200F03781002FBC
:1096200000F058812A6A147C591E09347A1EE140E0
:1096300022FA04F4A14200F25181002B00F04E8185
:10964000641A05F1080806E0A968286A00F062FCBF
:10965000013C0028D2D04246002CF5D1EF603B46B9
:1096600000E0EB68029A002A00F09C8049F2B062A8
:1096700048F20C5148F20C3BC1F6FF72C2F20001F5
:10968000029F0192C2F2000B0391286A0279013A0B
:1096900002EA532212F0FF09C3F3080840F08B805E
:1096A000B8F1000F40F08780A968002940F0BE8023
:1096B000EB69002B00F0D080AB60C8F50074017C32
:1096C0004269A4B2023B8B404A44BC4203EB02090C
:1096D00073D9BCB2B8F1000F04D1A869EB6883421A
:1096E00080F086804846012100F030FA002885D0BD
:1096F00008EB0B03181983424ED008F10408321D01
:10970000D844934238BF464543EA060E2CBF012297
:109710000022591C1EF0030F02F00102C1EB000EE3
:1097200018BF00220EF101099C46002A6ED0B9F143
:10973000090F6BD9AEF10302920801324FEA820A97
:10974000A6F104084FF0000E00940EF1010E58F837
:10975000044F4CF8044B9645F7D3CA45009C06EBE2
:109760000A0C03EB0A0E13D016F8228003F82280AD
:109770000EF1010398420BD09CF801308EF80130B5
:109780000EF10203984203D09CF802308EF80230AA
:10979000C1F1010108440644EB683F1B2344EB6020
:1097A0007FF473AFAA699A4275D26A79AB6142F0CD
:1097B00080026A717BE0AB687FE7B4F5007F89D1F6
:1097C000019B1B6899452CD048F20833C2F2000374
:1097D000494618680378FE2B51D03246FFF7B4FD96
:1097E00000283FF40BAF06F500764FF40074D3E782
:1097F00000F05EF900283FF401AF039A0199137855
:10980000C1F8009043F00103137071E7013B721E31
:1098100000F1FF3C12F801EF03F801EF9C45F9D18C
:10982000B6E7019A4FF0FF331360CDE705AA00F0C9
:1098300071FB00283FF4E5AE286A059B90F82040B4
:109840004FF6F872C0F6FF724FF6F871102C08BF91
:109850000A469342FFF430AF05F10802012100F0FF
:10986000EDF900283FF4CAAEEB69002B30D16A79DC
:10987000AB68EB6162F07F026A71286A1DE73046CF
:10988000FFF75CFAB0FA80F04009A9E702990029D5
:109890007FF4ECAE0BE048F20033C2F200036A79C9
:1098A0001B6823B1029B13B142F080026A71110759
:1098B0000AD5AB79002B3FF4A1AE120611D400F00B
:1098C000F7F800283FF49AAE029807B0BDE8F08F91
:1098D000AB68D2E7AF60EF603B46C3E6EB69AB60D5
:1098E000AFE60121286900F031F900283FF486AE87
:1098F00048F20C332C7DC2F2000313EB44143FF406
:109900007DAEAB7948F20032012B9CBFAB69E361BD
:10991000C2F20002EB69126863831B0CA38232B1AE
:1099200004F1160104F118009047238B63826B79D0
:1099300003F07F036B71C2E700B583B002AB012275
:1099400003F8011D1946FFF751FE03B05DF804FB53
:109950002DE9F84F90F82030C66949F2B068102B15
:1099600005460F469146C1F6FF7822D006EBD11688
:10997000D8F800108E422FD148F20C54C2F20004E5
:1099800048F20C3307F07F07C2F2000343F8279038
:1099900023782A7E43F00103012A237054D9AA6850
:1099A00048F20433C2F20003114419600120BDE8FB
:1099B000F88F06EB1126D8F80010B1420CD148F20E
:1099C0000C54C2F2000448F20C33FFB2C2F200039E
:1099D000314623F81790DBE748F20C54C2F200043A
:1099E00048F2083A2378C2F2000AA3B9DAF8000074
:1099F0000378FE2B2BD048F20C32C2F20002314623
:109A0000FFF7BAFAE8B195F82030C8F80060102BDB
:109A1000D9D03146B4E7DAF800000378FE2B32D013
:109A200048F20C32C2F20002FFF78EFC48B148F255
:109A3000043BC2F2000BDBF8001099B9002323703D
:109A4000D4E70020BDE8F88F0120BDE8F88F48F288
:109A50000C30C2F200003146FFF7DCF8B0FA80F0BB
:109A60004009CFE7DAF800000378FE2B15D048F262
:109A70000C32C2F20002FFF767FC0028E1D000239D
:109A8000CBF80030DAE748F20C30C2F20000FFF702
:109A900055F9B0FA80F04009C8E748F20C30C2F23C
:109AA0000000FFF74BF9B0FA80F04009E5E700BF8E
:109AB00070B548F20C54C2F2000423780BB90120AF
:109AC00070BD48F20835C2F2000549F2B06328685B
:109AD0000278C1F6FF73FE2A196820D048F20C32D2
:109AE000C2F20002FFF730FCB8B148F20436C2F20D
:109AF0000006316819B900232370012070BD286861
:109B00000378FE2B15D048F20C32C2F20002FFF7A8
:109B10001BFC10B100233360EDE7002070BD48F25C
:109B20000C30C2F20000FFF709F9B0FA80F04009EA
:109B3000DAE748F20C30C2F20000FFF7FFF8B0FAA3
:109B400080F040090028E5D1E7E700BF2DE9F843A0
:109B500049F2B065C1F6FF7588462B68834218D07C
:109B600048F20C54C2F2000448F208372278064644
:109B7000C2F20007C2B938680378FE2B38D048F229
:109B80000C32C2F200023146FFF7F6F910B32E6034
:109B900003E048F20C54C2F20004217848EA0101C3
:109BA00021700120BDE8F88338680278FE2A14D0BD
:109BB00048F20C321946C2F20002FFF7C5FB48B169
:109BC00048F20439C2F20009D9F80010D9B90023CB
:109BD0002370D0E70020BDE8F88348F20C30194626
:109BE000C2F20000FFF7AAF8B0FA80F04009E6E7F9
:109BF00048F20C30C2F200003146FFF70BF8B0FA21
:109C000080F04009C2E738680378FE2B0BD048F299
:109C10000C32C2F20002FFF797FB0028DAD00023D3
:109C2000C9F80030D3E748F20C30C2F20000FFF769
:109C300085F8B0FA80F04009EFE700BF2DE9F04F5A
:109C4000136889B0002B00F0AF8003F1010A0023F4
:109C50000693C3685E1CB046002B44D05446A04512
:109C600038BF02240191059248F20C3348F20C529D
:109C700048F20831C2F20003C2F20002C2F200014F
:109C800038BFA246B4420546029203914FF0000746
:109C9000994628D895F82030EE6949F2B06B102B20
:109CA000C1F6FF7B2BD0DBF8001006EBD416B142D7
:109CB0002BD104F07F0348F20C3659F82330C2F25E
:109CC000000623F0704393B10134A246EE680137D9
:109CD000BE4208D9A04538BF022406F1010638BFAC
:109CE000A246B442D6D9002009B0BDE8F08F631C6B
:109CF0000199CAEB0302914273D01C46E6E7DBF8F8
:109D0000001006EB1426B14219D0029B1B78F3B960
:109D100048F20833C2F2000318680378FE2B38D0EB
:109D200048F20C32C2F200023146FFF725F9002852
:109D3000D9D095F82030CBF80060102BB9D1E3B220
:109D400048F20C3639F81330C2F20006BBE7039B29
:109D50001868027848F20833C2F20003FE2A04931E
:109D600000F0A68048F20C32C2F20002FFF7ECFAD3
:109D7000049B0028B7D048F20432C2F200020492D9
:109D80001168D1B90299186800220A700378FE2B75
:109D9000C6D148F20C30C2F200003146FEF73AFF5D
:109DA000B0FA80F04009C2E7A1F10103B3FA83F3EE
:109DB0005B09D0F800A006934BE7039A079310685D
:109DC0000278FE2A00F09B8048F20C32C2F20002B8
:109DD000FFF7BAFA079B002885D0049900220A6091
:109DE000D0E7012C7FF67FAFEB6801339C423FF652
:109DF0007AAF6FF0704221462846FFF7A9FD002890
:109E00003FF471AFA2455ED204F1FF38B8F1010F03
:109E10007FF669AFEB6801334345FFF464AF48F266
:109E2000043348F20C59C2F20003C2F20009019354
:109E30002EE007EBD817BA420AD000213846FFF7C8
:109E400085FE00283FF44FAF95F82020102A2AD035
:109E500008F07F0246F8224099F80020297E42F05F
:109E60000102012989F8002003D9AA68019B17443F
:109E70001F60C24527D008F1FF38B8F1010F3FF449
:109E800032AFEA680132904504F1FF343FF62BAF60
:109E900095F82020EF69102ADBF80020C9D107EBE4
:109EA0001827BA42C9D15FFA88F226F81240D3E7E0
:109EB00048F20C30C2F20000FEF740FFB0FA80F02A
:109EC0004009049B55E7059B196871B101297FF68C
:109ED0000AAFEB68013399423FF605AF5246284678
:109EE000FFF736FD00283FF4FEAE059BC3F800A047
:109EF000069B13B10AF101032B600120F4E648F23E
:109F00000C30C2F20000FEF719FFB0FA80F04009F1
:109F1000079B60E72DE9F84FC36801338B423DD3BF
:109F200090F82030C46949F2B068102B17460E46ED
:109F30000546C1F6FF7813D004EBD114D8F8001011
:109F40008C4213D148F20C3306F07F01C2F20003B9
:109F5000012053F8213023F070433B60BDE8F88FB7
:109F600004EB1124D8F80010A14220D048F20C5A7A
:109F7000C2F2000A48F208399AF80030C2F2000929
:109F800003BBD9F800000378FE2B3FD048F20C3217
:109F9000C2F200022146FEF7EFFF10B90020BDE833
:109FA000F88F95F82030C8F80040102BCAD148F23D
:109FB0000C33F1B2C2F20003012033F811303B60E0
:109FC000BDE8F88FD9F800000378FE2B12D048F2D4
:109FD0000C32C2F20002FFF7B7F90028DED048F2D7
:109FE000043BC2F2000BDBF80010E1B900238AF851
:109FF0000030C6E748F20C30C2F20000FEF79EFEC9
:10A00000B0FA80F040090028E9D1C7E748F20C30E7
:10A01000C2F200002146FEF7FDFDB0FA80F04009D3
:10A020000028BED1BAE7D9F800000378FE2B0BD088
:10A0300048F20C32C2F20002FFF786F90028ADD0D8
:10A040000023CBF80030D1E748F20C30C2F2000018
:10A05000FEF774FEB0FA80F04009EFE790F839207F
:10A0600090F83800101A704790F8383090F839207E
:10A070009A4205D95A1C034480F83820187E70474C
:10A080004FF0FF30704700BF90F8383090F839201B
:10A090009A4286BF1B18187E4FF0FF30704700BFF2
:10A0A000704700BF38B50546B0F85E0090B195F82E
:10A0B0005D301446C3F1210294420CD805F13B00F7
:10A0C0001844224603F01CFC95F85D30234485F8C3
:10A0D0005D30204638BD012014462871EEE700BFF0
:10A0E000B0F85E306BB190F85D30202B07D8C21805
:10A0F000013380F85D30012082F83B107047012366
:10A1000003710020704700BF38B549F22074C1F6D2
:10A11000FF742269D578EDB2E9062BD51023D370F0
:10A120006B0626D505F0040505F0FF03002D6CD065
:10A1300048F20D53C2F20003616E002249F220750D
:10A140001A7084F85D20C1F6FF75002974D0884725
:10A1500095F85D30002B6FD02369D0229A70236967
:10A1600094F83B201A712369012284F85C200222B2
:10A17000DA7038BD05F0400303F0FF00002BD1D1A9
:10A180009379DBB203F0600160295CD0937803F02F
:10A19000100303F0FF01D3B115F0010545D194F888
:10A1A0005C1094F85D0049F220738842C1F6FF7399
:10A1B00055D95818013190F83B0083F85C101071A4
:10A1C0002369D0229A7023690222DA70D1E784F8D9
:10A1D0006010937943F020039371236994F8390058
:10A1E000197949F220721F28C9B2C1F6FF72BED890
:10A1F00048F20D54C2F200042478002CB7D0141891
:10A200000130217682F83900B1E7226984F83930CB
:10A21000C0239370236948F20D52C2F200021979EB
:10A22000012111700222DA70A3E7C0239370236921
:10A230001A790222DA709CE70122002384F85D205B
:10A2400084F83B3088E703F0DF039371A36E23B1FA
:10A2500084F8380094F839009847226996E7157118
:10A26000AEE700BF38B549F28C74C1F6FF742269BD
:10A27000D578EDB2E9062BD51023D3706B0626D521
:10A2800005F0040505F0FF03002D6CD048F20D53D6
:10A29000C2F20003616E002249F28C751A7084F8D4
:10A2A0005D20C1F6FF75002974D0884795F85D30B0
:10A2B000002B6FD02369D0229A70236994F83B2039
:10A2C0001A712369012284F85C200222DA7038BDF9
:10A2D00005F0400303F0FF00002BD1D19379DBB2EE
:10A2E00003F0600160295CD0937803F0100303F061
:10A2F000FF01D3B115F0010545D194F85C1094F835
:10A300005D0049F28C738842C1F6FF7355D9581825
:10A31000013190F83B0083F85C1010712369D02262
:10A320009A7023690222DA70D1E784F86010937979
:10A3300043F020039371236994F83900197949F2A5
:10A340008C721F28C9B2C1F6FF72BED848F20D54F4
:10A35000C2F200042478002CB7D014180130217602
:10A3600082F83900B1E7226984F83930C02393704C
:10A37000236948F20D52C2F20002197901211170CD
:10A380000222DA70A3E7C023937023691A790222AC
:10A39000DA709CE70122002384F85D2084F83B30CA
:10A3A00088E703F0DF039371A36E23B184F83800CC
:10A3B00094F839009847226996E71571AEE700BF17
:10A3C00038B549F2B464C1F6FF742269D578EDB2AC
:10A3D000E9062BD51023D3706B0626D505F00405AE
:10A3E00005F0FF03002D6CD048F20D53C2F20003BC
:10A3F000616E002249F2B4651A7084F85D20C1F6DE
:10A40000FF75002974D0884795F85D30002B6FD018
:10A410002369D0229A70236994F83B201A7123692A
:10A42000012284F85C200222DA7038BD05F0400376
:10A4300003F0FF00002BD1D19379DBB203F0600170
:10A4400060295CD0937803F0100303F0FF01D3B1CF
:10A4500015F0010545D194F85C1094F85D0049F2BF
:10A46000B4638842C1F6FF7355D95818013190F88A
:10A470003B0083F85C1010712369D0229A70236925
:10A480000222DA70D1E784F86010937943F0200358
:10A490009371236994F83900197949F2B4621F283D
:10A4A000C9B2C1F6FF72BED848F20D54C2F2000420
:10A4B0002478002CB7D014180130217682F83900A6
:10A4C000B1E7226984F83930C0239370236948F2D8
:10A4D0000D52C2F200021979012111700222DA70C4
:10A4E000A3E7C023937023691A790222DA709CE7EC
:10A4F0000122002384F85D2084F83B3088E703F0D4
:10A50000DF039371A36E23B184F8380094F8390007
:10A510009847226996E71571AEE700BF704700BF04
:10A520004DF21802F8B5C4F204024FF21413C4F24B
:10A530000F034FF4807111601A684FF20411C4F2D6
:10A540000F0142F0400240241A600A200C6003F020
:10A55000D9FE4FF45842C4F200024FF48043116810
:10A56000C4F2060341F04051116019784FF4A04243
:10A57000C4F2060241F002011970117848F2040396
:10A58000C4F2040341F0800111701A6842F0020223
:10A590001A601A6847F20801C4F2040122F00102AD
:10A5A0001A600B6848F23002C4F2040243F400035C
:10A5B0000B60116843F20406C4F20A0642F2380541
:10A5C00042F2340442F2341042F2A003C4F20A030D
:10A5D00041F00E01C4F20A05C4F20A04C4F20A00F2
:10A5E0004FF0840E11604FF44047C6F800E04FF082
:10A5F0004042012643F241012A6027601A46066064
:10A6000019601368002BFCDA4FF40053C4F20A03FC
:10A6100000221A600A2003F075FE4FF48A53C4F238
:10A620000A031A46196841F00201196013689B0772
:10A63000FCD401F05DFB48F6FC73C2F2000301217B
:10A6400003F1800243F8041F93424FF00104F9D153
:10A6500049F28C004FF480720021C2F2000008F031
:10A660004BFC49F28802C2F2000241F2900C41F226
:10A67000A8110023C4F20A0CC4F20A01137041F2BB
:10A680004815032241F2541E41F24C1741F258166C
:10A690004FF48A50CCF80040C4F20A050A60C4F2B4
:10A6A0000A0EC4F20A00C4F20A07C4F20A0649F20A
:10A6B000000148F6153441F28412C4F20A02C2F2D3
:10A6C0000001C0F208042B60CEF800103B6033603C
:10A6D000046013684AF6893143F480531360C0F272
:10A6E00000015D2003F0C8FB4EF20812CEF200021A
:10A6F0000423C0F200334FF0005111602B602B682F
:10A7000043F012032B602B6843F440232B60F8BD09
:10A7100002699368F0B50C465906074603D41268DF
:10A7200093685B06FBD54023D4F808E0A360236858
:10A73000136063685360E368D360236913616369DE
:10A740005361A169916104F1340393E80300E36A62
:10A75000E669256BD36202F13403D6619762156313
:10A7600083E803001368E16BD163012B134603D028
:10A770001B6819680129FBD101211C602160136845
:10A780009C4235D01346002000E00B461968586201
:10A790000D681962AC420E461846F6D1002173626C
:10A7A000316297F8343013F0FD0F0CD049F2840376
:10A7B000C2F200031968A1B151620A621E60012051
:10A7C000C2F808E0F0BD48F21453C2F20003196861
:10A7D0000029F1D148F21850C2F200005162026023
:10A7E000ECE748F21050C2F2000051620260E5E767
:10A7F00016460023D2E700BF2DE9F047CC88B4F518
:10A80000804F02D90020BDE8F08799469046074660
:10A810008A4601F0BFFA05460028F3D001F0BAFAE3
:10A820000446002877D0BAF80630002B44D148F20D
:10A8300080132860C8F200032AF47F664FF4207169
:10A8400026F00F060122C0F208016A6006F580506A
:10A85000A96006F50051C5F80CA02861696106F5EC
:10A860004050002106F58046A8614FF4805EEE61FD
:10A870004FF4405062604FF40056A3603B68E160C3
:10A880004FF48041C4F810E0A3626661C4F82C80E4
:10A89000A061E161BAF806302363DAF8003063633F
:10A8A000DAF80430A363386822602946C4F83C9083
:10A8B000BDE8F047FFF72CBF01F06CFA78B3BAF8A7
:10A8C00006209AF900601204F34342F00042F60FAA
:10A8D000DB0F28F47F6142F0800221F00F0142EA91
:10A8E00006221B020126466001F5805E826001F5AA
:10A8F000005601F5405243F0802301F58041C0F835
:10A900000C8043F08003C0F810E046618261C161B1
:10A910002860046090E7284601F046FA72E728466E
:10A9200001F042FA204601F03FFA6BE72DE9F047CB
:10A930008146884617469A4601F02CFAA0B1BC0B16
:10A94000064614D0054603E0013C286005460ED0BB
:10A9500001F020FA0028F7D100E02646304634689E
:10A9600001F022FAAE42F8D10020BDE8F0870023C2
:10A970000124B7F5804FC0F82890C0F82C800763F9
:10A98000C0F83CA004604363836332464FF080010B
:10A9900027D999F835E05460C4F200014FF480459E
:10A9A000002028F47F6323F00F0341EA0E21916019
:10A9B00003F5805C03F5005E03F5405103F5804329
:10A9C000C2F80C80C2F810C0C2F814E09161D361E3
:10A9D00090B97F1BB7F5804FA84412684FF08001F3
:10A9E000D7D8390441F4004199F835E0546001208A
:10A9F00041F080013D46D4E731464846BDE8F04786
:10AA0000FFF786BE2DE9F04748F21856C2F200065D
:10AA1000D6F80090B9F1000F00F0AC8048F214585D
:10AA2000C2F200080025D9F808301F0664D4D9F80E
:10AA300008301C0479D4D9F82430D9F82070002BC0
:10AA400000F081801F62D9F80820002F5AD05006EC
:10AA50007B625BD54846D9F828A001F0A5F9002112
:10AA600008460C46D6F800C0D8F800E0B94601E028
:10AA70001746A2B1BB6A3A6A9A45F9D17B6A002BA4
:10AA800068D01A62002A62D05362002C5DD027621F
:10AA90003D624F4508BF91461746002AEAD100287B
:10AAA0006CD100296DD1DAF8103033F01F0308D0D3
:10AAB0009A68520632D5CAF81030CAF80C50CAF853
:10AAC00018500CB913E03C46A268130409D5DAF813
:10AAD0003C3042F0400220461BB1A36AA260DB6B0F
:10AAE0009847276A204601F05FF9002FEBD1B9F1B2
:10AAF000000F98D1BDE8F087D9F82090B9F1000F88
:10AB000091D1F7E75106C8F8003026D44846B94637
:10AB100001F04AF9B9F1000F85D1EBE79A681A689C
:10AB20001B6833F01F03C3D1CBE7D9F82830DB6BA8
:10AB3000002B80D048469847D9F82430D9F82070A7
:10AB4000002B7FF47FAF37607DE73C46A0E79E4651
:10AB500001219AE79446012094E7D9F828A04846B5
:10AB600001F022F9DAF8103033F01F0304D0B946AF
:10AB70003C469DE7BDE8F087BDE8F087C6F800C019
:10AB80008FE7C8F800E08EE741F24413C4F20A03ED
:10AB90002DE9F0411E681E60710321D548F2185757
:10ABA000C2F200073C68DCB148F21458C2F2000857
:10ABB000A3681A0600F1A680A3681B0400F1BA80FE
:10ABC000636A256A002B00F0C1801D62002D00F031
:10ABD000C1806B6220462C4601F0E6F8002CE7D1DC
:10ABE000370320D548F21057C2F200073C68D4B1B1
:10ABF00049F28408C2F20008A3681D067DD4A36848
:10AC0000180400F18480636A256A002B00F08B80B1
:10AC10001D62002D00F08B806B6220462C4601F0F7
:10AC2000C3F8002CE8D1B10700F19780720713D563
:10AC300041F28413C4F20A031C6844F02A021A6029
:10AC4000A3073BD4270707D449F28803C2F20003C5
:10AC50001A78022A00F09680F00120D4B1012BD599
:10AC600049F28003C2F20003196829B34A691A60E5
:10AC70007AB1136941F2880441F28C00C4F20A04EB
:10AC8000C4F20A00013B00264FF040459661236064
:10AC90000560C8680368BDE8F0419B68184749F241
:10ACA0008803C2F200031A78012A00F0A080032A68
:10ACB00000F08A80B101D3D4BDE8F08114F0010521
:10ACC00049F288034CD0C2F200031A78012AB9D89D
:10ACD0004FF4845141F284020124C4F20A0148F283
:10ACE000A060C4F20A0264F31F404FF040451C709C
:10ACF00026F0807608601560B0E7246A002C7FF4A7
:10AD00007BAF90E7246A002C7FF452AF68E7A36A18
:10AD1000DB6B002B3FF477AF20469847636A256AC8
:10AD2000002B7FF475AF3D60002D7FF475AFC8F840
:10AD3000003072E7A36ADB6B002B3FF441AF204683
:10AD40009847636A256A002B7FF43FAF3D60002D72
:10AD50007FF43FAFC8F800303CE7FFF753FE65E7EC
:10AD600042F2380249F28C17C2F20003C4F20A021E
:10AD7000C2F2000702211D703868116000F070FFF8
:10AD80003D605FE765077FF569AF4FF4845441F29A
:10AD90008400C4F20A040325C4F20A0041F28411BB
:10ADA0001D70C4F20A0142F210774FF0404527604F
:10ADB000056009688C0504D542F23401C4F20A0129
:10ADC0000A60F2017FF54AAF41F28412C4F20A022E
:10ADD0000421197010680022C0F38160114600F050
:10ADE000FBFB49F28C13C2F20003186036E741F214
:10ADF0008412C4F20A0202211970136843F48073AA
:10AE000013602BE72DE9F04F85B00290F2B1006B93
:10AE100042F6AB23007DC0F2010303FB01F30228DD
:10AE20004FEA134100F01E81012A1CD9032A40F287
:10AE30007681062A40F277810C2A40F27281182A24
:10AE400040F26B8120230393009310E0026B42F6E3
:10AE5000AB23127DC0F2010303FB01F3022A4FEA88
:10AE6000134100F0578101239AB203920093029A92
:10AE7000BDF80C0092F83530A2F84000002B40F0ED
:10AE8000EB8084314FEA51184FF0020E00231A462E
:10AE9000019349F28C0C4FF0FF3392469946C2F26F
:10AEA000000C019E1CF83610F5000CEB0500414427
:10AEB0008278C77804790EEB0200814274440EEB6D
:10AEC000070B00F29F80584540F29A80A04238BF9D
:10AED0002046984228BF18460CEB050338BFB14600
:10AEE00059785B79414438BF4FF0000A8B45734471
:10AEF000C0F0A880A34540F2A0809B45594638BFCA
:10AF00001946884298BF01460CEB050042448079FF
:10AF100084BFB1464FF0010A94427044C0F087806C
:10AF20009C427FD98442224638BF02466544914202
:10AF300098BF0A464744E97984BFB1464FF0020AF8
:10AF4000BB4271446AD3834263D98B4238BF0B46FC
:10AF50009A4298BF1346009A88BFB146164488BFEC
:10AF60004FF0030A1F2E9DD91146019A01329142DA
:10AF7000019296D1BB2B6BD8029ABDF80C00A2F8B7
:10AF800044005FFA88F85FFA8EFE1FFA89F1B9F182
:10AF90001F0F82F84A8082F84BE0A2F848A0A2F87E
:10AFA00046101DD800980AEBC9039C1C1CF803200E
:10AFB00042440CF803201CF8042072440CF80420CE
:10AFC000DC1C04331CF8042072440CF804201CF828
:10AFD000032081447244B9F11F0F0CF80320E2D919
:10AFE000029C01201C2300FA0AF203FA0AFAA4F8D0
:10AFF000421084F8362084F837A005B0BDE8F08F01
:10B00000584663E75945FBD9A14238BF2146084657
:10B010005FE78842034638BF0B4699E7B842F8D24B
:10B020003B4692E783421A4638BF02467EE7934288
:10B03000F8D2824238BF024678E79C42214638BFA8
:10B0400019465EE78C42F8D2994238BF194658E754
:10B05000002005B0BDE8F08F66314FEA511E4FF079
:10B06000020813E70F2A6FD920234FF48070029A49
:10B0700057314FF0FF3749F28C0C4C09A2F84030A1
:10B080003E46C2F2000C00252B4600211CF803208E
:10B0900022449142034438BF1146FF2BF6D9B942EE
:10B0A00038BF2E4605F1010538BF0F46A842EBD147
:10B0B000BB2FCDD8029AE4B2FF2E134682F84A4045
:10B0C000A2F84400A2F8466098BF334607D81CF89F
:10B0D000032022440CF803200344FF2BF7D9012856
:10B0E0002CD0022821D0042895BF06F0030206F0D8
:10B0F0000702112301239340029A82F83630114649
:10B10000F60800230120A1F8426081F8373005B02D
:10B11000BDE8F08F01200346A9E71023A4E602232F
:10B12000A2E60823A0E604239EE606F001025523CA
:10B130009340029A82F836301146E1E7029AFF23E3
:10B1400082F836301146DBE7013A012303FA02F0B8
:10B15000B0F5807F88DCC20889D093B287E700BF52
:10B160002DE9F04706460D4617469A4600F000FEC8
:10B170000446002855D000F00DFE8046002800F05F
:10B18000D780602200214FF04009204607F0B4FE2E
:10B190004A460021404607F0AFFE0123032DC8F8C0
:10B1A0000030C8F80890C4F810802663636184F802
:10B1B00035A084F834504AD03FB172680AB968E0CB
:10B1C0001A46936B002BFBD194636DBB96F814E089
:10B1D000BEF1010F8CBF00210121C8064FF480434E
:10B1E000717D94F8362041F0704141EA0721089FB3
:10B1F00041EA074101430B4343EA0E336360F07DAC
:10B20000B37D94F8371042F0804242EAC05242EADD
:10B21000034343EA0123A36035F0020309D0032D61
:10B220003BD02046BDE8F0870023184696F814E08E
:10B23000D6E741F25812C4F20A021368B3B11A6891
:10B24000226044F002021A602046BDE8F087099AA5
:10B2500008992046FFF7D6FD814600286ED0002FC2
:10B26000ABD196F814E03B463846B9E761684FF435
:10B270008A5344F00200C4F20A0341F400416160C1
:10B28000206014601A6842F0200220461A60BDE86F
:10B29000F0877460002D99D0C6E7B4F84200B4F886
:10B2A00040101F28BDD849F20006C2F2000644F043
:10B2B000020756F82020D5074FEA800E28D402F066
:10B2C0000605022D22F01F0308D128E09C4216D06B
:10B2D0001A68D20708D41B6823F01F03B3F8402074
:10B2E0009142F3D99C420AD01A6832F01F0204D16D
:10B2F0001AE0126832F01F0216D09442F9D10844C5
:10B300001F288ED856F82020D5074FEA800ED6D5B4
:10B3100008441F28226046F80E70F3D981E7B3F87D
:10B320004050A942D2D9F3E71A6822601F60E6E7CD
:10B33000204600F027FD4046BDE8F087404600F07B
:10B3400033FD204600F01EFD4846BDE8F08700BFF3
:10B35000F8B590F8343013F0FD0F044600F09080FB
:10B3600048F6FC70C2F2000000F1800550F8041F9E
:10B37000CA070CD421F01F018C4203D17AE0944219
:10B3800072D011460B6823F01F02DB07F7D5854208
:10B39000ECD1236B1B7D022B00F0C380B4F8461068
:10B3A000B4F84460B4F8487094F84AE094F84B500C
:10B3B0001F291ED849F28C03C2F2000307EBC10219
:10B3C00002F1020C985CCEEB0000985413F80C00CC
:10B3D000401B03F80C0002F1030C043213F80C00BC
:10B3E000401B03F80C00985C3144401B1F29985403
:10B3F000E4D948F21056C2F20006306820B349F290
:10B400008407C2F2000701E02846EDB1836A056AAD
:10B410009C42F9D1436A002B00F099801D62002DF7
:10B4200000F093806B62236933F01F0205D08342E2
:10B43000EAD01B6833F01F02F9D18342E4D000F058
:10B44000B3FC2846002DE1D1206930F01F0306D05F
:10B45000056800F0A9FC35F01F032846F8D1204606
:10B46000BDE8F84000F08EBC23680B6085427FF495
:10B470007DAF8EE72368036085427FF477AF88E76E
:10B48000026822F01F02904201D166E01A4613685A
:10B4900023F01F039C42F9D163681D0403D5536850
:10B4A00043F4004353604FF48A5321681160C4F29F
:10B4B0000A0341F244111A6842F040021A60C4F2D1
:10B4C0000A010A6841F244139006C4F20A03F8D54F
:10B4D00020221A6048F21856C2F20006306800288E
:10B4E000B2D048F21457C2F2000702E02846002DFD
:10B4F000AAD0836A056A9C42F8D1436A5BB31D6295
:10B500003DB36B62236933F01F0205D08342EDD057
:10B510001B6833F01F02F9D19842E7D000F044FCD9
:10B52000E4E7B4F84620B4F8440094F84A50FF2AFF
:10B530003FF65FAF49F28C03C2F20003995C491BEE
:10B5400099540244FF2AF9D953E73B606BE7356011
:10B5500065E73B60D6E73560D2E74FF48A53C4F223
:10B560000A0341F24412196821F020011960C4F263
:10B570000A02136813F40043FBD141F25812C4F2DB
:10B580000A021360A6E700BF38B549F2B833C2F229
:10B5900000031D6865B1EC6834B123682046DB68A0
:10B5A00098476468002CF8D1AD68002DF3D138BD00
:10B5B00038BD00BF49F2A433C2F2000300211A686B
:10B5C000816041600AB905E01A465368002BFBD13F
:10B5D00050607047186070472DE9F04182B0804696
:10B5E0000F46164600F0B2FB044600284BD024223A
:10B5F000002107F081FC00250820E67584F81480FE
:10B60000A77565752B46009001952A462946204668
:10B61000FFF7A6FD0646206000283AD000F0CCFBDC
:10B62000D4F800E020614BF2957249F29211C0F219
:10B630000002C2F2000149F2B0360120C2F2000657
:10B64000CEF83C204FF4D06749F2A0122B46087088
:10B650008EF83500C2F20002C0F200174FF4002548
:10B660003146204637607560FFF7C6F849F2B833B7
:10B67000C2F200031A680AB908E01A469368002B60
:10B68000FBD19460204602B0BDE8F0811C602046EA
:10B69000F9E7204600F064FB3046F4E72DE9F04F6F
:10B6A00049F2A438C2F2000849F29015D8F80040D7
:10B6B00085B08146C2F20005002614B916E0646820
:10B6C000A4B1A268002AFAD129882068093900911A
:10B6D00049F2A9130768C2F2000349462046B84759
:10B6E000002847D126466468002CEAD12F8849F209
:10B6F000A014C2F2000427440934A74203D81AE078
:10B700003444A74217D963782678042BF8D1092E40
:10B71000F6D1D8F80050002DF2D04FF0000AC4EB5B
:10B72000070B0396AB684BB16D68002DFAD1039EF1
:10B730003444A742E7D805B0BDE8F08F2B68CDF8B8
:10B7400000B01B6801221E46494623462846B047E2
:10B7500070B16B68BAF1000F16D0CAF80430D9F88E
:10B760000C306B60AA46C9F80C50C5F80890DBE7AE
:10B77000AA46D9E7636856B173600023C4F80890FD
:10B780006360C9F80C40D6E7C8F80030E7E7C8F8AE
:10B790000030F2E72DE9F041C46B34B12368014673
:10B7A0005B682046BDE8F0411847836A1D6B2B7E1D
:10B7B000072B00F0DD8147D8032B00F009815AD810
:10B7C000012B00F0788100F2E2802C6849F2A01190
:10B7D0006368C2F2000149F2A03E49F2B832C97969
:10B7E00023F0FF63C2F2000EC2F2000223F4E02352
:10B7F00043EA01439EF8000011686360013080282D
:10B8000028BF012051B14B7D9842F7D00B4602E092
:10B810005A7D8242F2D09B68002BF9D149F2B034B4
:10B8200000270604C2F200043B468EF8000046F4EE
:10B83000A06621463A46284684E8C000FEF7DCFFB1
:10B8400001232B76BDE8F0810B2B26D03ED90D2BA2
:10B8500000F05281C0F0D5800E2B40F0DB812846ED
:10B86000FFF71CFF49F29213C2F200030F222A765F
:10B870001C70BDE8F081052B00F05A8100F2ED80CC
:10B8800049F2A013C2F200031A79032A03D95A79A4
:10B89000032A00F0C8810B232B7649F2B034C2F2A0
:10B8A00000044FF4D06649F2A0120023C0F2002633
:10B8B0004FF410272146C2F20002284684E8C00057
:10B8C000FEF79AFF0C232B76BDE8F081092B00F0E0
:10B8D000A3812CD82E692EB1C16A19B14B78032BE4
:10B8E00000F0718149F2A013C2F200039A78002A95
:10B8F000D1D009222A769C786F8C240449F2B03684
:10B90000C2F2000649F2A41244F040740023C2F2CD
:10B91000000244F4D06447F0FE773146284686E8BA
:10B920009000FEF769FF0A232B76BDE8F0812C69B1
:10B93000002CB0D0C06A0028ADD04378032BAAD128
:10B94000A3780133DBB2A370077803EB5702312AE7
:10B9500003DDC3F132077F00FFB2022F40F27A818C
:10B96000302B98BF022102D974E1312B0BD0E218A1
:10B97000023101338678D670C9B2DAB28F421346EB
:10B9800000F10200F1D8A3180022DA7083E749F22F
:10B99000A013C2F200031A796A765A79AA769A79C4
:10B9A000EA76597A1A7A42EA0122EA83D97A9A7AAD
:10B9B00042EA01222A849A7BD87B197C1A700243BE
:10B9C0005870997051EA02033FF465AF03232B7658
:10B9D00049F2B034C2F200044FF4D060C0F200303B
:10B9E00049F2A412002320604FF0FE762146C2F2F5
:10B9F000000228466660FEF7FFFE04232B76BDE8B2
:10BA0000F08149F2A013C2F20003DA789B7843EA8E
:10BA10000223B3F5007F40F2B08049F29013C2F2E6
:10BA200000034FF400721A804FF0007749F2B034EF
:10BA3000C2F200044FF4D06649F2A0120023C0F213
:10BA400000262146C2F20002284684E8C000FEF724
:10BA5000D3FE0D232B76BDE8F0812F692FB1C16A8B
:10BA600019B14B78032B00F08F8049F2A013C2F27A
:10BA700000035A78002A3FF439AF07222A765C780F
:10BA80006F8C240449F2B036C2F2000649F2A412C7
:10BA900044F040740023C2F2000244F4D06447F042
:10BAA000FE773146284686E89000FEF7A5FE08237B
:10BAB0002B76BDE8F08149F2B036C2F20006286864
:10BAC00073886B75416821F07F0119434FF4D0678B
:10BAD00049F2A01241602346C0F200174FF49014BF
:10BAE0003146C2F20002284637607460FEF784FED9
:10BAF00002232B76BDE8F08149F2A013C2F20003C5
:10BB000049F2B036DA792A771A7A6A775F79C2F21F
:10BB100000063F04234647F4106731462246284674
:10BB200037607460FEF768FE0E232B76BDE8F08167
:10BB300049F2A013C2F200031C786F8C240449F26E
:10BB4000B036C2F2000649F2A41244F04074002359
:10BB5000C2F2000244F4D06447F0FE773146284632
:10BB600086E89000FEF748FE06232B76BDE8F081BC
:10BB700049F2A013C2F2000381E749F29012C2F227
:10BB800000021F04138051E700223A700E78632EE2
:10BB900047D8022E62D9B81C0023022201E0312BC3
:10BBA0000AD00232D2B28C7800F8014F0133B2428F
:10BBB000DBB201F10201F2D31A463A440021D170FE
:10BBC0007B70BB7051E773780133DBB273700F7811
:10BBD00003EB5702312A03DDC3F132077F00FFB2C6
:10BBE000022F39D9302B98BF022202D934E0312BF1
:10BBF0000BD0F018023201338C78C470D2B2D8B2B4
:10BC00009742034601F10201F1D833180022DA709D
:10BC1000B07067E6BDE8F08149F2A013C2F20003FC
:10BC200069E66426B7E7D9799A7942EA01226A84FB
:10BC30001A7812B105222A767EE7597849F2A012C5
:10BC4000C2F2000200297FF418AF9278002A3FF474
:10BC500022AE4EE61A4696E61846D6E71346ACE7FD
:10BC600000283AD0F8B5C468064684B149F2A43534
:10BC7000C2F200050027236820461B6998476368C5
:10BC80002A68A76062602C601C46002BF3D17068A4
:10BC900028B1846BFFF75CFB2046002CF9D130689B
:10BCA000FFF756FB49F2B832C2F200021368CBB17B
:10BCB0009E4203D112E0A64204D023469C68002C89
:10BCC000F9D1F8BDA2689A60206908B100F082F845
:10BCD0002046BDE8F84000F043B87047B3681360F1
:10BCE0003446F1E7F8BD00BF704700BF704700BFA2
:10BCF00049F28043C2F20003194603F14002F0B456
:10BD00001E4641F8802F49F28055C2F2000549F2E3
:10BD1000E03049F2845246F8C01FC2F20000C2F27D
:10BD2000000249F2BC3449F200412F681F60C2F2A0
:10BD30000004C2F2000107681B6413682E602760CC
:10BD400004600B601160F0BC704700BF49F2E03343
:10BD5000C2F20003186808B102681A60704700BF99
:10BD600049F2E033C2F200031A68026018607047BB
:10BD700049F28453C2F20003186808B102681A60DD
:10BD8000704700BF49F28453C2F200031A68026090
:10BD90001860704749F28053C2F20003186808B176
:10BDA00002681A60704700BF49F28053C2F2000374
:10BDB0001A6802601860704749F26043C2F20003DB
:10BDC000186830B102681A600023037043708370F2
:10BDD000C370704749F26043C2F200031A68026000
:10BDE0001860704701EB410100EB4111884210D20D
:10BDF00010B449F28454C2F20004226800E01846EC
:10BE0000034643F8602B99420246F8D820605DF85B
:10BE1000044B704700EB8111884215D230B449F2CF
:10BE20008055C2F2000502462C6800E01A4613460F
:10BE300043F8404B99421446F8D8C343194421F0C3
:10BE40003F010844286030BC704700BF352303FB26
:10BE50000101884210D210B449F26044C2F20004D9
:10BE6000226800E01846034643F8352B9942024603
:10BE7000F8D820605DF8044B704700BFC36B5BB11E
:10BE8000C26A03F154018A4207D003F194018A4245
:10BE900004BF002283F81F227047002283F81E226D
:10BEA000704700BF0023C36003617047012A01D0BF
:10BEB000002070471A78092AFAD15A78042AF7D153
:10BEC0005A79012AF4D19A79032AF1D1F0B583B0D5
:10BED00003F10907089A9A180D46BA424FF000017B
:10BEE000044680F8201280F8211255D9587A032888
:10BEF00021D939188A421ED39B7A042B4CD00B2BA4
:10BF000013D149E0052B19D0252B14D18A4261D9D0
:10BF1000087803280FD90E18B2420CD34B78042BA3
:10BF200058D00B2B0F4655D03146242BEAD1BB7885
:10BF3000013B032BEAD9002003B0F0BD0628FAD953
:10BF4000FB78023B012BF6D8BB7813F0F00013D03E
:10BF50008028F0D194F820020028D7D103F00F03F5
:10BF600084F82032FB7884F8223278793B7943EAEE
:10BF70000023A4F8D430C9E794F821020028C5D1E1
:10BF800084F82132FB7884F8233278793B7943EACC
:10BF90000023A4F8D630B9E70023E36094F8212207
:10BFA0001AB1B4F8D630402B3DD900232361E268A2
:10BFB0000023A4F81A32A4F81C3284F8253284F83D
:10BFC000263284F8273284F82832A4F84C332AB376
:10BFD0000120B1E794F82022002ADDD0B4F8D43053
:10BFE000402BD9D894F822120093002301932846BD
:10BFF0000123FFF7B5F8E0600028CFD04CF25502DE
:10C00000C0F20002C2632346B4F8D42004F1140144
:10C01000FEF78CFC012384F81832BFE72069C01AB0
:10C0200018BF012088E7002694F8231200932846C1
:10C0300001963346FFF794F820610028B7D04BF6FD
:10C040007D63C0F20003C36384F81E6284F81F623C
:10C05000ADE700BF70B5C46B64B38268016BB4F820
:10C060001A32B4F81C62C2F30E428A1A920811D036
:10C07000043204EB820004F1100252F8041F39B1BB
:10C080000133502B28BF002303F1360544F8251057
:10C090008242F2D19E428CBF06F1FF364F36B4F891
:10C0A000D420A4F81A32F31AB3EB920F03D2002370
:10C0B00084F8183270BD234604F11401E068FEF7DD
:10C0C00035FC012384F8183270BD00BF10B5032180
:10C0D000044600F56870FFF785FE04F598600721B7
:10C0E000FFF798FE04F5D0600121FFF7AFFE0023B3
:10C0F000C4F85033C4F85433C4F85833C4F85C332C
:10C10000C4F86033C4F86433C4F86833C4F86C33DB
:10C11000C4F87033C4F87433C4F87833C4F87C338B
:10C12000C4F88033C4F88433C4F88833C4F88C333B
:10C13000C4F89033C4F89433C4F89833C4F89C33EB
:10C14000A4F81A32A4F81C32E36023612046BDE84B
:10C150001040FFF72FBA00BF03460069002837D010
:10C1600070B4B3F8D620920893F81E5293F81F4289
:10C17000EDB2AA42E4B215D9BCB1A24215D9651CF0
:10C1800003EB8404EEB2AA42C4F8941083F81F6251
:10C1900002D9D1B283F81F12920003F1940170BC4E
:10C1A000FEF7C4BBA242DFD9E9E76C1C03EB8505AF
:10C1B000A2426965E6B288BFD1B283F81E6288BF29
:10C1C00083F81E12920003F1540170BCFEF7AEBB5F
:10C1D000704700BF2DE9F84F1B015FFA83F9002A71
:10C1E0007ED0012A00F093804B780D4609781B061B
:10C1F00043EA014343F4704149F00407961E394372
:10C200000446FFF7A9FF022E05F102085BD90535A8
:10C2100004F1940B04F1540A1BE0CBB39A4237D9D2
:10C2200003F1010E04EB83035FFA8EFC7245C3F841
:10C23000941084F81FC202D9D3B284F81F3292003E
:10C2400023465946FEF772FB033E022E05F1030515
:10C2500039D915F8023C15F8032C15F8011C206992
:10C260001B0443EA02233B4343EA0161A84600283A
:10C27000EAD0B4F8D620920894F81EE294F81F325F
:10C280005FFA8EFE7245DBB2C7D89A42F4D9C7E78F
:10C290000EF101039A4204EB8E0E5FFA83FC88BF15
:10C2A000D3B2CEF854104FEA820284F81EC251462F
:10C2B00088BF84F81E32033E2346FEF737FB022E6A
:10C2C00005F10305C5D8022E2ED0012E12D049F457
:10C2D0007741204641F00501BDE8F84FFFF73CBF2C
:10C2E0004FF20601C0F2F70149EA0101BDE8F84F3B
:10C2F000FFF732BF98F8001049F4770949F00609B2
:10C3000049EA01212046BDE8F84FFFF725BF0B7829
:10C310004FF2070149EA0349CFF2007149EA0101EE
:10C32000BDE8F84FFFF718BF98F8003098F80110F3
:10C3300049F0774949F0070949EA0329204649EAC3
:10C340000141BDE8F84FFFF707BF00BF2DE9F843F3
:10C35000B0F81A22B0F81C329A423ED001334F2B6B
:10C3600084BF0026334604460F4690F8180203F1B6
:10C37000360198BF9EB254F82150A4F81C6260B9EF
:10C38000E16851B193428CBFD243C2F14F021344D2
:10C39000B4F8D420B3EB920F3DD205F00F064FEA6C
:10C3A0001528A6F1080208F00F01C5F30313062AA9
:10C3B00001F1010984F8243212D9B31E012B5FFA6E
:10C3C00088F77AD9052E74D0042E42D0731F022B21
:10C3D00040F28D800F2E00F01F810020BDE8F88311
:10C3E0000FB1B945F9D1082EC5F303331ED0092E7C
:10C3F00000F0CA800A2E40F0FF800A2BEDD1D4F85D
:10C400005833A02284F826225FFA89F9CBB92F0E7F
:10C41000C5F30746E7E072B62346B4F8D420E068D7
:10C4200004F11401FEF782FA62B6B6E7082BD4D104
:10C43000D4F85033802284F826225FFA89F9002B41
:10C44000E5D0C5F307462F0E48463A463146984791
:10C45000C9E0D4F86C83B8F1000F00F0C681B4F8DD
:10C460004C13B1F5917F80F016814B1C621899B284
:10C47000B1F5917FA4F84C13C5F3074682F82972F1
:10C4800000F06D814B1C621899B2B1F5917FA4F850
:10C490004C134FEA156582F8296200F059814B1C54
:10C4A0009BB22144A4F84C3381F829520020BDE806
:10C4B000F883F02F1BD9F72F19D0F82F00F08381C4
:10C4C0007AD9FC2F00F0798100F2C380FA2F00F0B6
:10C4D0008681FB2F81D1D4F88C33002B7BD1D4F80B
:10C4E0009C330BB138469847C5F3074676E0D4F83D
:10C4F0006C33002B00F05081B4F84C13B1F5917FF0
:10C5000080F01F814B1C9BB22144A4F84C3381F86E
:10C510002982052E00F00B81D4F86C73002F00F0F7
:10C52000E980B3F5917F80F08381591C89B223445F
:10C530002A0C072EA4F84C1383F8292240F02881F6
:10C54000002F00F0CB81B1F5917F00F07E814B1C74
:10C550009BB2DEB2180A21442D0E81F829521946E9
:10C560000022F02384F8276284F82802A4F84C23E0
:10C5700084F82632002F00F0CF8004F22920012217
:10C58000B8470120BDE8F883092B7FF426AF2F0EB2
:10C5900000F03F81D4F85433902284F826225FFAC9
:10C5A00089F9002B00F06381C5F30746FFB23A46D4
:10C5B00031464846984716E0F22F00F08C8040F252
:10C5C000D980F32F00F0F280F62F7FF406AFD4F875
:10C5D0008033002B88D09847C5F3074684F826821D
:10C5E0005FFA89F92F0E84F8259284F8276284F87F
:10C5F00028720120BDE8F8830B2E35D10B2B7FF478
:10C60000ECAED4F85C33B02284F826225FFA89F9C4
:10C61000002B7FF416AFFAE6F72F3FF64EAFF02F60
:10C62000B4F84C1302D000293FF4D7AED4F86C33E1
:10C63000002B00F02281B1F5917F80F011814B1C1D
:10C640009BB22144A4F84C3381F829820020BDE834
:10C65000F883FE2F00F0BD80FF2F7FF4BEAED4F82C
:10C660009833002BB7D13AE70C2E40F00B810C2BFE
:10C670007FF4B3AED4F86033C02284F826225FFA88
:10C6800089F9002B3FF4C3AEC5F30746484631464F
:10C690002F0E9847A7E7002204F22920C047D4F8BC
:10C6A0006C8384F829720121A4F84C13C5F3074662
:10C6B000B8F1000F7FF4E6AE0B46591C89B2234453
:10C6C000B1F5917FA4F84C134FEA156583F8296200
:10C6D0003FF483AEE3E6D4F87823002A3FF404AFB6
:10C6E0002E0C6B0C06F07F0003F47E531843F6B259
:10C6F000904773E7B3F5917FFFF417AF072E46D14C
:10C7000019120020F02284F8281284F827321946E2
:10C71000A4F84C0384F82622D4F87033002B00F0E0
:10C72000918004F2292098470120BDE8F883F72F73
:10C730007FF453AED4F86C73DEB2C3F3072019460E
:10C740000EE7002204F22920984700210123DBE6AE
:10C75000002204F22920C04700210123A1E6002283
:10C7600004F22920C047012184F829622D0EA4F883
:10C770004C1394E6F12F7FF430AED4F87433C5F344
:10C780000746002B3FF42AAF3046984726E7194664
:10C79000CEB2C1F30720E3E6B4F84C33B3F5917F92
:10C7A000BFF4B7AE5A1C194693B2ADE6D4F87C3349
:10C7B000C5F30746002BE7D110E7D4F89033002BE0
:10C7C0007FF409AF8BE6D4F88433002B7FF403AFFA
:10C7D00085E6D4F89433002B7FF4FDAE7FE6D4F8E1
:10C7E0008833002B7FF4F7AE79E6B4F84C23B2F52A
:10C7F000917FBFF4F2AD531C9BB22244B3F5917FFD
:10C80000A4F84C33C5F3074682F829723FF4E5AD2E
:10C8100053E7D4F85033802284F826225FFA89F94E
:10C82000C5F307463BB3314648463A469847DAE6F1
:10C830001946002204F22920B847D4F86C7300236B
:10C84000012174E60120BDE8F88304F229200022CA
:10C85000B8470126002001463346D4F86C737AE6C7
:10C86000002204F22920984700210123E9E6FFB2C3
:10C87000C5F30746B7E61F46B5E6B1F5917FBFF4AD
:10C88000ACADDCE60D2E0DD10D2B7FF4A6ADD4F8AA
:10C890006433D02284F826225FFA89F9002B7FF4D2
:10C8A000F3AEB4E50E2B7FF498ADD4F86823E02303
:10C8B00084F826327AB12E0C690C06F07F0301F45D
:10C8C0007E5119435FFA89F9A1F500514846904716
:10C8D000F6B22F0E87E65FFA89F998E5B1F5917FF8
:10C8E0007FF435AE0B460BE7B1F5607F28BF4FF400
:10C8F0006071F8B506460D4672B649F2905749F296
:10C900000A630024C2F20007C2F2000349F2985001
:10C910002146C2F2000070223E601C8006F0ECFA54
:10C92000D5B149F298572146C2F2000701244809BF
:10C9300001F01F0257F8203004FA02F201311343CC
:10C94000A94247F82030F2D130460023438001331A
:10C95000AB4200F58270F9D162B6F8BDF0B472B6A0
:10C9600049F20A67C2F2000749F298563C88C2F2BF
:10C97000000606EB840006F17003984212D256F8C6
:10C98000241099B9021D06F17305631CAD1A03EB5F
:10C99000950503E052F8041B41B90133AB421C4634
:10C9A0001046F7D162B60020F0BC7047B1FA81F3AF
:10C9B0004FF00042DA4021EA0201016001B901347E
:10C9C00049F20C61C2F200013C800A88013294B243
:10C9D0000C8062B6801B8010C3EB401000EB80100F
:10C9E00049F290518300C2F2000103F5FB5308683D
:10C9F0001C33012549F28C51C554C2F20001184480
:10CA00000B889A4288BF0C80F0BC7047428872B68F
:10CA10000378012B03D9013B037062B6704749F2DA
:10CA200098535011C2F20003D24370B402F01F02B7
:10CA300053F820404FF0004525FA02F2144343F822
:10CA4000204049F20A6149F20C63C2F20001C2F2CD
:10CA500000030E881A88B04202F1FF3238BF088006
:10CA60001A8062B670BC7047C368B3B130B401E0DD
:10CA7000DB688BB1187A9042FAD158685C7A006909
:10CA800050F82450002DF3D140F8241008780130DC
:10CA90000870DB68002BEDD130BC7047437A8B42C5
:10CAA00006D90369002253F8210043F8212070477A
:10CAB00000207047F8B5437A8B4270D9036953F868
:10CAC0002150002243F82120002D68D02B78012B23
:10CAD00029D972B649F20A6EC2F2000E49F298578D
:10CAE000BEF80040C2F2000707EB840007F17003B4
:10CAF000984212D257F82410B9B9021D07F17306F3
:10CB0000631CB61A03EB960603E052F8041B61B9E6
:10CB10000133B3421C461046F7D162B62B78013B75
:10CB20002B700020F8BD2846F8BDB1FA81F34FF014
:10CB30000042DA4021EA0201016001B9013449F200
:10CB40000C61C2F20001AEF800400A88013296B2D0
:10CB50000E8062B6C01B8010C3EB401000EB80104B
:10CB600049F290518300C2F2000103F5FB531C33DC
:10CB70000868012449F28C51C454C2F20001C4185F
:10CB80000B889A4200D90E804FF48072291D201D17
:10CB900000F0B6FE2B78013B2B702046F8BD00203C
:10CBA000F8BD00BF037C23BB4368427A5B7A9A429C
:10CBB0001FD830B472B60468E3682BB3DA6832B1B8
:10CBC00019688C4216D01346DA68002AF8D1D8606A
:10CBD0000023C360A37A0133A37202684168012372
:10CBE00013728A7A1A448A7242681372037462B6A4
:10CBF00030BC70475D6841688D42E4D11989038972
:10CC00009942F4D01346DFE7E060E1E7037C4BB3E1
:10CC10004368427A5B7A9A4224D872B60268D36833
:10CC200003B3984202D11EE0984202D0DB68002B89
:10CC3000FAD14368427A1B69002143F82210026846
:10CC4000937A013B937203689A7A02B91A72426826
:10CC5000937A013B937243689A7A02B91A7200235D
:10CC6000037462B67047C368D360E2E749F2945335
:10CC7000C2F200031A788AB94EF24040CEF20000A8
:10CC80004EF2081110B4CEF20001D024047001223B
:10CC900010460A601A705DF8044B70470020704718
:10CCA0004EF6FC52CEF20002F8B511684FF48053F4
:10CCB000CEF2000341F08071116049F288511A6888
:10CCC000C2F2000141F2040542F00102CEF2000579
:10CCD0000C681A602E6814B915E064699CB1237A57
:10CCE000002BFAD023682F681B68204698472B68D2
:10CCF000E188DB1B1B099AB28B42A28088BFE280CD
:10CD00006469002CEBD141F20403CEF2000349F236
:10CD100008621B68C2F200029B1B49F20E61148874
:10CD20001B09C2F2000198B2A342088001D9108009
:10CD3000F8BDF8BDF0B572B6B1B90468A4B1027916
:10CD40000F2A11D849F21061C2F200010B8843FA90
:10CD500002F5EF070DD502F1007202F59062B4EB17
:10CD6000421F06D162B6F0BD49F21061C2F2000165
:10CD70000B8813F0010226D09E0767D55D0767D5A3
:10CD80001C0767D5DA0667D59F0667D55E0667D5A7
:10CD90001D0667D5DC0567D59A0567D55F0567D59C
:10CDA0001E0567D5DD0467D59C0467D55A0409D5EF
:10CDB000DA0B08BF0F2206D062B6002210230260F1
:10CDC0000371F0BD0E220124944023430B8062B610
:10CDD00048F24005D1B2C4F2040501712E6848F250
:10CDE0003C04C4F2040446F002062E6002F1007313
:10CDF000226842F0020222604FF4004E48F21A0705
:10CE000048F21E0648F2180548F21F0403F5906325
:10CE1000C4F2000EC4F20007C4F20006C4F200051A
:10CE2000C4F200045B0140F28242CEF80020397067
:10CE3000002231702970217003601A605A609A6074
:10CE4000DA601A615A619A61DA61F0BD0122BAE7CB
:10CE50000222B8E70322B6E70422B4E70522B2E7CC
:10CE60000622B0E70722AEE70822ACE70922AAE7CC
:10CE70000A22A8E70B22A6E70C22A4E70D22A2E7CC
:10CE800003790F2B18D848F21A02C4F2000210B42A
:10CE9000137072B649F21063C2F200030479198864
:10CEA0000122A24021EA02021A8062B61022002367
:10CEB0005DF8044B02710360704700BF10B4EFF3DC
:10CEC000108272B6437F33B9017F012908D003294C
:10CED00016D00123437702B962B65DF8044B704760
:10CEE00049F22461C2F200010C6804B349F22061E6
:10CEF000C2F2000143610B68836108605861E8E792
:10CF000049F21461C2F200010C68CCB149F2186117
:10CF1000C2F2000143610B688361086058614EF6FC
:10CF20000453CEF200034FF080511960D1E749F26B
:10CF30002063C2F200034461846108601860C8E79E
:10CF400049F21863C2F2000344618461086018600A
:10CF5000E5E700BF70B5EFF3108272B649F21464D2
:10CF6000C2F20004206898B149F21866C2F20006C5
:10CF700000254369236073B19D6102B962B64577AC
:10CF800083689847EFF3108272B620680028F0D1CA
:10CF900002B962B670BD3360EFE700BF2DE9F84318
:10CFA00049F21C66C2F200063468002C38D02368AF
:10CFB000002B33D148F6FD0949F214674EF60458A8
:10CFC0001D46C0F20009C2F20007CEF20008A368B5
:10CFD00003B1DD6020693360036825751B684B452C
:10CFE00070D1037F4560022BC4606FD0EFF31082D5
:10CFF00072B6437F43B9017F012900F0968003296F
:10D0000000F0A6800123437702B962B66368002B63
:10D0100042D1346824B12368002BD8D0013B23606F
:10D02000EFF3108272B649F22C63C2F200030021C2
:10D030001868196002B962B6002800F0C1804FF08C
:10D0400000083568C4464FF0020E0EE0CB1A85602A
:10D05000C0F80CC001462B60E8604FF0010880F872
:10D0600014E00D463846002F54D08768002D56D066
:10D07000036829688B42E9D32C4603E011688B4290
:10D08000144638D3A2685B1A0360002AF6D1826086
:10D09000C4602946A060E2E73068236049F21C6260
:10D0A000C2F20002002872D001688B4211D2CB1A62
:10D0B000A060E5600360C46014602046022323750D
:10D0C0000446A8E72246002198479FE783689847CF
:10D0D0009CE7864603E011688B42964648D3DEF80B
:10D0E00008205B1A2360002AF5D1A260C4F80CE086
:10D0F000CEF80840E2E7D268C2608460E060C268AF
:10D10000CB1A294690600D46236080F814E038461B
:10D11000002FAAD1B8F1000F54D1BDE8F883856083
:10D12000C56001464FF0010899E749F22461C2F257
:10D130000001D1F800E0BEF1000F2DD049F22061CE
:10D14000C2F2000143610B6883610860586159E7CE
:10D15000396861B349F21861C2F2000143610B689A
:10D160008361086058614FF08053C8F8003049E788
:10D17000D268E260C4F808E0CEF80C40E268CB1A4E
:10D1800002219460CEF800302175044643E7A06088
:10D19000E0601460204691E749F22063C2F2000388
:10D1A000C0F814E0C0F818E0086018602AE749F2F7
:10D1B0001863C2F200034161816138601860D2E7F0
:10D1C000BDE8F8833160BDE8F88300BF49F23463FD
:10D1D000C2F200031A6801321A60FFF7DFBE00BF17
:10D1E0000368C9B21B6818470368C9B21B681847AF
:10D1F0000368C9B21B6818470368C9B21B6818479F
:10D2000008B5084601F04EFB012008BD08B50846E8
:10D2100001F048FB012008BD38B508460D4605F071
:10D22000CFFE04460146284601F09CFB204638BD4F
:10D2300010B508461446114601F094FB204610BD77
:10D2400001F08EBC08B5084601F0FCFA003018BFAA
:10D25000012008BD08B5084601F0CCFA003018BF1F
:10D26000012008BD0846114601F028BA084601F021
:10D2700079BA00BF084601F001BA00BF01F07EB9DB
:10D280004FF42853C1F2755303EB5100B0FBF1F09A
:10D2900001F094B810B54FF42853C1F275531446F9
:10D2A00003EB5100B0FBF1F001F088F82046BDE837
:10D2B000104001F01FB900BF01F036BC01F0F6BB11
:10D2C00001F0E2BB01F0BEBB01F0CABB704700BF7A
:10D2D000F8B572B106460F4614460025336817F8B4
:10D2E000011B1B6830469847013C0544F6D128468F
:10D2F000F8BD1546FBE700BF70B500298AB00CDB0E
:10D300003ED130238DF8253001222121036801AC64
:10D310005B68214498470AB070BD4CF6CD43494242
:10D32000CCF6CC43A3FB0123DB0803EB8302A1EB88
:10D33000420130318DF82510B3B32D264CF6CD4582
:10D34000CCF6CC452122A5FB0341C90801EB8104A1
:10D35000013AA3EB4403D2B20AAC1444303304F8CC
:10D36000243C0B460029EED106B3013AD2B20AABF7
:10D37000134411462D2203F8242CC1F12202C5E7E3
:10D380004CF6CD43CCF6CC43A3FB0123DB0803EBE7
:10D390008302A1EB420130318DF825100BB100263C
:10D3A000CCE701222121B1E72122DEE71146C2F1BB
:10D3B0002202ABE700B542F23C33C0F20E0383B069
:10D3C00002681B88ADF8043001A95368022298470F
:10D3D00003B05DF804FB00BFF0B507468BB0002A30
:10D3E00033D0012A08BF0A2251B3212400E0F4B24D
:10D3F000B1FBF2F502FB1511C8B2092900F13001A9
:10D4000098BFC8B20AA988BF3730214488BFC0B2CC
:10D4100001F8240C661E2946002DE8D133B1013CE9
:10D42000E4B20AAB23442D2203F8242C3B6801AA62
:10D4300011195B683846C4F1220298470BB0F0BD61
:10D4400030228DF825202124E8E70368C9B21B6843
:10D4500098470BB0F0BD00BF2DE9F04357EC106BBF
:10D460008BB005460C4610EE102A3B4610EE100A13
:10D47000394605F09FF9002840F0F78027F0004971
:10D480004FF6FF73304649464FF0FF32C7F6EF7351
:10D4900005F090F9C0B94FF6FF73304649464FF09A
:10D4A000FF32C7F6EF7305F067F968B92B6842F2EF
:10D4B00048315B682846C0F20E0103229847804637
:10D4C00040460BB0BDE8F0834FF6FF734FF060426B
:10D4D000C4F2EF133046394605F062F9002840F0F7
:10D4E000AB804FF6FF734FF06042CCF2EF13304643
:10D4F000394605F037F9002840F09E8000220023CD
:10D500003046394605F02EF9002840F0A8808046C4
:10D5100000210020C3F6E0717CB14FF0000949F60C
:10D520009913C3F6B97309F101094FF0204204F0D1
:10D53000A7FE5FFA89F39C42F1D802460B463046BB
:10D54000394604F0EBFC06460F4605F071F98146BA
:10D5500000287FD04CF6CD4ECCF6CC4EAEFB00234F
:10D56000DB0803EB8302A0EB420230328DF825206A
:10D57000212283B1AEFB0301C90801EB8100013A0E
:10D58000A3EB4003D2B20AA81044303300F8243C85
:10D590000B460029EED1B8F1000F06D0013AD2B205
:10D5A0000AAB13442D2103F8241C2B6801A9114454
:10D5B0005B68C2F12202284698478046002C3FF45F
:10D5C0007FAF2E2348468DF8043004F0E3FD024679
:10D5D0000B463046394604F09FFC0F2C28BF0F2421
:10D5E00004F101095FFA89F9012400230022C4F241
:10D5F000240304F045FE0F46064605F019F90AAB70
:10D600002344C0B200F1300203F8242C04F0D2FD10
:10D61000013402460B46E4B23046394604F07CFC45
:10D62000A145E2D12B684A4601A95B682846984784
:10D6300040460BB0BDE8F0832B6842F244315B6892
:10D640002846C0F20E0103229847804640460BB0A0
:10D65000BDE8F08330238DF8253021229BE707F1C8
:10D6600000431F464FF0010852E72B6842F2403159
:10D670005B682846C0F20E010322984780461FE7E8
:10D6800030B44FF4804144F20102C4F20701C4F205
:10D69000070249F608036024E120C1F6FF730C700D
:10D6A00010701B784BF20805082B4BF20C0429462E
:10D6B00054D00A2B62D00C2B2346C4F20305C4F2CB
:10D6C0000304C4F20B01C4F20B030CBF35205D2030
:10D6D00012222860226008601A6049F23163C2F2A7
:10D6E00000034BF220011B783BB30B46C4F20B0343
:10D6F000C4F2030101220A601A6049F60903C1F667
:10D70000FF734BF224011B78012B4BD9042B1CD93E
:10D71000082B3ED9102B0B46C4F20B03C4F20301B5
:10D7200094BF862287220A601A6049F23063C2F2EF
:10D73000000301221A7030BC70470A46C4F20B0283
:10D74000C4F203010B601360D7E70B46C4F20B036E
:10D75000C4F2030184220A601A60E6E72346C4F299
:10D760000305C4F20304C4F20B01C4F20B0321202D
:10D7700013222860226008601A60AEE72346C4F2D4
:10D780000305C4F20304C4F20B01C4F20B033920F5
:10D79000EEE70B46C4F20B03C4F2030185220A60D4
:10D7A0001A60C2E70B46C4F20B03C4F203018022E5
:10D7B0000A601A60B9E700BFF0B542F24C33C0F21C
:10D7C0000E0385B0596818689A68DB686C460FC408
:10D7D0000123C4F202031B7899072DD50022C4F25D
:10D7E00002028027137813F0700318BF137000F043
:10D7F000DDFA0720C4F2020004210B220A23C4F23E
:10D800000201C4F20202C4F20203077000261224CD
:10D8100005200E706D461470187072B63446C4F24E
:10D82000020445F001052046A84762B600F0DEFA82
:10D83000237813F070030ED140F641530121C0F25A
:10D840000303C4F2020101E0013B02D00A78D207CF
:10D85000FAD505B0F0BD237005B0F0BDB0F5805F1E
:10D860000CD210B50123C4F2020304461B78DB0777
:10D8700006D504F1A0500078C0B210BD002070475A
:10D88000FFF79AFF04F1A0500078C0B210BD00BFAE
:10D89000B0F5805F23D238B50123C4F202030D46F0
:10D8A0001B78DA0704461BD504F1A0542378AB4259
:10D8B00014D000F07BFA0022C4F20202137813F0B5
:10D8C000700318BF137001222570C4F2020213788E
:10D8D000DB07FCD5BDE8384000F088BA38BD70479A
:10D8E00004F1A054FFF768FF2378AB42E1D1F5E7DC
:10D8F00008B5F6F739F9F7F7F3FE02F0B9FBFAE7E6
:10D90000844641EA000313F003036DD1403A41D34A
:10D9100051F8043B40F8043B51F8043B40F8043B09
:10D9200051F8043B40F8043B51F8043B40F8043BF9
:10D9300051F8043B40F8043B51F8043B40F8043BE9
:10D9400051F8043B40F8043B51F8043B40F8043BD9
:10D9500051F8043B40F8043B51F8043B40F8043BC9
:10D9600051F8043B40F8043B51F8043B40F8043BB9
:10D9700051F8043B40F8043B51F8043B40F8043BA9
:10D9800051F8043B40F8043B51F8043B40F8043B99
:10D99000403ABDD2303211D351F8043B40F8043B39
:10D9A00051F8043B40F8043B51F8043B40F8043B79
:10D9B00051F8043B40F8043B103AEDD20C3205D349
:10D9C00051F8043B40F8043B043AF9D2043208D041
:10D9D000D2071CBF11F8013B00F8013B01D30B88B3
:10D9E00003806046704700BF082A13D38B078DD091
:10D9F00010F003038AD0C3F10403D21ADB071CBF63
:10DA000011F8013B00F8013B80D331F8023B20F8CC
:10DA1000023B7BE7043AD9D3013A11F8013B00F805
:10DA2000013BF9D20B7803704B7843708B7883708D
:10DA30006046704748F2340408B5C4F2040408E0B4
:10DA4000236859050DD423681A050FD42368DB0415
:10DA500011D423685803F3D501F046FA2368590519
:10DA6000F1D501F0A7F823681A05EFD502F084FB81
:10DA70002368DB04EDD502F02DFCEAE708B5FFF7DB
:10DA8000D9FF00BF4FF40053C4F2050310221A80DF
:10DA9000704700BF704700BF42F20E03C4F2050397
:10DAA0004CF2205210B51A804DF628121A8000BF91
:10DAB00000BFFFF7E7FF48F23003C4F204034FF062
:10DAC00030621A6048F23803C4F2040343F68272EB
:10DAD000C0F204021A6048F23C03C4F204030122BB
:10DAE000C2F600321A604EF68853CEF200034FF4AD
:10DAF00070021A604FF40053CEF208030322C8F2FA
:10DB000000521A604DF21002C4F20302136813F4BB
:10DB1000807307D14DF21401C4F203010B604FF47E
:10DB2000A85313604DF20203C4F207031A781107D9
:10DB300003D51A7842F008021A704FF46043C4F219
:10DB40000703AA221A7042F2906149F240634AF236
:10DB50004412C0F20E01C1F6FF73C1F6FF72934288
:10DB600004D251F8040F43F8040BF8E74BF200031A
:10DB700049F6A422C1F6FF73C2F2000200219342CB
:10DB800002D243F8041BFAE748F6004040F20001D5
:10DB90000023C1F6FF70C0F2000151F8232040F8C5
:10DBA0002320013348F60042742BC1F6FF72F4D1F2
:10DBB0004FF464434EF26441CEF200038020CEF273
:10DBC000000103F8010B8B42FBD14EF60853CEF255
:10DBD00000031A604FF4A043C4F206038A221A70AD
:10DBE0004FF48043C4F2060324225A70A0221A7014
:10DBF0009A799207FCD59A79D406FCD44FF48042E6
:10DC0000C4F20602937903F00C03082BFAD14EF20A
:10DC10000103C4F2070360221A704EF20303C4F238
:10DC200007031A78802AFCD14FF48043C4F206031C
:10DC300001221A715D225A719A799006FCD59A795F
:10DC40005106FCD548F24402C4F204020021C0F29D
:10DC50000621116048F24802C4F20402002111605A
:10DC600020221A704FF48042C4F20602937903F026
:10DC70000C030C2BFAD148F20403C4F204034FF452
:10DC80008652C0F207021A604EF21403CEF200036D
:10DC90004BF61F72C0F202021A604EF21803CEF267
:10DCA000000300221A604EF21003CEF20003072296
:10DCB0001A604EF62053CEF200030022C2F2200278
:10DCC0001A6062B600F0F6F84DF21403C4F20303D2
:10DCD0001B68DA070ED54EF67A30C5F6834000F0A1
:10DCE000D3F84EF21C03C4F203034CF2A532C5F67E
:10DCF00094221A604FF47043C4F207031B785B064A
:10DD000012D54EF21C04C4F203044CF2A53322686F
:10DD1000C5F694239A4207D14EF67A30C5F6834071
:10DD200000F0B2F80023236004F0FEFDFFF7B2FE1E
:10DD3000FFF7DEFDFEE700BF08B549F60C03C1F6AC
:10DD4000FF731A6830B169461044A1F5005188424A
:10DD500002D21860104608BD04F0E0FD0C230360F9
:10DD60004FF0FF3008BD00BFFEE700BFEFF31380A8
:10DD700070B9EFF310836BB9EFF305825AB94FF422
:10DD80008070EFF311832BB1984228BF184670477B
:10DD90004FF0FF3070470F2A01D81846F1E74EF2D6
:10DDA000F033CEF20003D05CEBE700BF4EF203028B
:10DDB000C4F207021378802B01D00020704748F28C
:10DDC00044014EF20103C4F204010020C4F207032F
:10DDD00010B4C2F22820002408601C701378802B35
:10DDE000FCD001205DF8044B704700BF4EF20302E7
:10DDF000C4F207021378012B01D0002070474EF2C5
:10DE00000103C4F20703602119701378802BFCD141
:10DE100048F24403C4F204030022C0F206221A604E
:10DE20000120704704F0A8BD04F0A6BDF0B44D1E5B
:10DE30002E46002400E00134B0FBF2F302FB130095
:10DE4000092800F130078ABF3730F8B2C0B206F8AF
:10DE5000010F1846002BEED10A1953704CB11078FF
:10DE600015F8016F28700133E01A834202F8016946
:10DE7000F5DB0846F0BC704748F600431030C1F6A9
:10DE8000FF7343F82010704730B44DF214034DF285
:10DE900004014FF45042C4F20303C4F20301C4F27C
:10DEA0000302002410251C600C6010601D6030BC53
:10DEB000704700BF2DE9F8434EF20413CEF2000381
:10DEC0004FF000621A604FF080521A604FF000521B
:10DED0001A6048F204004FF080421A60C4F2030056
:10DEE0004FF0004248F2080C48F20C071A60C4F2E6
:10DEF000030C0022C4F20307026028234EF6FF70D1
:10DF000048F2140648F21C0548F2240448F22C0E8C
:10DF100048F23401CCF80000C4F203063B60C4F2BE
:10DF20000305C4F20304C4F2030EC4F2030148F271
:10DF30003C07C4F20307336049F21C0C2B6048F223
:10DF40004406236049F20C05CEF8003049F214046F
:10DF50000B6049F224013B60C4F20B05C4F20B04D0
:10DF6000C4F20B0CC4F20306C4F20B0149F22C07F5
:10DF7000C4F20B07336049F23C0E2B6049F23406C1
:10DF80002360CCF800300B6049F244013B60C4F2DE
:10DF90000B06C4F20B0EC4F20B014FF40047C4F29F
:10DFA00003073360CEF8003049F204060B60092104
:10DFB0003960C4F2030649F2080E49F20C07C4F2B4
:10DFC000030EC4F20307326049F21406CEF80000D3
:10DFD000C4F203063B604FF4104E48F20407C4F24B
:10DFE000030EC4F20B07336048F20806CEF80010A7
:10DFF000C4F20B063A6048F20C0E48F21407C4F261
:10E000000B0EC4F20B0730604FF40046CEF8003020
:10E01000C4F20B063B6049F2040E49F20807C4F251
:10E020000B0EC4F20B0731604FF41046CEF80020FF
:10E03000C4F20B06386048F22C00C4F204002B60D6
:10E0400023603160046848F20401C4F2040144F41E
:10E0500000740460086849F2040EC4F20C0E49F220
:10E06000080749F20C0649F214054FF4104440F039
:10E070000070C4F20C07C4F20C06C4F20C05C4F222
:10E080000C040860CEF8002047F6FF7108223960C2
:10E0900033602B602260FFF7F3FA72B64EF218037A
:10E0A00049F234644EF60452C2F20004CEF2000388
:10E0B000CEF200021B682568126862B6510102D5D3
:10E0C000322B88BF0135C3F52F3303F21F3346F6D9
:10E0D00017479B08C1F2C1674FF47A72A7FB03137D
:10E0E00002FB05F54EF218094EF6045805EB9305B0
:10E0F000CEF20009CEF20008192672B6D9F8001047
:10E100002268D8F800E062B6C1F52F3303F21F335E
:10E110009B08A7FB03031EF0806FC5EB93034FF42E
:10E120007A7002D0322988BF013200FB0233B3F586
:10E130007A7F04D3013E05D005F57A75DDE701F05D
:10E1400097FFDAE701F080FC72B64EF218034EF644
:10E150000452CEF20003CEF200021B68256812685A
:10E1600062B6520102D5322B88BF0135C3F52F3379
:10E1700003F21F3346F617479B08C1F2C1674FF4FD
:10E180007A72A7FB031302FB05F54EF218094EF64F
:10E19000045805EB9305CEF20009CEF2000840F2D8
:10E1A000131672B6D9F800102268D8F800E062B6EB
:10E1B000C1F52F3303F21F339B08A7FB03031EF0A7
:10E1C000806FC5EB93034FF47A7002D0322988BF79
:10E1D000013200FB0233B3F57A7F04D3013E05D050
:10E1E00005F57A75DDE701F043FFDAE7BDE8F8836E
:10E1F0003F280FD810B442F25C33C0F20E0353F83C
:10E20000302092F8804234B1012379B182F8803015
:10E210005DF8044B704703EBC0035B681A6841B9B3
:10E2200022F002021A605DF8044B704782F8003158
:10E23000F9E742F003021A60F5E700BF3F2823D850
:10E2400042F25C33C0F20E0303EBC00201295268B4
:10E250000FD004291DD053F83000002380F88032FD
:10E2600099B1022922D003290DD14FF48173136093
:10E27000704753F830004FF4A27380F88012136097
:10E28000136823F02003136070474FF4807313600A
:10E29000704753F830104FF4A273012081F88002C8
:10E2A0001360136843F020031360704740F20313B8
:10E2B0001360704772B64EF2180349F234624EF69C
:10E2C0000451C2F20002CEF20001CEF200031B683C
:10E2D00010680A6862B6520102D5322B88BF01303D
:10E2E000C3F52F3303F21F3346F61741C1F2C16164
:10E2F0004FF47A729B08A1FB031302FB00F000EBC2
:10E30000930070472DE9F843054672B64EF21803A4
:10E3100049F234664EF60452C2F20006CEF2000311
:10E32000CEF200021B683468126862B6520102D550
:10E33000322B88BF0134002D3DD0C3F52F3303F2BB
:10E340001F3346F617479B08C1F2C1674FF47A7234
:10E35000A7FB031302FB04F44EF218094EF604580F
:10E3600004EB9304CEF20009CEF2000872B6D9F89D
:10E3700000103268D8F800E062B6C1F52F3303F21E
:10E380001F339B08A7FB03031EF0806FC4EB9303AE
:10E390004FF47A7002D0322988BF013200FB023379
:10E3A000B3F57A7F04D3013D05D004F57A74DDE737
:10E3B00001F05EFEDAE7BDE8F88300BF48F2340200
:10E3C000C4F20402F0B5116849F28063C2F200039E
:10E3D00041F4806111601F7849F2C46649F23D65DD
:10E3E00049F2CC6449F2C56149F23C62C2F20006CE
:10E3F000C2F20005C2F20004C2F20001C2F2000241
:10E400000023152F33702B7023700B70137061D0A5
:10E410001B2F57D0002F3FD049F61003C1F6FF73D2
:10E420001B78052B46D01A2B5CD0012B24D01F283B
:10E430002BD80020064601254FF42043C4F20603E2
:10E440004EF21F414FF46142CEF200011E700424CF
:10E450005D70CEF200024FF0020E88273C26402568
:10E4600098729C704FF0004083F813E05C751F7445
:10E47000DE700D701060F0BD4AF24403C4F2040374
:10E480004FF451721F281A60D3D9C0F34436C0F339
:10E49000471500F01F00CFE74AF24003C4F204031F
:10E4A00040F213321A6049F61003C1F6FF731B786D
:10E4B000052BB8D14CF21C03C4F204034FF4517283
:10E4C0001A60B4E749F23C03C4F2040340F2133289
:10E4D0001A60A1E74CF21803C4F2040340F21332AD
:10E4E0001A6099E749F23803C4F204034FF45172F9
:10E4F0001A609CE74FF42043C4F2060341079B785F
:10E5000000F0030203F0EC034FF4204143EA02035E
:10E51000C4F2060100F00F0248BF43F01003042AC2
:10E520008B7025D04FF42043C4F20603C2065B79FA
:10E530004FF4204203F0EF03C4F2060248BF43F059
:10E540001003537192794FF4204302F0EF028106D9
:10E55000C4F2060348BF42F010029A71C20506D504
:10E560005A781978D2B241F0200119705A70704768
:10E570008B7943F040038B71D4E700BF48F234033A
:10E58000C4F204031B685B0557D510B549F23C641F
:10E59000C2F20004237823B101F06AFD2378002B36
:10E5A000FAD14EF280114FF42042CEF20001C4F2B3
:10E5B000060249F280634FF000440020C2F20003DB
:10E5C0000C60D0701B78152B38D01B2B4ED033B974
:10E5D0004AF24003C4F2040340F203121A6049F6FF
:10E5E0001003C1F6FF731B7803F07F03052B35D0B2
:10E5F0001A2B2BD0012B06D14AF24403C4F2040398
:10E6000040F203121A6049F23860C2F200004FF47F
:10E610002041C4F2060149F2C46249F23D63C2F2EC
:10E620000002C2F2000300680C79C9790021117060
:10E63000197008B10123037010BD70474CF2180324
:10E64000C4F2040340F203121A60C8E749F2380327
:10E65000C4F2040340F203121A60D4E74CF21C0324
:10E66000C4F2040340F203121A60CCE749F23C03FF
:10E67000C4F2040340F203121A60B0E749F23C62AC
:10E6800038B5C2F200020546137803F0FF04002BF0
:10E69000FAD101212846FFF7D1FD21462846FFF790
:10E6A000A7FD42F25C32C0F20E0249F2C863C2F228
:10E6B000000352F835201A6038BD00BF09B140F0A0
:10E6C000800049F61003C1F6FF731A78904220D0FB
:10E6D00010B448F23404C4F204042468640515D567
:10E6E00002F07F02052A35D01A2A2CD0012A17D031
:10E6F000002900F07F020CBF4FF451714FF45871A4
:10E70000052A1AD01A2A12D0012A03D018705DF8EF
:10E71000044B70474AF24402C4F204021160F5E768
:10E720004AF24402C4F2040200241460E0E749F211
:10E730003802C4F204021160E8E74CF21C02C4F291
:10E7400004021160E2E749F23802C4F20402002434
:10E750001460CDE74CF21C02C4F2040200241460E1
:10E76000C6E700BF49F28063C2F200031A78824212
:10E7700011D048F23401C4F204010968490509D5F1
:10E78000152A2FD01B2A26D072B1152813D01B288A
:10E7900019D008B1187070474AF24002C4F204025E
:10E7A00040F213311160F5E74AF24001C4F204016E
:10E7B00015280A60EBD14CF21802C4F2040240F2B0
:10E7C00013311160E6E749F23C02C4F2040240F260
:10E7D00013311160DEE749F23C02C4F20402002169
:10E7E0001160D2E74CF21802C4F204020021116059
:10E7F000CBE700BF48F23403C4F204031B6813F4F0
:10E80000806308D03F2808D949F23863C2F2000378
:10E810000020186070471846704742F25C3310B50C
:10E82000C0F20E0349F23864C2F2000453F83030EB
:10E8300023600121FFF702FD236800221A700120E6
:10E8400010BD00BF48F23403C4F204031B6813F484
:10E8500080630DD012280DD014281BD04FF4204314
:10E86000C4F2060300205A7B02F0FE025A7370477E
:10E87000184670474AF20C03C4F2040340F2023215
:10E880001A604FF42043C4F2060301205A7B02436E
:10E890005A7370474CF21403C4F2040340F202327C
:10E8A0001A60EEE72DE9F84F48F23403C4F204038E
:10E8B0001B685A054FD549F2C863C2F200031B68B2
:10E8C0000BB101221A7049F2CC69C2F2000949F277
:10E8D000C56599F8004001343F2C88BF4FF0000A0D
:10E8E000C2F2000549F240684FF4204694BF5FFA37
:10E8F00084FA54460746AB46C2F20008C4F2060644
:10E900002B78A34216D1FFF731FA402825DC337962
:10E910001B06F5D59BF8003001333F2B86BF002244
:10E920001346DAB218F80330DBB2F3712A702B7891
:10E93000A342E8D049F23C634FF42042C2F2000304
:10E94000C4F20602FFB20120BC2108F8047018705E
:10E9500089F800A0D170BDE8F88FFF28D0DD01F064
:10E9600087FBCDE748F23403C4F204031B685A0561
:10E9700066D52DE9F04F49F2C863C2F2000383B0B7
:10E980001B6805460BB101221A706B189D4201935A
:10E990004DD249F2CC6849F2C56449F2406949F266
:10E9A0003C6B4FF42047C2F20008C2F20004C2F2EE
:10E9B0000009C2F2000BC4F206070BE015F8012BA8
:10E9C00009F80A2001238BF80030019B88F80060C9
:10E9D000AB422CD098F80030227803F1010ABAF14A
:10E9E0003F0F86BF0026B2465FFA8AF69245E5D110
:10E9F000BC22FA7005E03A7913060BD422789245CE
:10EA0000DCD1FFF7B3F94028F5DDFF28F6DD01F092
:10EA10002FFBF3E7227801323F2A86BF00210A4606
:10EA2000D1B219F80220D2B2FA712170E6E74FF4A0
:10EA30002043C4F20603BC22DA7003B0BDE8F08FB5
:10EA4000704700BF10B549F23C64C2F2000423785D
:10EA500023B101F00DFB2378002BFAD110BD00BFCC
:10EA600049F2CC6349F2C562C2F20002C2F200036D
:10EA70001B781078DBB2C0B283422CBF3F3000F16C
:10EA8000FF30C01A704700BF49F2C46249F23D63CB
:10EA9000C2F20002C2F2000310781B78C0B2DBB2EF
:10EAA000984238BF4030C01A704700BF30B449F2B6
:10EAB000C46349F23D64C2F20003C2F200041A7852
:10EAC0002378D2B2DBB29A422AD001333F2B14D939
:10EAD00049F2846149F23863C2F20001C2F20003D4
:10EAE000087819680023C0B2237021B1D31A1A2BF9
:10EAF00001DC00230B7030BC704749F2846049F29E
:10EB00003861C2F20000C2F20001C05C0968DDB2E7
:10EB1000C0B225700029EED09A4238BF4032E5E7F6
:10EB20004FF0FF30E7E700BF49F2C46249F23D63AE
:10EB3000C2F20002C2F2000312781B78DBB29A42E2
:10EB40000AD00133402B49F2846228BF0023C2F26D
:10EB50000002D05CC0B270474FF0FF30704700BF7A
:10EB600048F23403C4F204031B685B0520D54FF45C
:10EB70002043C4F206034021DA7802F0CB02DA70B7
:10EB80005974D87849F23D6240F03400C2F2000274
:10EB900049F23861D870C2F200011278096849F26E
:10EBA000C463C2F20003D2B21A7009B100230B7021
:10EBB000704700BFF0B44FF42043C4F206031A7943
:10EBC00012F0300F38D072B6997D01F0FF020029A3
:10EBD00058D062B649F2C46749F23D61C2F20007FB
:10EBE000C2F200013C780D7849F284661846E4B21E
:10EBF000EDB2C2F20006631C402BC17928BF00238E
:10EC0000AB4202F1FF32C9B21CBFF1541C4612F0F4
:10EC1000FF02F0D149F23862C2F20002E3B2126898
:10EC20003B704AB1AC4236BFC5F14005641B641964
:10EC3000272CC4BF012313704FF42042C4F20602F4
:10EC4000D178C9B20D0622D44A0619D54FF4204313
:10EC5000C4F206031B795B0612D549F2C862C2F200
:10EC6000000249F23C63C2F20003126800211970ED
:10EC700002B111704FF42043C4F206033C22DA7053
:10EC8000F0BC70474022D9795A7462B6D4E7137940
:10EC90001C06D9D549F2CC6349F2C566C2F200031D
:10ECA000C2F200061C783378E4B2DBB29C4211D089
:10ECB00049F24065C2F2000501E0A3420AD00133E7
:10ECC000402B28BF00231079E85CC0B2D071107DC2
:10ECD0000728F2D94FF42042DBB2C4F206023370A7
:10ECE0001379180644BF7C23D370ADE7431E042B71
:10ECF0001AD872B649F22C72C2F2000252F82300FE
:10ED000080B149F68821C2F2000170B4058831F85B
:10ED10001340466842F82360621B21F8132062B654
:10ED200070BC704762B670470020704701380428F5
:10ED30000ED872B649F28473C2F2000353F8203041
:10ED400043B100205B680130002BFBD162B67047F5
:10ED5000002070471846F9E770B472B642F2845248
:10ED6000C0F20E0213781E0709D540F20003C1F667
:10ED7000FF73196A002960D0996A00295FD053781F
:10ED80001D0709D540F20003C1F6FF73196C002975
:10ED90005BD0996C002954D093781C0709D540F2B8
:10EDA0000003C1F6FF73196E002950D0996E002937
:10EDB00049D0D378190709D540F20003C1F6FF7393
:10EDC000D3F8801079B3D3F88810C1B113791B0739
:10EDD0000BD540F20003C1F6FF731425D3F8A02031
:10EDE00012B3D3F8A820152552B162B649F2B57313
:10EDF000C2F2000300221A7070BC00F0D9BE1125C7
:10EE000049F2B572C2F2000203EBC5061178C824BC
:10EE100008300139C0F240047060117043F8354089
:10EE200062B670BC7047102549F2B572C2F200029A
:10EE300003EBC50611788824EAE70425F4E70525E5
:10EE4000DEE70925DCE70D25DAE70825ECE70C25E8
:10EE5000EAE700BF431E042B27D8400140F200021E
:10EE6000C1F6FF7240F0100030B4104472B649F29F
:10EE7000C472C2F20002D45C012C27D02BD3022C26
:10EE800027D0032C12D049F28470C2F2000050F84F
:10EE9000232012B349F29872C2F2000252F8230002
:10EEA000416042F8231062B630BC70470830042538
:10EEB0000C88D55410F0080F14BFC823882343EAE8
:10EEC000044308310360416062B6EDE70830022573
:10EED000EEE70525ECE70325EAE749F2987240F8EA
:10EEE0002310C2F20002DCE72DE9F04F42F2940356
:10EEF0008BB042F298024FF4035142F2C4004FF437
:10EF0000025B42F29009C4F20703C4F20702C4F2A2
:10EF10000701C4F20700C4F2070BC4F2070901930A
:10EF200002920591069053E040F200059E08C1F65A
:10EF3000FF7505EBC608441ED8F8042003F008034B
:10EF4000E4B2A2F1080003F0FF07002B40F0AB8011
:10EF500055F836301B0C99B222F8081C002B00F033
:10EF6000958049F22C7EC2F2000E22F8067C5EF8F3
:10EF7000243042F8047C49F2D46A002B00F09B82D2
:10EF8000C2F2000A5AF82420506049F68827C2F2DB
:10EF900000074AF8240037F81430194427F81410F1
:10EFA00000F0E2FD002800F08B82C822882318F0D0
:10EFB000080FC0F24002C0F2400300F1080018BF81
:10EFC0001346C8F8040045F8363008238BF80030A3
:10EFD0009BF80040E4B2610725D549F2C073C2F244
:10EFE00000031B78E3B149F24173C2F200031978C0
:10EFF00001F0FF0221B1013AD2B21A7002B900BE8B
:10F0000049F2D473C2F20003197801F0FF0229B16A
:10F01000013AD2B21A70002A00F0008200F0F4FD2A
:10F0200004238BF8003004F0080303F0FF02002BE8
:10F0300000F0B78099F80030DBB218097FF474AFA4
:10F0400040F200049A08C1F6FF7404EBC20154F8C0
:10F0500032304968C3F38303092B00F0C28050D8D3
:10F06000013B012B0ED849F2AC73C2F2000342F20D
:10F0700021001B88834200F02681C823C0F2400390
:10F0800044F83230019A012313709EE7C822882386
:10F0900018F0080FC0F24002C0F2400318BF134638
:10F0A00045F8363091E700F083FD49F28472C2F2F0
:10F0B000000252F82410002900F0158249F2C470B1
:10F0C000C2F200004B68075D42F82430012F01F1C5
:10F0D0000803C8F8043000F00382C0F0FE81022F5C
:10F0E00000F0F881032F01D10423035518F0080F15
:10F0F0000A880CBF8823C82343EA024345F8363008
:10F1000063E70D2BBED191E88010C823C0F2400305
:10F1100049F2AC7E49F2D06649F2407544F832308B
:10F12000C2F2000EC2F20006C2F20005BBB240F20B
:10F130008162012193422061A061CEF804C0CEF823
:10F1400000703060297000F29180B3F5D06F80F0CC
:10F150005683B3F5817F00F0048200F2E381802BB7
:10F1600000F04483822B40F00382BEF8043003F0A9
:10F170007F03052B00F2FC814FF4035149F2B87272
:10F180009B00C2F20002C4F207011944002313706D
:10F1900053700B789F0740F1FF8301231370022106
:10F1A00000E3E00700F13D81210600F1AB81A207F9
:10F1B0000CD542F28803C4F207034FF402511A78C7
:10F1C000C4F20701D2B202201A700870E30605D516
:10F1D0004FF40253C4F2070310221A700BB0BDE8BB
:10F1E000F08F49F2D066C2F2000632687AB349F273
:10F1F000E86EC2F2000E49F2407549F2B473C2F2F1
:10F200000005C2F20003BEF800102F7818784029DC
:10F210008C4640F0020828BF4FF0400C002F87F0CA
:10F2200001072F70CCEB01010CBF8825C82504EB2A
:10F23000C80789B280F0010045EA0C457A60AEF853
:10F24000001044F8385062441870B9B3326049F283
:10F25000AC73C2F200031A88B2F5A06F7FF412AF4C
:10F2600000219A785970029B1A700BE742F2210232
:10F27000934200F0CF8059D8B3F5086F00F0888230
:10F28000B3F5106F40F0748149F2C073C2F200030D
:10F2900040F200079EF802201A70C1F6FF7707F1CE
:10F2A000A00803E00837B84500F0B1813B6A1A06B0
:10F2B000F8D5786A083800F07BFCF3E7BCF1400F22
:10F2C00018BF0022C2E749F69423C2F200030D786A
:10F2D00048781D7058708D78C8789D70D8701868FF
:10F2E0000D791D7186284D7989795D71997100F0CC
:10F2F000808149F2B47349F24075C2F20003C2F250
:10F3000000051978287881F00106002841F00201F3
:10F310001E700CBF8823C82344F8313004EBC101B0
:10F3200080F00100002328704B60A6E642F2212203
:10F33000934240F08B8249F23467C2F2000749F6EB
:10F340009C2249F2E473C2F20002C2F200033F6859
:10F350009EF802E017600390079183F800E0002117
:10F36000079F089108468C460A4649F2B473C2F2D8
:10F370000003002F1F78049747F0020E04EBCE0A1B
:10F3800008BF4FF08808CAF8042018BF4FF0C8081B
:10F390003A4640EA080049F2407A40F2000882F01A
:10F3A000010244F83E009DF80C702F7049F2B470D1
:10F3B000C1F6FF78C2F2000A1A70C2F200000029FA
:10F3C00040F0DD80BCF1400F24D142F0020204EB9A
:10F3D000C204089F6760039C40F20000C1F6FF7002
:10F3E0004FEA014E002C40F0E4809DF81C402C7048
:10F3F0004EF0880E9DF8104040F832E00F441C702B
:10F400003C46402906D1002149F2E863C2F20003DC
:10F4100034601980019A0123137033E600F000FE76
:10F42000FCE542F2940449F2B471C4F20704C2F25A
:10F430000001022040F200032070C1F6FF730A7041
:10F4400049F2EC61C2F20001596049F24471C2F222
:10F450000001D9604FF4035C8821C0F24001C4F27E
:10F46000070C42F2880E196099601A619A61C4F221
:10F47000070E0D234FF4025742F2980642F28C0514
:10F4800042F284008CF80030C4F20707FF23C4F274
:10F490000706C4F20705C4F207008EF80030012108
:10F4A0004FF09F0E3B7032702B7080F800E021709F
:10F4B0000BB0BDE8F08F4EF82400C2F2000A64E5FC
:10F4C00049F2B573C2F2000345F836001A780132EA
:10F4D0001A707AE50523035508E60323035505E66C
:10F4E0000223035502E649F2C473C2F200031A5D17
:10F4F000022A7CD0FFF469AD032A40F0818001220A
:10F500001A5562E54FF40352C4F207024FF4025356
:10F51000C4F207030D2010708021A20719707FF537
:10F5200055AE46E640F20232934240F08681BEF884
:10F53000043003F07F0349F2AC72052BC2F20002E3
:10F5400016D85188A1B94FF403529B00C4F20702A8
:10F550001A440391137843F00203137001230793B5
:10F56000FDE6BEF8043003F07F03052B40F2738103
:10F57000059A0F231370019A0123137082E5402925
:10F580007FF623AF42F0020208EBC203089C5C60E6
:10F59000039BE3B19DF81C508AF80050C823C0F2C9
:10F5A00040039DF8105005704039403448F832301F
:10F5B0002AE79DF81C402C709DF810401C70089B99
:10F5C0004EF0C80E0B441C4640F832E019E79DF897
:10F5D0001C408AF800409DF8104004708823089C65
:10F5E000C0F240034039403448F832300CE7195536
:10F5F000EBE449F24173C2F200030F21197078E67F
:10F6000018F0080F0CBF022203221A55DDE449F25C
:10F610002C7349F2847249F2987149F2C47049F628
:10F62000882749F2D46AC2F20003C2F20002C2F291
:10F630000001C2F20000C2F2000704940796089588
:10F64000CDF824B0C2F2000A804600241E461546BA
:10F6500003978B46306828B1476800F0A9FA38460E
:10F66000002FF9D12868002333604AF8243028B1EC
:10F67000476800F09DFA3846002FF9D1002298F82B
:10F6800000302A604BF8042B039A4FF00001032B43
:10F6900022F8141004D074D9042B74D0052B03D194
:10F6A0004FF0010388F800300134052C06F1040600
:10F6B00005F1040508F10108CCD142F2845749F262
:10F6C000B578C0F20E07C2F2000800223B7888F835
:10F6D0000020069A049C079E089DDDF824B0137054
:10F6E0001B0700F1CC807B7842F2C802C4F207020B
:10F6F000002140F2000A18072163A163C1F6FF7AD6
:10F70000137000F13081BB7842F2CC020021C4F2C8
:10F7100007022165A16540F2000A19071370C1F6BE
:10F72000FF7A00F1058142F2D002C4F20702FB78B1
:10F7300000212167A16740F2000A13701A07C1F681
:10F74000FF7A00F1D68042F2D4023B79C4F207027C
:10F75000002140F20007C4F89010C4F8981013700C
:10F760001B07C1F6FF7700F1A6802B7807931A4696
:10F7700082F0010200230392C4F8B030C4F8B8301C
:10F78000EDE5022B90D14FF0000388F800308BE7B5
:10F7900049F2C073C2F2000349F2B872C2F2000229
:10F7A0001B781370BEF80600884280F03A8149F257
:10F7B000B473C2F2000340281978049141F0020E9C
:10F7C00004EBCE01844628BF4FF0400C02EB0C073F
:10F7D0004A60002203920122CCEB000107920897B5
:10F7E0004FEA0C404FF0C808049AD2E549F2B872CB
:10F7F000C2F200020023137053700221D2E742F2DA
:10F800008C53C0F20E035A68002A3FF4B1AEBEF822
:10F810000200BEF8047004E00C335A68002A3FF47A
:10F82000A7AE19888142F7D15988B942F4D1000AAC
:10F8300003280CBF11781989B4E7B3F5A06F7FF4E2
:10F8400097AE002303930123079388E542F2213208
:10F850009342F6D08CE6BEF80220002A7FF488AEF0
:10F860004FF403529B00C4F207021A44002303938F
:10F87000137823F002031370012307936FE500F060
:10F8800073F9002800F0B98000F108038820636252
:10F89000C0F24000206200F067F940F20003C1F6B8
:10F8A000FF73002800F0A280C8220830C0F2400296
:10F8B000D8629A6217E700F057F9002876D000F175
:10F8C00008038820C7F8A430C0F24000C4F8A000A4
:10F8D00000F04AF940F20003C1F6FF7300285DD042
:10F8E000C8220830C0F24002C3F8AC00C3F8A82018
:10F8F0003BE700F039F9002800F08D8000F10803A3
:10F900008820CAF88430C0F24000C4F8800000F0BB
:10F910002BF940F20003C1F6FF73002873D0C82210
:10F920000830C0F24002C3F88C00C3F888200AE710
:10F9300000F01AF9002853D000F108038820CAF813
:10F940006430C0F24000206600F00EF940F200037F
:10F95000C1F6FF7300283CD0C8220830C0F2400234
:10F96000D8669A66DFE600F0FFF860B300F108039E
:10F970008820CAF84430C0F24000206400F0F4F857
:10F9800040F20003C1F6FF73B0B1C8220830C0F2E4
:10F990004002D8649A64B6E6022103E798F8002092
:10F9A000C3F8A800531C88F80030DEE698F8003051
:10F9B000013388F8003089E798F800209864531CD8
:10F9C00088F800309FE698F80030013388F800305E
:10F9D000D3E798F800209866531C88F80030A2E618
:10F9E00098F80030013388F80030ACE798F8002030
:10F9F0009862531C88F8003075E698F8003001339F
:10FA000088F8003046E798F80020C3F88800531CB7
:10FA100088F8003097E698F80030013388F8003015
:10FA200073E740298C4628BF4FF0400C02EB0C03D3
:10FA30000893002303930123CCEB01014FEA0C4010
:10FA400007931F4691E400BFF8B540F20004C1F6E9
:10FA5000FF7400F095FE04F1A800234600221A600E
:10FA60005A60083383424FF00001F8D148F2340263
:10FA7000C4F204024FF458431068C4F2000340F487
:10FA8000802010601A6842F2441EC4F2070E42F051
:10FA900040724FF405571A60C4F20707032342F27D
:10FAA0009C068EF80030C4F20706A02342F2B0058F
:10FAB0003B70C4F20705C4F3072342F2B40C4FF4C1
:10FAC000025042F288023370C4F20700C4F30743C5
:10FAD000C4F20702C4F2070C42F2100E2B70240E7F
:10FAE000FF23C4F2070E42F294074FF404568CF839
:10FAF0000040C4F207070370C4F20706137042F215
:10FB000084054EF235444EF2041042F208128EF88B
:10FB10000030C4F207050123CEF20004CEF200004B
:10FB2000C4F207023B70317070274FF400161021A9
:10FB30002B70277006601170F8BD00BF00F002B98D
:10FB400000F0D6B800F0AEB800F0ECB800F036BA6D
:10FB500000F00CBA0846114600F012B9084600F051
:10FB6000F9B900BF704700BF72B649F62402C1F66A
:10FB7000FF721168B1FA81F31D2B16DC4FF00040C3
:10FB8000D84021EA000110B4116062B648F6D052A4
:10FB900003EBC303DB00C1F6FF72D1180024D4507D
:10FBA00008464C605DF8044B704762B60020704711
:10FBB00048F6D053C1F6FF7348F63962C31AC3F64C
:10FBC000E302A2FB03231B091D2B12D849F2B572D5
:10FBD000C2F2000212786AB972B649F62402C1F67E
:10FBE000FF724FF00040116820FA03F319431160CF
:10FBF00062B6704749F2C072C2F200021278002A5F
:10FC0000EAD0FFF7A9B800BF38B549F2C973C2F20C
:10FC100000031D783DB949F2CC74C2F2000421689A
:10FC200009B14B8803B938BD9B000B800420FFF756
:10FC300011F9256038BD00BF70B549F2D074C2F229
:10FC400000042368B3B11E885A88910803EB810130
:10FC50000432B2428D6803D25A802B46184670BDDA
:10FC60001846FFF7A5FF0520FFF740F82B46206058
:10FC7000184670BD49F2C073C2F200031B780BB97D
:10FC80000023EBE70520FFF731F80346206000284A
:10FC9000F6D00688002ED7D1FFF78AFF26603346BC
:10FCA000DCE700BF38B549F2E074C2F20004206816
:10FCB00078B143880288C118013393420D7A02D289
:10FCC0004380284638BDFFF773FF00232846236092
:10FCD00038BD49F2C073C2F200031B782BB1022079
:10FCE000FFF704F820600028E3D14FF0FF3038BD63
:10FCF00010B549F2E074C2F20004206818B14388DC
:10FD00001844007A10BD49F2C073C2F200031B7898
:10FD10002BB10220FEF7EAFF20600028EFD14FF060
:10FD2000FF3010BD49F2E072C2F2000249F68823AA
:10FD3000C2F20003126858881AB1138852889B1ABD
:10FD40001844704749F2C073C2F200031B78B3B184
:10FD500010B549F2E074C2F20004206848B1FFF720
:10FD600027FF002302202360FEF7C0FF30B1FFF71A
:10FD70001FFF0220FEF7BAFF0028F8D110BD704720
:10FD80002DE9F04F49F2D57B83B0C2F2000B01237D
:10FD90008BF80030009100297CD049F2D878C2F26B
:10FDA0000008044649F2C077D8F80000CDF804B046
:10FDB0000E46C2F20007002800F08A8049F2DC7586
:10FDC000C2F20005B0F802E0CEF14002B24228BF14
:10FDD00032460EEB020189B200F108034FF0000A2F
:10FDE000B61A418002F1FF3C734485F800A0002A56
:10FDF00044D00EF108010EF10C0E251D014486447D
:10FE0000A94238BF74452CBF01250025092A94BF9B
:10FE1000002505F00105002D51D044EA0105AD078C
:10FE20004DD1A2F1040E4FEA9E0E0EF1010EBCF16F
:10FE3000020F4FEA8E0940D955469B46A4F1040AA9
:10FE400001355AF8043F41F8043BAE45F8D85B460B
:10FE50004A454B44C9EB0C0C04EB09016DD00D78FD
:10FE60001D70BCF1000F26D04D785D70BCF1010F04
:10FE700021D0897899702244418814463F2910D8AE
:10FE800049F2D473C2F2000305221A70002E92D1F7
:10FE9000DDF804B0009800238BF8003003B0BDE813
:10FEA000F08F4023038001460320FEF7D3FF00209C
:10FEB000C8F80000E4E72244DEE72146CFE7013B33
:10FEC000224414F8011B03F8011F9442F9D1D3E72F
:10FED0003B78A3B344F6210949F2DC75C0F201096D
:10FEE000C2F200054FF0010ADDF804B008E0B9F1F4
:10FEF00001091BD02B78CBB900F0BAF83B7803B3DB
:10FF00000320FEF713FF0728F1D88BF800A0FFF7B6
:10FF10002BFEC8F8000000287FF454AF49F2D573D7
:10FF2000C2F20003B9F101091870E3D101234FF0C7
:10FF3000FF302B7003B0BDE8F08F0A469CE7DDF878
:10FF400004B000234FF0FF308BF8003003B0BDE861
:10FF5000F08F00BF00B583B002AB012103F8010DA3
:10FF60001846FFF70DFF03B05DF804FB38B549F202
:10FF7000D875C2F2000549F2D574C2F200042868AF
:10FF80000123237028B1408800232370C0F1400072
:10FF900038BD49F2C073C2F200031B7813B90020C8
:10FFA000207038BD0320FEF7C1FE0728F7D8FFF701
:10FFB000DBFD28600028E6D1F1E700BFF8B549F283
:10FFC000C073C2F200031B78D3B149F2D875C2F2F4
:10FFD000000549F2D574C2F200042E68012727708B
:10FFE0007EB149F2D473C2F20003002772881F70F9
:10FFF000314632800320FEF72DFF2F60002323704F
:020000021000EC
:10000000F8BDFFF7B1FD49F2D473C2F2000328B185
:10001000014603201E70FEF71DFFEFE71F70EDE79E
:1000200038B549F2D573C2F200031B78A3B949F27F
:10003000D874C2F20004216879B103F0FF054B883F
:100040000B800320FEF706FF256038BD49F2D4730C
:10005000C2F2000301221A7038BDFFF785FD0028A7
:10006000F4D00146BDE838400320FEF7F3BE00BFE0
:1000700038B549F2E574C2F20004237803B138BD03
:1000800001232370FFF74EFE002849D1FEF7FCFC48
:10009000002842D100F05EF800283BD100F008F9BA
:1000A000002834D100F09CF970BB00F031FA40BB5D
:1000B00000F0C6FA10BB00232370EFF30583002B7A
:1000C000DDD1EFF3108172B649F22463C2F200036E
:1000D000186840B349F22864C2F20004227812BBC7
:1000E00045691D60012323700DB3AA6101B962B691
:1000F00000254577836898472570C0E700F028F809
:10010000D9E700F023F8D3E700F01EF8CDE700F0C0
:1001100019F8C7E700F014F8C0E7FDF7D7F8B9E71A
:10012000FFF720FDB2E70029A9D162B638BD49F238
:100130002063C2F200031D600029D9D1D7E700BFB8
:10014000704700BF704700BF704700BF704700BFD7
:10015000704700BF49F6580249F2ED73C2F200023F
:10016000C2F2000310781B78C0B2DBB2984238BFED
:100170004030C01A704700BFF0B44FF43043C4F2AF
:1001800006031A7912F0300F38D072B6997D01F05B
:10019000FF02002958D062B649F6580749F2ED71BE
:1001A000C2F20007C2F200013C780D7849F6180649
:1001B0001846E4B2EDB2C2F20006631C402BC179CE
:1001C00028BF0023AB4202F1FF32C9B21CBFF15479
:1001D0001C4612F0FF02F0D149F2E872C2F20002AE
:1001E000E3B212683B704AB1AC4236BFC5F140057C
:1001F000641B6419272CC4BF012313704FF43042D1
:10020000C4F20602D178C9B20D0622D44A0619D525
:100210004FF43043C4F206031B795B0612D549F64E
:100220005C02C2F2000249F2EC73C2F200031268EF
:100230000021197002B111704FF43043C4F206036B
:100240003C22DA70F0BC70474022D9795A7462B609
:10025000D4E713791C06D9D549F6600349F6590647
:10026000C2F20003C2F200061C783378E4B2DBB2BB
:100270009C4211D049F2F075C2F2000501E0A342A0
:100280000AD00133282B28BF00231079E85CC0B2C4
:10029000D071107D0728F2D94FF43042DBB2C4F29E
:1002A000060233701379180644BF7C23D370ADE780
:1002B00049F6D40249F66903C2F20002C2F2000311
:1002C00010781B78C0B2DBB2984238BF4030C01AF9
:1002D000704700BF30B44FF44043C4F206031A79AC
:1002E00094062ED549F6D402C2F20002D8791378CA
:1002F00049F66901C2F2000101333F2B0978C8BFFA
:1003000000238B42C0B206D049F69404C2F2000426
:10031000D9B2E054117049F66402C2F200021168C9
:1003200079B149F6D502C2F200021278D2B29342F4
:1003300036BFC2F140029B1A9B18272BC4BF012372
:100340000B704FF44042C4F20602D378DBB21806B9
:100350001DD45A0619D54FF44043C4F206031B7945
:100360005B0612D549F6D802C2F2000249F66803CC
:10037000C2F2000312680021197002B111704FF42B
:100380004043C4F206032C22DA7030BC7047117966
:100390000906DED549F6DC0149F6D500C2F20001B6
:1003A000C2F200000C780178C9B28C4214D04A1C09
:1003B000272A88BF002549F66C0188BF2A46C2F269
:1003C000000198BFD5B24FF440448A5CC4F20604E1
:1003D000D2B2E2710570BCE76C21D170B9E700BF01
:1003E00049F6501249F6E503C2F20002C2F20003D8
:1003F00010781B78C0B2DBB2984238BF4030C01AC8
:10040000704700BF30B44FF45043C4F206031A796A
:1004100094062ED549F65012C2F20002D87913780C
:1004200049F6E501C2F2000101333F2B0978C8BF4C
:1004300000238B42C0B206D049F61014C2F2000469
:10044000D9B2E054117049F6E002C2F2000211681C
:1004500079B149F65112C2F200021278D2B2934237
:1004600036BFC2F140029B1A9B18272BC4BF012341
:100470000B704FF45042C4F20602D378DBB2180678
:100480001DD45A0619D54FF45043C4F206031B7904
:100490005B0612D549F65412C2F2000249F6E40393
:1004A000C2F2000312680021197002B111704FF4FA
:1004B0005043C4F206032C22DA7030BC7047117925
:1004C0000906DED549F6581149F65110C2F200016D
:1004D000C2F200000C780178C9B28C4214D04A1CD8
:1004E000272A88BF002549F6E80188BF2A46C2F2BC
:1004F000000198BFD5B24FF450448A5CC4F20604A0
:10050000D2B2E2710570BCE76C21D170B9E700BFCF
:1005100049F6CC1249F66113C2F20002C2F200039E
:1005200010781B78C0B2DBB2984238BF4030C01A96
:10053000704700BF30B44FF42043C4F20E031A7961
:1005400094062ED549F6CC12C2F20002D87913785F
:1005500049F66111C2F2000101333F2B0978C8BF8F
:1005600000238B42C0B206D049F68C14C2F20004BC
:10057000D9B2E054117049F65C12C2F2000211685F
:1005800079B149F6CD12C2F200021278D2B293428A
:1005900036BFC2F140029B1A9B18272BC4BF012310
:1005A0000B704FF42042C4F20E02D378DBB218066F
:1005B0001DD45A0619D54FF42043C4F20E031B79FB
:1005C0005B0612D549F6D012C2F2000249F660135A
:1005D000C2F2000312680021197002B111704FF4C9
:1005E0002043C4F20E032C22DA7030BC704711791C
:1005F0000906DED549F6D41149F6CD10C2F2000144
:10060000C2F200000C780178C9B28C4214D04A1CA6
:10061000272A88BF002549F6641188BF2A46C2F2FE
:10062000000198BFD5B24FF420448A5CC4F20E0496
:10063000D2B2E2710570BCE76C21D170B9E700BF9E
:1006400049F6482249F6DD13C2F20002C2F2000365
:1006500010781B78C0B2DBB2984238BF4030C01A65
:10066000704700BF30B44FF48043C4F20C035A68A3
:1006700094022ED549F64822C2F20002D8681378B7
:1006800049F6DD11C2F2000101333F2B0978C8BFE2
:1006900000238B4207D049F60824C2F20004C0B2FE
:1006A000D9B2E054117049F6D812C2F200021168B2
:1006B00079B149F64922C2F200021278D2B29342CD
:1006C00036BFC2F140029B1A9B18272BC4BF0123DF
:1006D0000B704FF48043C4F20C039A68100202D5E9
:1006E0005B6819021DD4520219D54FF48043C4F23D
:1006F0000C035B685B0212D549F64C22C2F2000281
:1007000049F6DC13C2F2000312680021197002B12D
:1007100011704FF4AC73C4F2883300221A6030BCFD
:10072000704749F6502349F64921C2F20003C2F24C
:10073000000118780B78DBB2984214D00133272BD4
:1007400088BF002549F6E01088BF2B46C2F20000A2
:1007500098BFDDB24FF48044C35CC4F20C04DBB23A
:10076000E3600D70BFE74FF4AE714FF4AC73C4F2A9
:100770008831C4F28833002401200C601860B2E78D
:1007800010B584B072B6FDF711FB00230421C4F24A
:100790000203C4F2020100207022C4F20710802478
:1007A0001A7008601A461C7013781B06FCD50C23BF
:1007B000C4F202031C68FDF719FB62B649F27F63BD
:1007C000C0F298039C429CBF04EB840464000A229C
:1007D000204601A9FDF72AFB9DF8042049F6F00305
:1007E000C1F6FF7352B39DF805105A8061B39DF8AE
:1007F0000620998052B39DF80710DA8041B39DF826
:100800000820198132B39DF809105A8121B39DF84F
:100810000A20998112B39DF80B10DA8101B39DF87B
:100820000C2019824AB19DF80D105A82092229B173
:10083000162299821A7004B010BD082201325200AB
:10084000D2B21A7004B010BD0122F7E70222F5E718
:100850000322F3E70422F1E70522EFE70622EDE7A2
:100860000722EBE70B460146184602F051B800BFDD
:10087000F0B52DED048BB0EE409AF0EE609A3A4C54
:100880008BB000F015FA94F90030B0EE408AF0EE2B
:10089000608A013338D0B0EE490AF0EE690A01F0FF
:1008A000FBF988B32CA3D3E9002351EC190B01F019
:1008B00077FF054680BB2AA3D3E9002351EC190B2F
:1008C00001F050FF00B394F90030284A0895002643
:1008D00000270421022B8DED049B8DED029BCDE9B9
:1008E00006678DE8060030D0684601F0DDF960B398
:1008F000089B1BB102F012F8089B03609DED060BEC
:100900000BB0BDEC048BF0BDB0EE480AF0EE680A07
:100910000BB0BDEC048BF0BD144A94F90030019289
:10092000032100228DED049B8DED029B0091089226
:100930002BB90F4B4FF06042CDE90623D4E70D49A8
:100940000020022BCDE90601CED101F0E7FF2223E2
:100950000360CDE7AFF30080EF39FAFE422E864008
:1009600051302DD5104987C00699FF1FE0250E0094
:10097000FFFFEF470000F07F2DE9F04F2DED028BD8
:10098000DFF824A38BB057EC106B55EC114B00F043
:1009900023FB9AF90080B0EE408AF0EE608AB8F14D
:1009A000FF3F48D022462B462046294601F002FF51
:1009B000834600283FD132463B463046394601F057
:1009C000F9FE8146002840F09080304639460022EA
:1009D000002301F0BDFE002836D00022002320466F
:1009E000294601F0B5FE8346B8B19FEDA57B0122F3
:1009F000A94BCDF820900092CDE90267CDE90445DE
:100A00008DED067B0193B8F1000F5BD09FED9E0B3F
:100A10000BB0BDEC028BBDE8F08F45EC104B01F044
:100A20003BF940B1002200232046294601F09AFEFE
:100A3000002840F0C580B0EE480AF0EE680A0BB01E
:100A4000BDEC028BBDE8F08FB0EE480AF0EE680A0C
:100A500001F022F98046002861D04FF000084FF0E5
:100A6000000951EC180B42464B4601F071FE00287C
:100A7000E1D047EC106B01F00FF90028DBD045EC1A
:100A8000104B01F009F90028D5D09AF90030824ABC
:100A9000019204210022022BCDE90267CDE9044531
:100AA000CDE906890091089203D0684601F0FCF870
:100AB00070B901F033FF2223036009E09FED707BE2
:100AC0008DED067B684601F0EFF8002800F08E807F
:100AD000089B1BB101F022FF089B03609DED060BF4
:100AE0000BB0BDEC028BBDE8F08F00220023204646
:100AF000294601F02DFE00289DD09FED630B664B2B
:100B0000CDF820B00122B8F1020FCDE90267CDE99E
:100B100004458DED060B8DE80C00D3D18FE747EC33
:100B2000106B01F0B9F8002897D045EC104B01F09C
:100B3000B3F8002891D053EC182B18EE100A194680
:100B400001F038FE00287CD103239AF9008000933D
:100B5000514B0890CDE90267CDE904450193B8F106
:100B6000000F48D1DFF844914FF060480022002385
:100B700030463946CDE9068901F0F4FD002894D0CD
:100B80000022464B2046294601F07AFB04460D46DA
:100B900045EC104B01F094F8204653EC102B2946FD
:100BA00001F0D6FD002849D13D4B9AF900804FF065
:100BB0006042CDE90623B8F1020F7FF476AF78E703
:100BC000354A9AF90030CDF820B00121CDE902670D
:100BD000CDE904458DE80600002B3FF46FAF3149A5
:100BE0000020022BCDE906017FF46CAF01F096FEE8
:100BF000212303606CE79FED267B00220023304613
:100C000039468DED067B01F0ADFD0028D3D00022E2
:100C1000224B2046294601F033FB04460D4645ECA5
:100C2000104B01F04DF8204653EC102B294601F0F3
:100C30008FFD18B91B4B0022CDE906239AF90080DD
:100C4000B9E7154B9AF90090CDF820800122CDE943
:100C50000267CDE904458DE80C00B9F1000F3FF4BF
:100C60002DAF002200231046194601F033FCB9F1E4
:100C7000020FCDE90601B9D024E700BFAFF3008031
:100C80000000000000000000000000000000F03F35
:100C9000000000000000F07FE4250E000000E03FAF
:100CA000FFFFEFC70000F0FF0699FF1FFFFFEF47B0
:100CB0002DE9F04F55EC104BBD4925F000428A421A
:100CC00083B04FEAD5770DD9BA498A422AD9C5F3FC
:100CD0001303234340F0FA800FB19FED9D0B03B047
:100CE000BDE8F08FB44B9A4200F2D580B34B9A42E4
:100CF00000F2EA8098A3D3E9002310EE100A2946F7
:100D000001F00CF90022AE4B01F04AFD002800F082
:100D10001C81204629460022A94B01F0FFF841EC36
:100D2000100BDCE78EA3D3E9002310EE100A29464E
:100D300001F036FD002840F0D3808BA3D3E90023D7
:100D40002046294601F00EFD0028C6D19D4E88A3FD
:100D5000D3E9002306EBC7062046294601F090FAA6
:100D6000D6E9002301F0DAF801F03AFD064601F079
:100D700021FA81A3D3E900238046894601F080FA55
:100D800002460B462046294601F0C6F87CA3D3E96B
:100D90000023CDE900014046494601F071FA824640
:100DA0008B4652465B46DDE9000101F0B5F804468A
:100DB0000D4622462B462046294601F061FA72A3D1
:100DC000D3E900238046894601F05AFA70A3D3E99B
:100DD000002301F0A1F842464B4601F051FA6EA300
:100DE000D3E9002301F09AF842464B4601F048FA55
:100DF0006BA3D3E9002301F08FF842464B4601F084
:100E00003FFA69A3D3E9002301F088F842464B4634
:100E100001F036FA02460B462046294601F07CF8DE
:100E200080468946002E65D02046294642464B46DC
:100E300001F026FA424604460D464B4600204FF08C
:100E4000804101F069F802460B462046294601F030
:100E500041FB02460B465046594601F05DF8DDE97C
:100E6000002301F059F80B4602465549002001F0D5
:100E700053F86FF47F739E4260DA06F57A7601EBE1
:100E8000065100224FF0B87301F0FAF941EC100B53
:100E900003B0BDE8F08F4C4B9A423FF657AF4B4B37
:100EA0004FEAC7084344D3E9002310EE100A29464D
:100EB00001F032F8464BC7F101069844CDE9000134
:100EC000D8E900ABF61B6CE7002672E710EE102A9B
:100ED0002B462046294601F021F841EC100BFEE696
:100EE0001DA3D3E900231046194601F0C9F941ECCE
:100EF000100BF4E602460B462046294601F0C0F9E5
:100F0000002206460F464FF080434046494601F016
:100F100003F802460B463046394601F0DBFA22461A
:100F20002B4600F0F9FF02460B460020244900F052
:100F3000F3FF41EC100B03B0BDE8F08F01EB06515D
:100F400041EC100B03B0BDE8F08F064631E700BF5F
:100F500000000000000000009C7500883CE4377E23
:100F6000EF39FAFE422E864051302DD5104987C008
:100F7000FE822B654715F73F0000E0FE422EE63F5C
:100F8000763C7935EF39EA3DD0A4BE726937663ECA
:100F9000F16BD2C541BDBB3E2CDE25AF6A56113F79
:100FA00093BDBE166CC1663F3E5555555555C53F60
:100FB000412E8640FFFFEF7F422ED63FFFFF2F3EA0
:100FC0000000F03FE8250E00B1A2F03F08260E0019
:100FD000F8250E00FFFFFFFF2DE9F04F51EC110B3C
:100FE00021F0004858EA000493B03CD053EC102B99
:100FF0006D4E23F00044B44210EE10AA1D462BDCC7
:10100000894611EE10EA26D0B04525DC664EB04583
:1010100077D0002D16461F46CDE9000175DB4FF055
:10102000000BBEF1000F2DD15F4B984500F0898079
:101030005E4B98455ED0B9F1804F00F0DE835C4B8B
:1010400099451FD1002D1DDB47EC106B13B0BDE897
:10105000F04F00F049BD5AB104F1404404F580144A
:1010600054EA0A0306D19FED4A0B13B0BDE8F08F96
:10107000A045CBDD4F4813B0BDE8F04F00F018BEDF
:101080004FF0000B47EC106B00F0FEFD51EC100B25
:10109000BAF1000F1ED0ED0F05F1FF3A5BEA0A032B
:1010A00063D0454B984540F38D8003F10473984518
:1010B00040F33884414B9C4262DDB9F1000F62DDA0
:1010C00035A3D3E900231046194601F0D9F841ECC5
:1010D000100BCAE724B1354B25F040429A42DAD1D1
:1010E000B9F1000FC0F2CB83002DC0F2748341EC44
:1010F000100BBAE7B9F1000FC0F27A8447EC106B1D
:10110000B3E7BEF1000F84D0A6E72D4B984529DC4C
:10111000A3F15473984582DD4FEA2853A3F2FF33BD
:10112000142B40F37F84C3F134032EFA03F202FA46
:1011300003F39E457FF473AF02F00102C2F1020B8C
:101140006FE704F1404303F5801353EA0A038AD0A2
:101150001A4B9C4240F38583B9F1000F13DB9DEDE0
:10116000000B82E74FF0020B5BE732463B4610462E
:10117000194600F0D1FE02460B4601F0ABF9B6E786
:10118000B9F1000F9CDB9FED060B6EE7AFF300801B
:10119000000000000000F03F9C7500883CE4377EB2
:1011A00000000000000000000000F07F0000F03FA1
:1011B0000000E03FA43901000000E041FFFFEF3FE5
:1011C000FFFF3F43B4F5801F4FF0000205DAD64B16
:1011D00001F056F86FF034020C462315D34EC4F3D9
:1011E0001304A3F2FF33134444F07F55B4421A466C
:1011F0000D9345F4401540F34983CD4B9C4240F399
:101200002D849FEDB37B8DED087B8DED0E7B9FEDE7
:10121000B27B13468DED067B01330D93A5F580154A
:101220004FF00008DDE906232946CDE90A0100F068
:1012300073FEDDE9062306460F46DDE90A0100F0EC
:101240006DFE02460B460020BA4901F043F9034601
:101250000C46CDE9103402460B463046394601F0C3
:101260000FF86B1043F0005303F5002303EB080560
:101270000A4600230146CDE902120293DDE9028904
:101280000024CDE904122B4622464046494600F090
:10129000F7FF02460B463046394600F03DFEDDE9D9
:1012A000062306460F462046294600F035FE024634
:1012B0000B46DDE90A0100F02FFE42464B4600F0E6
:1012C000DFFF02460B463046394600F025FEDDE9D9
:1012D000102300F0D5FFDDE90445CDE906012246E3
:1012E0002B462046294600F0CBFF7DA3D3E90023FF
:1012F00004460D4600F0C4FF7BA3D3E9002300F0B1
:101300000DFE22462B4600F0BBFF79A3D3E9002354
:1013100000F004FE22462B4600F0B2FF76A3D3E98C
:10132000002300F0FBFD22462B4600F0A9FF74A32A
:10133000D3E9002300F0F2FD22462B4600F0A0FF87
:1013400071A3D3E9002300F0E9FD224606460F46CB
:101350002B462046294600F093FF02460B463046B6
:10136000394600F08DFF424604460D464B46DDE906
:10137000040100F0D3FDDDE9062300F081FF2246E1
:101380002B4600F0CBFD424606460F464B464046F4
:10139000494600F075FF0022674BCDE90A0100F0D5
:1013A000BDFD32463B4600F0B9FD02980D460446AD
:1013B00022462B464046494600F062FF0022804606
:1013C00089465D4B2046294600F0A6FDDDE90A234B
:1013D00000F0A2FD02460B463046394600F09CFD67
:1013E000DDE9042300F04CFF224606460F462B465B
:1013F000DDE9060100F044FF02460B46304639465F
:1014000000F08CFD06460F4602460B464046494614
:10141000CDE9048900F082FD02983DA3D3E90023C1
:1014200004460D4600F02CFFDDE904238046894682
:101430002046294600F070FD02460B4630463946EC
:1014400000F06AFD34A3D3E9002300F019FF34A3B0
:10145000D3E9002306460F462046294600F010FF38
:1014600002460B463046394600F058FDDDE90E23B2
:1014700000F054FD06460D980F4600F09BFE3246E4
:1014800004460D463B464046494600F047FDDDE92F
:10149000082300F043FD22462B4600F03FFD029852
:1014A00022462B46CDE9020100F036FDDDE9082396
:1014B00000F032FD42464B4600F02EFD02460B4640
:1014C0003046394600F028FD8046894636E000BFA8
:1014D0000000000000000000000000000000F03FDD
:1014E000EF4E454A287ECA3F65DBC9934A86CD3F09
:1014F00001411DA96074D13F4D268F515555D53FEF
:10150000FFAB6FDBB66DDB3F033333333333E33F86
:10151000000000E009C7EE3FFD033ADC09C7EE3FDB
:10152000F5015B14E02F3EBE000040438E9803009F
:1015300079B60B000000F03F000008400BF1FF33CC
:1015400053EA0A0300F088819FEDD77B8DED067B7F
:10155000DDE900AB53465C46CDE90034002300933F
:10156000DDE90045504622462B46594600F0D4FCA2
:10157000DDE9022300F084FE524606460F465B4634
:101580004046494600F07CFE02460B46304639464E
:1015900000F0C4FC2246804689462B46DDE9020164
:1015A000CDE9048900F06CFE0B46024606460F4664
:1015B0004046494600F0B2FCD54B994204460D46E0
:1015C0008A4640F3238101F13F4303F5E0030343DF
:1015D00040F01882B6A3D3E90023DDE9040100F04E
:1015E0009DFC3246804689463B462046294600F00F
:1015F00093FC02460B464046494601F0D1F80028CC
:1016000040F00082A8464FEA28534FF48012A3F21C
:10161000FE3342FA03F35344C3F30A52BD4DA2F220
:10162000FF321541C3F3130B0020C2F1140423EA67
:1016300005014BF4801BBAF1000F02460B464BFA32
:1016400004FB30463946B8BFCBF1000B00F064FC18
:1016500002460B4606460F46DDE9040100F05EFC3B
:101660004FEA0B5A002494A3D3E9002320460D46E9
:1016700000F006FE3246804689463B462046294613
:1016800000F04AFC02460B46DDE9040100F044FC90
:101690008BA3D3E9002300F0F3FD8BA3D3E9002350
:1016A00006460F462046294600F0EAFD02460B4654
:1016B0003046394600F032FC06460F4602460B46DD
:1016C0004046494600F02AFC42464B4604460D4639
:1016D00000F022FC02460B463046394600F01CFC66
:1016E0002246804689462B462046294600F0C8FD02
:1016F00077A3D3E9002306460F4600F0C1FD76A389
:10170000D3E9002300F008FC32463B4600F0B8FD68
:1017100073A3D3E9002300F001FC32463B4600F0FE
:10172000AFFD71A3D3E9002300F0F6FB32463B4640
:1017300000F0A6FD6EA3D3E9002300F0EFFB3246D4
:101740003B4600F09DFD02460B462046294600F030
:10175000E3FB06460F4602460B462046294600F0AC
:101760008FFD0022CDE900014FF08043304639461D
:1017700000F0D2FB02460B46DDE9000100F0AAFEB4
:10178000424606460F464B462046294600F078FD65
:1017900042464B4600F0C2FB02460B4630463946F5
:1017A00000F0BAFB22462B4600F0B6FB02460B4681
:1017B0000020594900F0B0FB8A44BAF5801F024668
:1017C0000B46C0F25B815146DDE9062300F058FD6F
:1017D00041EC100B49E404F1404404F5801454EA50
:1017E0000B0300F03781BBF1010F7FF480AC0246A0
:1017F00001F1004343EC102B37E432463B463046C0
:10180000394600F03DFD41EC100B2EE4434B21F036
:101810000048984540F31581414B0B4403430CD1DC
:1018200032463B4600F078FB02460B46DDE90401F8
:1018300000F0A2FF00283FF4E6AE2FA3D3E9002377
:10184000DDE9060100F01CFD2BA3D3E9002300F025
:1018500017FD41EC100B08E49FED297B8DED067B15
:1018600076E6B9F1000FBFF68EACDDE9003400EE8C
:10187000103A04F1004300EE903AFFF7F6BB02463F
:101880000B460020244900F025FE2DE49FED1E7B31
:101890008DED087B8DED0E7B9FED037B4FF00008F7
:1018A0008DED067BBEE400BF000000000000F03FAD
:1018B000FE822B654715973C00000000432EE63F53
:1018C000EF39FAFE422EE63F396CA80C615C20BE6F
:1018D000D0A4BE726937663EF16BD2C541BDBB3E36
:1018E0002CDE25AF6A56113F93BDBE166CC1663F14
:1018F0003E5555555555C53F59F3F8C21F6EA501C4
:10190000000000000000F0BF000000000000000028
:10191000FFFF8F40FFFF0F000000F03FFFCB904024
:1019200000346F3F6C4B9C427FF72AAC6B4B9C4260
:101930003FF7C3AB0022694B00F0EEFA56A3D3E9A0
:10194000002304460D4600F09BFC55A3D3E9002379
:10195000804689462046294600F092FC0022CDE9C7
:1019600002015F4B2046294600F08AFC02460B46E6
:101970004DA1D1E9000100F0CFFA22462B4600F03C
:101980007FFC02460B460020564900F0C5FA22466D
:101990002B4606460F462046294600F071FC0246BB
:1019A0000B463046394600F06BFC41A3D3E90023D7
:1019B00000F066FC02460B46DDE9020100F0ACFADD
:1019C00002460B4604460D464046494600F0A6FA3C
:1019D00042464B460020CDE9020100F09DFA024646
:1019E0000B462046294600F097FA80468946A5E531
:1019F00032463B460020394900F06CFD41EC100BAB
:101A0000FFF733BB2CA3D3E90023DDE9060100F087
:101A100037FC29A3D3E9002300F032FC41EC100B82
:101A2000FFF723BBBEF1000F7FF42AABC3F1140311
:101A300048FA03F202FA03F3984527D0F346FFF77A
:101A4000F7BA284B98453FF7DEADDDE900349A46FA
:101A50009B4607E602460B46FFF789BB9FED187BC6
:101A60008DED087B9FED187B8DED0E7B9FED187B38
:101A70004FF480288DED067BFFF7D4BB584643EC2E
:101A8000102B00F0B1F951EC100B9DE602F00102B1
:101A9000C2F1020BFFF7CCBA000000604715F73F18
:101AA00044DF5DF80BAE543E555555555555D53F61
:101AB000FE822B654715F73F9C7500883CE4377E16
:101AC0000000004003B8E23F06D0CF43EBFD4C3EA0
:101AD000000000000000F83FFEFFEF3F0000F03F75
:101AE0000000D03F0000E03F2DE9F041654955EC92
:101AF000104B0E462940B14200F09780002D2B4636
:101B000010EE102A74DD2F157FD0A7F2FF37C3F334
:101B10001303F90743F4801365D403EBD271002655
:101B20000B447F105200B64616204FF400110EEB06
:101B300001049C424FEAD2754FEA420203DC1B1BB0
:101B400004EB010E0E44013805EB43034FEA51014B
:101B5000EDD1844620244FF0004109E020D003EB72
:101B6000D275013C4FEA51012B444FEA420220D08A
:101B70009E4501EB0C05F1DA002D05EB010C09DBAC
:101B8000F0469542CEEB030300D9013B521B0844BB
:101B9000C646E4E7BCF1000FF2DB0EF10108F0E706
:101BA00095421ED8002D05EB010C50DB9846002312
:101BB000ECE7134304D0421C4DD000F0010318445D
:101BC00040087110F30701F17F5101F5001148BF82
:101BD00040F0004001EB0753024643EC102BBDE8F8
:101BE000F0817346BBE75B0003EBD273520094E7CE
:101BF00025F00041214328D0ADBB2F46D30A153F25
:101C00005205002BFAD0DD0228D4002100E0014665
:101C10005B00DC0201F10100F9D5C0F1200422FAD9
:101C200004F423437F1A82406FE710EE102A2B46FC
:101C300010EE100A294600F023FB22462B4600F046
:101C40006DF941EC100BBDE8F081BDE8F081BCF10D
:101C5000000FA2DAAAE701362046B2E720244FF0AF
:101C6000FF310020DBE710EE102A2B4620462946E4
:101C700000F052F902460B4600F02CFC41EC100B30
:101C8000BDE8F0810000F07F53EC102B23F00043FF
:101C900043EC102B704700BF10EE903A43F0004029
:101CA00000F58010C00F704700207047FFFFFFFF56
:101CB0009FED010B704700BF000000000000F87F9F
:101CC000F0B553EC102BC3F30A56A6F2FF301328DD
:101CD00083B019464FEAD37410EE105A2FDC002857
:101CE00049DB3F4E064103EA060717432CD076082E
:101CF00033401D430CD04FF48023132821EA0606FD
:101D000043FA00F141EA06010CBF4FF000450025FF
:101D1000344800EBC4042A46D4E9004510462B465B
:101D2000224600F0FBF8CDE9000122462B46DDE912
:101D3000000100F0F1F841EC100B03B0F0BD3328C6
:101D400006DDB0F5806F42D043EC102B03B0F0BD40
:101D5000A6F213464FF0FF30F0400242F4D04008A4
:101D60000242D5D04FF0804325EA000043FA06F640
:101D700046EA0005CCE723F00040104310EE107A4D
:101D8000E2D0C3F313000743784207431548590CC8
:101D90003F0B490407F4002700EBC40047EA0103A6
:101DA000D0E90067194610463B46324600F0B6F8C7
:101DB000CDE900013B463246DDE9000100F0ACF818
:101DC00021F0004343EAC47141EC100BBEE710EE72
:101DD000100A194600F0A2F841EC100BB6E700BF5C
:101DE000FFFF0F0018260E0053EC102B70B5C3F345
:101DF0000A541946054614BB23F0004111432AD06A
:101E000019460022384B394E10EE100A00F038FA0D
:101E1000B54202460B461FDBC1F30A54363C2C4444
:101E200040F2FE7084421FDC002C2DDD21F0FF41CA
